:020000040800F2
:1080000020DE002051100108198300081B8300089E
:108010001D8300081F830008218300080000000062
:10802000000000000000000000000000598200086D
:1080300025830008000000008D820008B18101083E
:108040006B1001086B1001086B1001086B10010820
:108050006B1001086B1001086B1001086B10010810
:108060006B1001086B1001086B1001086B10010800
:108070006B1001086B1001086B1001086B100108F0
:108080006B1001086B1001086B1001086B100108E0
:108090006B1001086B1001086B1001086B100108D0
:1080A0006B1001086B1001086B1001086B100108C0
:1080B0006B1001086B1001086B1001086B100108B0
:1080C0006B1001086B1001086B1001086B100108A0
:1080D0006B1001085B8501086B1001086B1001082B
:1080E0006B1001086B1001086B1001086B10010880
:1080F0006B1001086B1001086B1001086B10010870
:108100006B1001086B1001086B1001086B1001085F
:108110007B8701086B100108693901086B100108A1
:108120006B1001086B1001086B1001086B1001083F
:1081300000F002F800F080F80AA090E8000C8244F9
:108140008344AAF10107DA4501D100F075F8AFF2D6
:10815000090EBAE80F0013F0010F18BFFB1A43F025
:1081600001031847F8890300188A03000A444FF0F6
:10817000000C10F8013B13F0070408BF10F8014B86
:108180001D1108BF10F8015B641E05D010F8016BCB
:10819000641E01F8016BF9D113F0080F1EBF10F82F
:1081A000014BAD1C0C1B09D16D1E58BF01F801CB52
:1081B000FAD505E014F8016B01F8016B6D1EF9D5D5
:1081C0009142D6D3704700000023002400250026EA
:1081D000103A28BF78C1FBD8520728BF30C148BF2A
:1081E0000B607047642924F04181732924F0B7841F
:1081F0000020704710B510BD70477047704770473A
:1082000054656D636F545354415438000000006549
:10821000000000671FB524F0B0FA24F08DFD0400C3
:108220000020002126F046FB401C60600020002159
:1082300026F056FBE0601FBD24F046FF1146FFF715
:10824000E9FF02F0E6FA25F0B7F903B4FFF7D2FF31
:1082500003BC10F03DF800001A4B19680868B0E83C
:10826000F00F80F309884FF0000080F311884EF082
:108270000D0E70470000000003480068006880F39E
:10828000088862B600DF00BF08ED00E0EFF3098068
:108290000C4B1A6820E9F00F106008B54FF0BF00D2
:1082A00080F311880FF047FD4FF0000080F3118834
:1082B000BDE8084019680868B0E8F00F80F3098845
:1082C000704700BFAC02002001B44FF0BF0080F344
:1082D000118801BC704701B44FF0000080F3118891
:1082E00001BC70470B49D1F800C04A685CF8043BF8
:1082F0001068184442F8040B8C4528BFA1F1DC0C2F
:108300008A4228BFA1F1DC02C1F800C04A6020F017
:1083100000407047B4D700207047FEE7FEE7FEE755
:10832000FEE7704770477047704700000CB50022A9
:10833000019200925248016841F4803101604FF48B
:10834000A063016801F4003100910199491C019179
:10835000009911B901999942F3D10168890302D5B5
:108360000121009100E000920099012930D1454996
:108370000A6842F010020A600A6822F003020A60EA
:108380000A6842F002020A60416841604168416047
:10839000416841F480614160416821F47C11416091
:1083A000416841F4E8114160016841F08071016069
:1083B00001688901FCD5416821F0030141604168F1
:1083C00041F0020141604168C1F381010229FAD103
:1083D0000CBDABE710B52A48016841F0010101600E
:1083E0004168294A114041600168284A11400160F2
:1083F000016821F480210160416821F4FE0141609F
:108400004FF41F018160FFF7E4FF21494FF0006046
:10841000086010BD10B51A4A506800F00C011D4BE1
:108420001D4800290ED004290ED008290ED0036063
:108430005168194AC1F30311121D515C0268CA4008
:10844000026010BD0360F3E70360F1E7516801F4D7
:108450007011536803F48033022404EB914133B16B
:1084600053689B0307D50D4B59430160E0E70B4B65
:1084700059430160DCE7074B59430160D8E700002E
:1084800000100240002002400000FFF8FFFFF6FE4F
:1084900008ED00E000127A001400002000093D0001
:1084A0009A48994941609A494160704797480169E3
:1084B00041F08001016170479448C068C10701D054
:1084C00001207047410701D502207047C00601D541
:1084D000032070470020704770B50446FFF7ECFF9B
:1084E0000546012D05D10FF0D3FF641EA4B2002C68
:1084F000F4D104B9FF25284670BD70B5054645F690
:10850000FF763046FFF7E8FF002812D17F4C206944
:1085100040F0020020616561206940F04000206168
:108520003046FFF7D9FF012803D0216921F002016D
:10853000216170BD70B506460D46FF20FFF7CCFFE8
:1085400000280ED1714C206940F001002061358077
:10855000FF20FFF7C1FF012803D0216921F00101AD
:10856000216170BD008870472DE9F04105460E4637
:108570001746002407E036F814102846FFF7DAFF04
:10858000AD1C641CA4B2BC42F5D3BDE8F081C107A8
:1085900003D030F8010C000A70470088C0B2704761
:1085A00010B50446002307E02046FFF7DBFF21F863
:1085B0001300A41C5B1C9BB29342F5D310BD2DE9A4
:1085C000F05F82460F461546AAF10062B2F5002F11
:1085D00052D2FFF765FF4FEAD228C2F34906C6F52B
:1085E0008064A54200D82C46DFF828B137E0321865
:1085F0003BF812208A4203D1401C80B2A042F6D33D
:10860000A04214D24846FFF778FF002006E0821906
:1086100037F810102BF81210401C80B2A042F6D38D
:1086200048464FF480623B49FFF79EFF04E0224634
:1086300039465046FFF798FFA54202D1BDE8F05FEA
:1086400034E708F10108002607EB44070AEB440A67
:10865000281B85B24FF48064A54200D82C464FF009
:10866000006000EBC82942142A494846FFF798FFEA
:1086700000204FF6FF71C1E7BDE8F09F30B504461A
:108680000D46002306E02046FFF781FFE854641CF6
:108690005B1C9BB29342F6D330BD70472DE9F04787
:1086A000ADF5006D0D46904600240746A0F1006030
:1086B000B0F5002F23D200264FF48069EA4615E07A
:1086C0006878000215F8021B08442146641CA4B215
:1086D0002AF811004A46944206D1002469463846D9
:1086E000FFF742FF07F50067B61CB6B24645E7D371
:1086F000002C04D0224669463846FFF735FF0DF5B9
:10870000006DBDE8F08700002301674500200240AE
:10871000AB89EFCD8C0900202A4908432A4908601B
:10872000704770B50F23C27801260178002A1ED049
:10873000254A126802F4E062C2F5E062120AC2F150
:108740000404D3404578A54082781A402A43120198
:1087500001F1E02181F80024007800F01F018E4033
:108760004009800000F1E020C0F8006170BD01F018
:108770001F0086404809800000F1E020C0F88061B9
:1087800070BD124A114001430F48001F016070473D
:108790000D4A121D002903D0116801431160704772
:1087A00011688143116070474FF0E021042804D024
:1087B000086920F0040008617047086940F004006F
:1087C000086170470000FA050CED00E080FFFF1F14
:1087D00010B5DB4988420AD144150121204607F033
:1087E000D0FA2046BDE81040002107F0CABAD549AA
:1087F00088420AD104150121204607F0C2FA20461A
:10880000BDE81040002107F0BCBACF4988420AD128
:108810000121CC03204607F0B4FA2046BDE8104001
:10882000002107F0AEBA10BD10B54268C74B1A4020
:108830000C790B6842EA0422134343608268C44BFC
:108840001A40D1E9024323434C7942EA44021343DC
:108850008360C26A22F47002097C491EC9B242EAEE
:108860000151C16210BD002101600171417181603F
:10887000C160012101747047002904D0816841F072
:10888000010181607047816821F0010181607047BA
:10889000002904D0816841F480718160704781684B
:1088A00021F4807181607047C9B2002A03D0426808
:1088B0000A434260704742688A4342607047816859
:1088C00041F008018160704701460020896809076E
:1088D00000D501207047816841F004018160704734
:1088E000014600208968490700D50120704700290A
:1088F00004D0816841F4A00181607047816821F44F
:10890000A00181607047014600208968490200D5B6
:1089100001207047426822F46042491E42EA413118
:1089200041607047002904D0416841F40061416012
:108930007047416821F400614160704770B50726B7
:1089400009290AD9C568A1F10A0404EB4404A64028
:10895000B543A3401D43C56007E0056901EB410431
:10896000A640B543A3401D4305611F23072A09D232
:10897000446B521E02EB820293409C4391400C4395
:10898000446370BD0D2A09D2046BD21F02EB820230
:1089900093409C4391400C43046370BDC46A0D3AFC
:1089A00002EB820293409C4391400C43C46270BD31
:1089B000002904D0816841F480118160704781688A
:1089C00021F4801181607047C06C80B270475C48B0
:1089D0004C3000687047002904D0416841F4806140
:1089E00041607047416821F480614160704700290F
:1089F00004D0416841F4805141607047416821F4DE
:108A0000805141607047826822F4E0420A438260EC
:108A10007047002904D0816841F4004181607047AB
:108A2000816821F4004181607047002904D0816889
:108A300041F4021181607047816821F40211816064
:108A40007047014600208968890200D501207047DF
:108A500070B5072609290AD9C568A1F10A0404EBF3
:108A60004404A640B543A3401D43C56007E0056923
:108A700001EB4104A640B543A3401D430561836B50
:108A8000C3F30154121B921C02EB82021F24944078
:108A9000A34391400B43836370BD826B22F4401269
:108AA000491E42EA01518163704708B50090009861
:108AB000084400900098026008BD08B50090009836
:108AC0000844283000900098006880B208BD4268D1
:108AD000204B1A400A4342607047416282627047ED
:108AE000426822F01F020A4342607047144908316D
:108AF000002804D0086840F4000008607047086847
:108B000020F40000086070470246002012680A4204
:108B100000D001207047C9430160704710B502467C
:108B200000200B0A5468C9B20C401168194202D0E7
:108B3000002C00D0012010BD090AC9430160704714
:108B40000024014000280140003C0140FFFEF0FFEE
:108B5000FDF7F1FFFFFD3FFF01684FF6FE72114088
:108B600001600021016041608160C1607249724A08
:108B70000839904204D1486840F00F0048607047BF
:108B80006D4A1432904204D1486840F0F0004860C9
:108B90007047694A2832904204D1486840F47060B6
:108BA00048607047644A3C32904204D1486840F4BF
:108BB000704048607047604A5032904204D1486823
:108BC00040F47020486070475B4A6432904204D1A0
:108BD000486840F4700048607047574A78329042C5
:108BE00004D1486840F0706048607047534A111FD4
:108BF000904204D1086840F00F00086070474F4A67
:108C00001432904204D1086840F0F00008607047C8
:108C10004A4A2832904204D1086840F470600860E3
:108C20007047464A3C32904204D1086840F4704094
:108C300008607047414A50329042FAD1086840F4C7
:108C400070200860704730B5026847F6F0739A43A9
:108C50000C6A8B682343D1E904452C4323438C6978
:108C60002343CC6923434C6A23438C6A2343134335
:108C70000360CA6842600A6882604968C16030BDAA
:108C80000021016041608160C160016141618161D9
:108C9000C1610162416281627047002904D00168AC
:108CA00041F001010160704701684FF6FE7211400A
:108CB00001607047002A03D002680A4302607047CF
:108CC00002688A430260704741607047406880B222
:108CD000704702460020D10003D5184908390968B9
:108CE00002E0154908390968114200D00120704797
:108CF000C10003D51149091F086070470E490839A2
:108D00004860704702460020D10003D50B4908395E
:108D1000096802E0084908390968114200D00120B9
:108D20007047C10003D50549091F08607047024913
:108D300008394860704700000800024008040240FB
:108D400010B59C49884209D10121042007F019F887
:108D50000021BDE81040042007F013B8964988426E
:108D600009D10121082007F00CF80021BDE81040CE
:108D7000082007F006B89149884209D10121102046
:108D800006F0FFFF0021BDE81040102006F0F9BFFB
:108D90008B49884209D10121202006F0F2FF0021F1
:108DA000BDE81040202006F0ECBF8649884209D17A
:108DB0000121402006F0E5FF0021BDE810404020E1
:108DC00006F0DFBF8049884209D10121802006F0EA
:108DD000D8FF0021BDE81040802006F0D2BF7B49BB
:108DE00088420AD184150121204606F0CAFF204698
:108DF000BDE81040002106F0C4BF10BD10B5012130
:108E0000084606F0BEFF0021BDE81040012006F034
:108E1000B8BF2DE9F0410022CC7804F00F03E4063E
:108E200001D58C7823430C784FF00F0714F0FF0F17
:108E30004FF0010C1CD005680CFA02F40E88264095
:108E4000A64211D1960007FA06F825EA080503FAAA
:108E500006F848EA0505CE78282E02D0482E02D022
:108E600002E0446100E00461521C082AE4D305607A
:108E70000A88FF2A1ED94568002202F108060CFA6A
:108E800006F40E882640A64210D1960007FA06F88E
:108E900025EA080503FA06F848EA0505CE78282EE3
:108EA00000D14461CE78482E00D10461521C082ABA
:108EB000E3D34560BDE8F0814FF6FF7101800221E8
:108EC00081700421C17070470246002092680A42F6
:108ED00000D001207047806880B2704702460020B1
:108EE000D2680A4200D001207047C06880B2704743
:108EF0000161704741617047002A01D001617047EC
:108F000041617047C160704741F480328261816184
:108F1000826181698069704710B52D4B1A684FF6E0
:108F20008074224042EA00100843186010BD2949AD
:108F3000C8617047F0B5264C002801DAE36900E00B
:108F40006368C0F30346420D120185B2C0F30157B6
:108F50009540032F07D0C2020CD50322B2409343A1
:108F600043F0706209E023F07062636823F070637D
:108F7000636002E0AB4343F0706201B12A43002812
:108F800001DAE261F0BD6260F0BD10B58A07120F30
:108F90000F23934021F003040D4921448C689C4326
:108FA0008C608B68904003438B6010BD0949DC31B5
:108FB0000860704700080140000C014000100140AB
:108FC0000014014000180140001C01400020014035
:108FD00000000140000020420FB41CB5074B06AA58
:108FE0007B4469460090059823F08FFD0020694678
:108FF00023F09EFD1CBC5DF814FB00004D3B0200FD
:109000000000000000000000000000000000000060
:109010000000000000000000000000000000000050
:10902000FD4A01211160FD49087001200FF0DDBBF0
:1090300010B5FB48012404701AF07CF8F948C068A8
:109040001AF07FF8F84902200870F848047010BD43
:10905000012080F31388F6480168F64A01F4E061C4
:1090600011430160BFF3408FFEE7F0B587B00121E7
:10907000202006F070FE0121042006F06CFE012184
:10908000102006F068FE0121082006F064FE012190
:10909000402006F060FEE84810250224007AE74EE2
:1090A00004280BD34020ADF818008DF81B508DF824
:1090B0001A4006A9E248FFF7ACFE0AE00420ADF82A
:1090C00018008DF81B508DF81A4006A93046FFF79E
:1090D000A0FE4FF40040ADF814008DF817508DF845
:1090E0001640374605A93846FFF793FEADF8104005
:1090F0008DF813508DF8124004A93846FFF789FE09
:109100000820ADF80C008DF80F508DF80E4003A923
:109110003846FFF77EFE0126ADF808608DF80B504B
:109120008DF80A4002A93846FFF773FEADF80460D7
:109130008DF807508DF8064001A9C248FFF769FE77
:1091400007B0F0BD10B545F2555006F0C3FC052040
:1091500006F0C3FC4FF47A6006F0C2FC06F0C8FCCF
:10916000BDE8104006F0BFBC06F0BDBC2DE9F84FCD
:1091700040F2053008F033FBB349087040F2F625A1
:10918000284608F02CFB6C1EFF2807D1002128463A
:1091900008F026FB6421204608F022FB204608F058
:1091A0001EFB0446284608F01AFBA84904EB0020E1
:1091B0000880A14F012697F8F302012806D987F805
:1091C000F362012140F2F32008F00AFBA0495E207F
:1091D00008800021942008F003FB40F2D32008F01F
:1091E000FEFA04464FF4357008F0F9FA994904EB99
:1091F00000200881072008F0F2FAFF2804D0082098
:1092000008F0EDFAFF2803D10921072008F0E8FA59
:1092100040F2625008F0E3FA044640F2645008F06D
:10922000DEFA8D4904EB0020088040F263542046AA
:1092300008F0D5FA89490870012804D90E70012177
:10924000204608F0CDFA78790025FF282ED102F0CB
:10925000FFF90021052008F0C3FA6521042008F079
:10926000BFFA01F0B8FC87F8DA50787A00F03F01D5
:109270007972092008F0B4FA0024002104F5A170E5
:1092800008F0AEFA641CE4B2072CF6D300240021E7
:1092900004F2491008F0A4FA641CE4B2072CF6D3D7
:1092A00097F86E00012801D987F86E5040F29C446F
:1092B000204608F094FA6A4908704FF0FE0AFF2829
:1092C00001D0012805D881F800A05146204608F0B9
:1092D00087FA97F85902FF2808D197F85A02FF2811
:1092E00004D1C82087F8590287F85A5297F87800B5
:1092F000DFF8708138B10421012812D0022820D073
:1093000003282AD124E0294687F89B509B2008F0A7
:1093100067FA314688F8006040F2673008F060FA7A
:109320001BE097F89B0020B987F89B109B2008F062
:1093300057FA294688F8005040F2673008F050FA92
:109340000BE040F2673008F04AFA88F8000004E0C9
:1093500087F89B109B2008F043FA43480570434967
:1093600097F89B0008704249087008B141480670A0
:10937000DFF8049199F8000016F005FD3F490880D8
:1093800099F800203E483F4932B197F86C2002809E
:1093900097F86D00088005E097F87120028097F833
:1093A000700008804FF0000B002404F1B900009019
:1093B00008F015FA30B1009808F011FA032801D22C
:1093C0004FF0010B641CE4B2052CEED32E48BBF128
:1093D000010F05D0057097F8CC002C4910B10AE0B8
:1093E0000670F8E797F8CB0028B997F8CE0010B9C7
:1093F00097F8CD0078B12648057017F8CD0F7A7828
:1094000000EB0220234A80B21080BA7BCD3F032AB2
:1094100047D00E7040E049E0A0012142547B00207B
:109420008C060020000000209A06002098060020EC
:109430000CED00E00400FA05607F002000140140FC
:10944000000C014000080140B2030020640000202D
:10945000480000202C120020C60300201903002021
:109460005C0400207B000020B10300206E0000207F
:109470003B000020680000203A000020540000203B
:10948000B4030020B6030020780000207E000020F6
:109490008C0000209600002097F8D310012204F0E1
:1094A0001DFDB879FF2803D010B111E00D70F8E769
:1094B00087F806A087F8F352FE48A0F800A00146FE
:1094C0000122FD48FFF77BF8B979062008F088F9FA
:1094D0004FF42E7B584608F082F987F8B8020C2822
:1094E00005D987F8B8520021584608F079F997F85D
:1094F000D902012806D987F8D952002140F2D92093
:1095000008F06EF997F8DC02012806D987F8DC52DA
:1095100000214FF4377008F063F900244FF0030A7C
:10952000381990F8F710FF2906D180F8F7A0032129
:1095300004F1F70008F054F9641CE4B2082CEFD3EE
:1095400097F8B802192805D987F8B852002158466B
:1095500008F046F9012008E0391891F8BA22FF2AEC
:1095600001D181F8BA52401CC0B297F8B812491C18
:109570008142F1D8D1490D8097F80201FF2803D12B
:1095800097F80121FF2A05D02843000297F801210E
:1095900002430A801B2008F022F904461C2008F030
:1095A0001EF904EB002A2F2008F019F90446302098
:1095B00008F015F904EB0020C14C824501D2267059
:1095C00000E02570312008F00AF98246322008F0C8
:1095D00006F90AEB002B452008F001F982464620E7
:1095E00008F0FDF80AEB0020834501D2667000E028
:1095F000657040F2673008F0F2F888F80000012842
:1096000001D988F8006097F86103B8B997F8E100CC
:1096100097F87E10884203D397F87D1088420DD9C1
:10962000C8203C4687F8E100C821E12008F0D8F8BE
:1096300094F8591294F85A0216F0ADFBF62008F08F
:10964000CEF887F8F6009F48017841F007010170D5
:109650009D48007810B3787A40F00100787289F85C
:109660000060787A00F0FB017972092008F0B8F800
:109670007B2023F06DF840F25324204608F0AFF829
:10968000022803D90021204608F0AAF840F2EF246E
:10969000204608F0A4F8FF2807D00AE0787A00F006
:1096A000FE00787289F80050DBE70021204608F0C0
:1096B00097F808F0E1F885488088002806D1BDE8D1
:1096C000F84F40F2E171842001F046BEBDE8F88F0A
:1096D00010B501210D2006F03EFBBDE81040012130
:1096E0007B48FFF727BC2DE9F0410024794800268C
:1096F0000682794D744995F89B000870774F0121D7
:109700003970704B07221A7085F87A63C82285F881
:109710007B2395F87F20012A01D9714A117095F8B1
:10972000B932704A0BB980B11170107816F02BFB6A
:109730006D4908803A786D486D494AB195F86C20BA
:10974000028095F86D00088008E004201070ECE7B6
:1097500095F87120028095F87000088095F89210B5
:109760006448012905D00321817195F8D80010B112
:1097700003E08671F9E76048067015F0D9FE5F488E
:10978000291991F8B2100155641CE4B2072CF7D3E3
:10979000BDE8F08110B501F01EFAFFF7E5FCBDE869
:1097A0001040A0E7564800240470564804704FF457
:1097B000FA600EF08DFEFFF78BFF07F069FC524850
:1097C000047007F0D8FC14200EF082FEF9E74F4D2C
:1097D000DFF83C91DFF83C814F4EDFF840A1DFF825
:1097E00040B1504F00247C71B8F800207979CA400C
:1097F000D00702D0685C401C6854685C06280FD310
:109800006C5419F8010010B1401E09F8010019F854
:10981000010028B9D00703D000223E4801F053F9D7
:109820007879401CC0B278710328DDD37C71BBF815
:1098300000207979CA40D00702D0705C401C705477
:10984000705C06280FD374541AF8010010B1401E42
:109850000AF801001AF8010028B9D00703D0002245
:109860002F4801F030F97879401CC0B27871032894
:10987000DDD342F210700EF02BFEB4E786B0FFF796
:10988000D7FB00201AF002FA00201BF0D5FB264877
:1098900015F076F825491420087025490B2008702A
:1098A000244902200870244905200870234C002513
:1098B000104E45E0500000200077000870020020A4
:1098C00074020020390000203B0000208C11002091
:1098D0000004300004120020607F00203A000020C5
:1098E000340000203700002054000020B403002082
:1098F000B6030020961600205A000020C400002065
:10990000FC000020F3000020F7000020D50000201C
:109910009E00002086000020D20000209B00002036
:109920008800002000000020A88200207D04002084
:109930007A0400207B0400207E0400200F03002016
:1099400020780C2802D1FFF773FB257020781328AC
:1099500008D1FFF76DFB00201AF098F900201BF0EA
:109960006BFB2570B07978B9757000234FF41672CF
:10997000FE4901A8009519F09EFB024622B1002382
:10998000FA4901A81BF0E9FA05200EF0A1FD90E7C5
:109990000026F74801240470F64F97F8D8000028F5
:1099A00004D0C0EB00108100F3480180DFF8CCB395
:1099B0000025DFF8CC83FFF7D7FBF249087808B120
:1099C000401E0870087808B9EF480570DFF8BC93AE
:1099D00099F800000D280AD13878ABF800007878A3
:1099E000ABF802000222E549E948FEF7E8FD99F8E4
:1099F00000000E280BD1B878ABF80000F878ABF86F
:109A00000200E3480222DD491030FEF7D8FDE14AAA
:109A10001078012803D1E0490878401C0870DE481E
:109A20000178052901D915700570DC4908780128ED
:109A300006D1887918B1CD71401E887100E0CC71D3
:109A4000D7490878012806D1887918B1CD71401E10
:109A5000887100E0CC71D3490878012806D1887953
:109A600018B1CD71401E887100E0CC71CE490878E4
:109A7000012806D1887918B1CD71401E887100E0A7
:109A8000CC71CA490878012806D1887918B1CD71FE
:109A9000401E887100E0CC7197F8D80050B1B649EB
:109AA000088808B1401E0880C1480988027811431F
:109AB00000D10470761CF6B23C2E07D397F85C03F5
:109AC00018B1BC480178491E01700026B9480078D9
:109AD00030B997F85C0318B187F85C53B6488470C6
:109AE00099F80000102803D189F8005001F0B0FD6A
:109AF00099F80000112809D003F01DFEAF49088035
:109B0000DFF8BCA2DAF80000B8B121E09F48057088
:109B100014244FF45A7640F26C75B44205D0652C8B
:109B200003D0FF21204607F05BFE641CA4B2AC42C8
:109B3000F3D301F08DFDFFF78BFA97F8B90238B136
:109B400003F002FF88F8044088F8024088F80140DA
:109B50009C4A107801280CD19B490878401CC0B25F
:109B60000870052805D115700D7002F03BFE924873
:109B70008470DAF8000098B197F8631081B1401E44
:109B8000CAF8000060B99B2007F029FE8F490870D1
:109B900087F89B008E49087088F802408648457017
:109BA0008C490888012801D9401E08808A49088804
:109BB00008B1401E0880088838B997F8ED00FF28E2
:109BC00003D001218548FFF795F997F8ED00FF28AC
:109BD00003D101218148FFF78BF98149087818B139
:109BE00088F80140401E08707E49087818B188F84E
:109BF0000240401E0870087858B97B480470DFF8AE
:109C0000ECA19AF80000012801D102F04CFA8AF880
:109C100000507749087818B1401E087088F8034052
:109C20007449087808B1401E0870087878B97248FD
:109C3000017801290BD105700F2089F8000088F800
:109C4000014088F8024088F805406C4805706C496E
:109C50000888401E80B2088008B96A480470DFF89E
:109C6000A89199F8000010B1401E89F8000099F8F9
:109C7000000020B900220121644800F024FF99F877
:109C8000010010B1401E89F8010099F8010020B9C7
:109C9000002203215D4800F016FF99F8020010B180
:109CA000401E89F8020099F8020020B9002205211F
:109CB000564800F008FF99F8030010B1401E89F8DB
:109CC000030099F8030020B9002207214F4800F053
:109CD000FAFE99F8040010B1401E89F8040099F8C2
:109CE000040020B900220921484800F0ECFE99F850
:109CF000050010B1401E89F8050099F8050020B94B
:109D000000220B21414800F0DEFE99F8060010B158
:109D1000401E89F8060099F8060020B900220D219E
:109D20003A4800F0D0FE4FF47A700EF0D1FB42E6D4
:109D30000EB513484FF0010880F8008080F80180CC
:109D400080F8028080F8038080F8048080F8068024
:109D500001212248FFF7CCF82E492D4808601B4806
:109D600001781B48017047F6176055E0F0060020A7
:109D700028000020607F00205C00002050000020B0
:109D80009611002009030020080300200F03002083
:109D9000107700081303002014030020AE110020E8
:109DA000B8110020C2110020D6110020CC110020D3
:109DB0005A0000200E030020000000204400002074
:109DC0004C00002069000020660000203B000020BD
:109DD0002C000020200300203E000020000801404D
:109DE00030000020310000206A0000202D000020FB
:109DF00032000020EE000020EF000020F0000020E4
:109E000060000020620000209802002096020020DE
:109E100008010020040100204FF6FF76ED21CDE976
:109E20000016002302901A462421F02008F0F0F8D2
:109E300047F61965CDE9016538200E210090C82349
:109E4000FB4A084608F0C8F86921662009F03EF888
:109E50009421662009F03AF8BF21662009F036F80F
:109E6000CDE90065F3A36C220A21012008F09AF8DD
:109E7000CDE90065F0A397220A21012008F092F8AD
:109E8000CDE90065EDA3C2220A21012008F08AF87D
:109E9000EB4F0024DFF8ACA39AF80600401CC0B2D8
:109EA0008AF80600052801D98AF80640DFF8989359
:109EB00099F8000001285BD0022868D004287FD0E0
:109EC000052877D00728FCD0062874D00828FCD0B5
:109ED0000B2871D00F2870D0DC49087800286DD08D
:109EE00000200870DA490978012968D09AF8020040
:109EF00080B308F038FED74880F8018080F80280EF
:109F000080F8038080F804806921662008F0DEFF75
:109F10009421662008F0DAFFBF21662008F0D6FF02
:109F2000CDE90065C3A36C220A21012008F03AF8AC
:109F3000CDE90065C0A397220A21012008F032F87C
:109F4000CDE90065BDA3C2220A21012008F02AF84C
:109F50008AF80240C0490878002870D000200870B4
:109F6000BE4880F800809AF80600052868D0DFE037
:109F7000284607F05CFECDE900651E22B8A3114615
:109F8000012008F00FF80EF0C3FAFFF761F889F826
:109F90000040284607F04BFECDE900651E22B3A322
:109FA0001146012007F0FEFF01F052FB02F018FC01
:109FB00017E205E06AE076E082E086E0A0E0A1E05A
:109FC00089F80040AB4890F8650001280FD0B0B187
:109FD00002281CD0032822D0042828D0052830D0FD
:109FE000062836D007283CD0082842D048E04FF455
:109FF000964948460EF07CF9C7F8029040E04FF4CD
:10A00000165948460EF074F9C7F8029038E04FF43C
:10A01000164948460EF06CF9C7F8029030E04FF44C
:10A02000614948460EF064F9C7F8029028E04FF401
:10A03000E13948460EF05CF9C7F8029020E06EE086
:10A040006FE04FF4963948460EF052F9C7F8029087
:10A0500016E04FF4966948460EF04AF9C7F80290A8
:10A060000EE04FF4965948460EF042F9C7F80290B8
:10A0700006E04FF4615948460EF03AF9C7F80290ED
:10A08000B879032894D10EF043FAAAE17A480088FF
:10A09000C1B2C0F3072015F024FF002001F0ECFE50
:10A0A00089F800409DE174480088C1B2C0F30720E0
:10A0B00015F071FE012001F0DFFE89F8004090E10B
:10A0C00015F036FA89F800408BE1CDE9006559A317
:10A0D0006C220A21012007F065FFCDE9006556A337
:10A0E00097220A21012007F05DFFCDE9006553A307
:10A0F000C2220A21012007F055FF89F8004070E1D3
:10A100000120EEE640B95D48008884380F2803D36B
:10A11000022008F009FD60E102F06AFF5DE1012024
:10A120001DE757480022B0F90010104609F0ECFA7C
:10A13000DFF8409199F85C03F8B1DFF848A19AF88C
:10A14000000018B908F00FFD8AF80080CDE900651D
:10A150004DA36C220021012007F024FFCDE900650A
:10A160004BA397220021012007F01CFF99F806104D
:10A170002022002008F018FDB3E099F80800042818
:10A1800055D944480078012804D09AF807100129CD
:10A190001FD01FE008F0E7FC4FF4784BCDE900B585
:10A1A0003DA367220021012007F0FCFECDE900B5A8
:10A1B0003BA392220021012007F0F4FECDE900B577
:10A1C00039A3BD220021012007F0ECFE8AF80780A8
:10A1D00087E058B13748B0F9000007F035FF36483E
:10A1E000007808F014F908F05CF97AE08AF8074082
:10A1F00008F0B9FC174880F8018080F8028080F8E8
:10A20000038080F8058080F804806921662008F0CA
:10A210005DFE9421662008F059FEBF21662008F0FB
:10A2200055FEED21002347F617601A4646E04DE043
:10A2300084F103085345540046414E0053595300DE
:10A2400096160020000000200F0300203502002099
:10A250006900002096110020330000203402002005
:10A260005570646174696E67000000005265737414
:10A2700061727400607F00204200002048000020CE
:10A280005E0200200D0300204D4F44425553000054
:10A29000494400003E020020486967680000000051
:10A2A000566F6C74616765006F6E20525334383599
:10A2B00000000000540000202C000020CDE9001612
:10A2C00002902D21EF2007F0A3FE0AE0FD48B0F92F
:10A2D000000007F0B9FEFC48007808F098F808F094
:10A2E000E0F84FF0000A504603F0B9FD0AF1010A08
:10A2F0000AF0FF0ABAF1090FF5D308F0F4F908F0F3
:10A3000007F999F80800042811D9F04800780128C5
:10A3100006D0EF48007838B1012009F082F90FE04B
:10A32000002009F07EF90BE009F00EF908E0E8489A
:10A33000007818B1012009F074F901E009F004F97E
:10A34000DFF8909399F8070048B1CDE90165002343
:10A35000E14A1A210D20009407F03EFE08E0CDE905
:10A36000016500231A461A210D20009407F050FEC3
:10A3700099F8080048B1CDE901650D23D74A1A21A3
:10A380001846009407F028FE08E0CDE901650D238A
:10A3900000221A211846009407F03AFE99F80700A7
:10A3A00010B1401E89F8070099F8080010B1401E4E
:10A3B00089F80800CA48007878B1CA48807902282C
:10A3C00014D050B1012808D0CDE901651A21D2235B
:10A3D000C54A0846009407F0FFFDC448007802F023
:10A3E00093FF4FF496700EF073F853E5CDE90165D5
:10A3F0001A21D223BE4A0846009407F0EDFDECE78F
:10A400000EF0FBF9BB4D4FF4964095F86510092905
:10A4100031D2DFE801F0050A0D12171C21262B00AE
:10A420004FF416500DF064FF27E00DF061FF24E0BB
:10A430004FF416400DF05CFF1FE04FF461400DF04B
:10A4400057FF1AE04FF4E1300DF052FF15E04FF4E2
:10A4500096300DF04DFF10E04FF496600DF048FF80
:10A460000BE04FF496500DF043FF06E04FF46150BF
:10A470000DF03EFF01E00DF03BFF00200024291805
:10A4800081F8A941401CC0B20828F8D39A4F9B4DCF
:10A490009B4E387830B1401EC0B23870012801D1CF
:10A4A00013F022FC287830B12878401E28702878D4
:10A4B00008B90EF02DF87089322802D2401C708144
:10A4C00013E0748107F0D8F98E4882888E490A809B
:10A4D00082798A70C279CA70027A0A7102788B49CD
:10A4E0000A7042784A70807888700A200DF0F0FF78
:10A4F000CFE708B50AF01BFA7E4D47352878697812
:10A5000000EB012182480180A978EA7801EB022161
:10A51000418029796A7901EB02218180A979EA7960
:10A5200001EB0221C180297A6A7A01EB02210181C3
:10A53000A97AEA7A01EB02214181297B6A7B01EB4E
:10A5400002218181A97BEA7B01EB0221C1810421E7
:10A550007048FEF7CFFC4FF400716F48FEF7C8FC5F
:10A5600045200BF0E8F9664C0027E7706B4E4FF082
:10A5700032084FF001090123002269496948CDF8EA
:10A5800000800BF048FB08B986F80090E078401C8A
:10A59000C0B2E0700A28EED33078012800D03770BE
:10A5A000DFF884A1614E624FDFF81C81DFF884B1CF
:10A5B000042561480178491C017009F06BFE09F01F
:10A5C000FEFFFEF7D1FD4FF0000C84F804C0002020
:10A5D000484A131893F89E12022901D0042942D147
:10A5E000DFF858E13EF810E0BEF1010F02D0237908
:10A5F000C3B133E09AF8001031BB357087F8009092
:10A6000088F8005082F89B5093F89E12022906D1D8
:10A6100092F86310C1EB01118900CBF8001084F8A7
:10A6200004901BE092F8B93213B104290DD015E063
:10A63000DBF8001041B986F800C03D7088F800C012
:10A6400082F89BC08AF800C008E086F800C03D7020
:10A6500088F800C082F89BC08AF800C01D4981F8C4
:10A66000049081F80290401CC0B20828B0D30AF0D0
:10A670005FFA204890F8EF1201297AD1304A90F819
:10A68000F1121288511A00D5494290F8B423914230
:10A690006FDD84F8009084F8019090F86310FF2932
:10A6A00002D13C2180F8631090F8631049B1C1EBEE
:10A6B00001118900CBF80010224981F80090357013
:10A6C00043E04FE0540000202C0000203E02002018
:10A6D00008030020961100200CF30308B0F50308CE
:10A6E00019030020872200209CFD0308F8000020A9
:10A6F00054F80308607F00201D0300201B03002086
:10A70000000000208C110020D0030020C80300208E
:10A71000E011002000180140000C01403D02002023
:10A72000800200207C020020290000203B00002045
:10A73000370000204C0000204402002018120020A6
:10A74000520200203A00002013E088F80050417ABD
:10A7500041F001014172092007F042F887F80090AA
:10A76000022060709A4880F8029080F8019080F88A
:10A7700004904FF496700DF0ABFE1AE7002400250C
:10A78000944900200870944908709449FF2008708B
:10A790009349087040F6B8300DF09AFEDFF8449205
:10A7A000914E924FDFF8488299F8000015F0EBFACD
:10A7B0003080B7F90810884203D0388184490120DD
:10A7C00048706D1CADB298F8800100EB8000A84283
:10A7D00004D2012015F04CFD002502E0002015F008
:10A7E00047FD641CE4B2052C09D998F8DB00032866
:10A7F0000BD0012003F031FC002404F092FC0AF09D
:10A80000B6FCC8200DF064FECEE7022003F025FC64
:10A81000F2E72DE9FF41002476490803FDF7B1FF77
:10A82000FEF756FF4FF4A060FDF776FFFEF79CFCA5
:10A8300048200DF019FE40F2CF21642009F0B2F853
:10A8400006F022FFFEF77EFC00F0C5F9FEF70DFCD6
:10A850000AF0F2F9002101200AF050FB0021022049
:10A860000AF04CFB002103200AF048FB00210420E1
:10A870000AF044FB002105200AF040FB5C485E49D9
:10A8800090F86A000870FEF771FCFEF76DFCFEF7A9
:10A890006BFC01215948FEF72BFB07F017FBFEF775
:10A8A00022FFFEF761FC0125FEF75EFC142C0AD2A4
:10A8B00007F04AF8012806D0641CE4B264200DF0C9
:10A8C00007FE002DF0D100240620CDE900044FF44E
:10A8D000617802942346424649A14D4803940DF005
:10A8E00042F80220CDE900044FF4C8760294002318
:10A8F000324648A1494803940DF035F80525CDE9C5
:10A90000005402940023324645A1474803940DF0B9
:10A910002AF80326CDE9006402940023642243A1AF
:10A92000464803940DF01FF80127CDE90074029406
:10A930000023642242A1464803940DF014F8CDE9A7
:10A94000005402940023424642A1444803940DF06F
:10A950000AF8CDE9007402940023642240A144481F
:10A9600003940DF000F8CDE90054029400234FF455
:10A97000167240A1424803940CF0F5FFCDE9006443
:10A980000294002364223FA1424803940CF0EBFFA1
:10A990000DF0C6FA04B00020BDE8F0813E4D00265F
:10A9A0004FF47A77287870B1401EC1B2297051B93E
:10A9B000002400222146394800F085F8641CE4B2E6
:10A9C000032CF6D32E7038460DF082FDEAE7000026
:10A9D00096110020730000209002002091020020B8
:10A9E00092020020370000205400002000000020C8
:10A9F000607F0020008000087700002000080140F0
:10AA0000436F6E74726F6C4C6F6769630000000077
:10AA10007DA70008496E707574000000F3A400085B
:10AA2000434F4D4D0000000001A4000844697370BD
:10AA3000616C79526566726573680000319D00082B
:10AA4000536F66747761726574696D65720000009A
:10AA5000919900084D535450000000007D98000863
:10AA6000436F6F6C696E674C6F636B4F757400005A
:10AA7000CF970008576966697461736B0000000026
:10AA80003D7301084B65797061647348616E646C55
:10AA900065000000A59700087200002080000020DB
:10AAA00048437047C84000F00100704701238B40C5
:10AAB000DBB20178002A02D0194301707047DA43F3
:10AAC00011400170704701238B409BB20188002A1E
:10AAD00002D0194301807047DA431140018070476A
:10AAE00001228A40D1B20078084201D1002070478B
:10AAF0000120704770B540F27A4006F070FEFE4DBE
:10AB0000287040F27C4006F06AFE4FF6FF7404EABB
:10AB10000020688040F27B4006F061FE69880844AE
:10AB2000688040F27D4006F05AFEF44D287040F2F5
:10AB30007F4006F054FE04EA0020688040F27E4028
:10AB400006F04DFE6988084468804FF4906006F076
:10AB500046FEEB4D287040F2824006F040FE04EACB
:10AB60000020688040F2814006F039FE6988084480
:10AB7000688040F2894006F032FEE24D287040F2D3
:10AB80008B4006F02CFE04EA0020688040F28A40E8
:10AB900006F025FE69880844688040F2834006F08C
:10ABA0001EFED94D287040F2854006F018FE04EADA
:10ABB0000020688040F2844006F011FE6988084455
:10ABC000688070BD01EB002109B27F2801D908B26D
:10ABD0007047084670472DE9F84F6E2006F0FFFDDC
:10ABE000DFF8288388F86E000024012805D988F84A
:10ABF0006E4000216E2006F0F3FD0025C44E4FF498
:10AC00008F67284606F0EBFDA5F15F02A42A1FD24C
:10AC100098F86E1001EBC10303EB411106EBC10381
:10AC200013F812C0844507D803EB420252788242DF
:10AC300002D308F805000DE0B64800EB8100284477
:10AC400010F85F1C08F80510284606F0C9FD01E061
:10AC500008F805006D1CADB2BD42D2D998F85D0070
:10AC6000FF2801D188F85D40AB4998F85D00087075
:10AC7000AB4D0222A9492846FDF792FCA74E327837
:10AC800098F80610FF291BD0D1B1914205D0318030
:10AC9000012231462846FDF792FC00256F462846E2
:10ACA00006F09DFD78556D1CADB2042DF7D39C4B7D
:10ACB0009B4D9DF8001010332035FF2910D01BE06C
:10ACC000022296492846FDF76BFC307888F806008A
:10ACD000FF2801D00028E0D1FE2088F80600DCE73C
:10ACE0009DF80100FF2807D19DF80200FF2803D13D
:10ACF0009DF80300FF282ED0F1B398F800008142A0
:10AD000024D09DF8010098F8012090421ED09DF8B3
:10AD1000022098F80250AA4218D09DF8032098F813
:10AD20000350AA4212D0318070801D4602227B4916
:10AD30002846FDF744FC9DF8021031809DF8031071
:10AD40007180022275492846FDF739FC98F8D9022E
:10AD5000FF2830D036E0022270491846FDF720FC6B
:10AD6000307888F80000B07888F8010002226B493A
:10AD70002846FDF715FC00E006E0307888F8020070
:10AD8000B07888F80300E1E7022264491846FDF72D
:10AD900007FC307888F80000B07888F801000222BB
:10ADA0005E492846FDF7FCFB307888F80200B07851
:10ADB00088F80300CAE788F8D942002140F2D92078
:10ADC00006F00EFD98F87E03FF280DD188F87E432B
:10ADD00088F87D43002140F27D3006F001FD00211E
:10ADE00040F27E3006F0FCFC98F87E034B4D0002EA
:10ADF000283D98F87D130143298398F81B1098F893
:10AE00001C00012601EB002298F82F00454900EBB9
:10AE10000020824201D20E7000E00C7098F83100E0
:10AE200098F8322000EB022298F8450000EB002051
:10AE3000824201D24E7000E04C704FF45A7738468F
:10AE400006F0CDFC38490870FF2804D10C7021466B
:10AE5000384606F0C5FC98F85C00344BFF2803D157
:10AE600098F85B10FF290AD098F85B10FFF7AAFE4C
:10AE7000188098F881132020FF290AD01BE01C803D
:10AE800000215B2006F0ACFC00215C2006F0A8FC51
:10AE9000EFE74F2188F88113662188F8821388F83C
:10AEA000831388F8844388F8850388F8860388F834
:10AEB000870388F8880398F889236F21FF2A11D126
:10AEC0004C2288F8892388F88A13772288F88B2304
:10AED00088F88C4388F88D0388F88E0388F88F03F0
:10AEE00088F8900398F891236427FF2A2ED14D22E9
:10AEF00088F8912365221BE0AE110020B8110020D4
:10AF0000C2110020CC110020D6110020607F00204B
:10AF1000FA0003088A0303083C02002050000020C6
:10AF20000077000874020020120300206402002051
:10AF300088F8922388F8937388F8944388F89503E7
:10AF400088F8960388F8970388F8980398F8992367
:10AF5000FF2A11D1482288F89923692288F89A2378
:10AF600088F89B4388F89C0388F89D0388F89E0323
:10AF700088F89F0388F8A00398F8A123FF2A12D12C
:10AF8000412288F8A123752288F8A223742288F828
:10AF9000A32388F8A41388F8A54388F8A60388F8A3
:10AFA000A70388F8A80398F889034C2800D0EE710D
:10AFB00098F8ED00FF2806D0C0EB00104FF6FF71A7
:10AFC00001EA8000E88298F8A903FF2801D188F8F7
:10AFD000A94398F89702FF2811D198F89602FF2804
:10AFE0000DD1002140F2972006F0FAFB88F8974235
:10AFF000012140F2962006F0F3FB88F8966298F85B
:10B000002D04FF280ED1002505F22D4080B200212D
:10B0100006F0E6FB08EB050080F82D446D1CADB290
:10B020002E2DF1D314F009F998F882004546022834
:10B0300001D985F8824095F89200DFF82CB40128F8
:10B0400004D985F8924003208BF8060095F8B403E4
:10B05000FF2806D11E2185F8B4134FF46D7006F059
:10B06000BFFB40F28C4006F0BAFB00EB80004000D2
:10B07000FE4908804FF47A72904201D90A8005E0B7
:10B08000B0F5FA7F02D24FF42F70088040F28D4065
:10B0900006F0A5FBF6490870FFF72CFD95F8F102C4
:10B0A000FF2800D010B9A02085F8F102F149A87955
:10B0B000087040F28F4A504606F091FBDFF8B893D3
:10B0C0004FF49268FF2804D1404606F088FBFF2821
:10B0D0003AD0504606F083FBC9F80000404606F01F
:10B0E0007EFBD9F8001041EA0020C9F8000040F2C8
:10B0F000914006F074FBD9F8001041EA0040C9F80D
:10B10000000040F2924006F06AFBD9F8001041EAD4
:10B110000060C9F800000021DFF86093002001EB17
:10B1200041024FEA820801EB410209EBC20208EB3F
:10B1300040032B4493F8B5C3BCF1180F11D902EBAF
:10B14000400C8CF8014010E02878697840EA012032
:10B15000A97840EA0140E97840EA0160C9F80000B6
:10B16000D9E702EB400A8AF801C093F8B6333B2BCB
:10B1700002D902F8104001E002F81030401C80B201
:10B180000628D4D3491C89B20829C7D30020BC495A
:10B190002A1892F82D240A54401C80B22E28F7D386
:10B1A00095F878043238652801D385F8787440F230
:10B1B000954006F014FBB34F0002388040F29440F3
:10B1C00006F00DFB39880843388040F2974006F0BE
:10B1D00006FBAD4F0002388040F2964006F0FFFAC1
:10B1E0003988084338800027A046E81990F867128C
:10B1F000FF2907D180F8678207F2672080B200211B
:10B2000006F0EEFA7F1CBFB2092FEED395F881014C
:10B21000FF2806D185F88181002140F2811006F0D7
:10B22000DFFA95F88001FF2806D185F8808100219A
:10B230004FF4C07006F0D4FA0021944A944F0020D5
:10B2400007EB811343F82020401C80B21028F9D36B
:10B25000491C89B20729F2D39BF80600032838D18C
:10B260000024DFF830A20AF266390AF1D60AE1B208
:10B270005046FFF735FC40B1E1B24846FFF730FCDD
:10B2800024F056FA07EB8411C861641CA4B2052CA3
:10B29000EDD305215046FFF723FC50B195F862032A
:10B2A00095F86313000200B2084424F029FAC7F8A5
:10B2B0005C0106215046FFF713FC50B195F864037A
:10B2C00095F86513000200B2084424F019FAC7F893
:10B2D0009C0195F85F03FF2812D195F8601328466A
:10B2E000FF290DD180F85F8380F86083002140F250
:10B2F0005F3006F075FA00214FF4587006F070FACE
:10B30000E879092803D00921072006F069FA95F8A1
:10B310005F0040F26134152805D1314685F861633C
:10B32000204606F05DFA95F8A200152805D13146B1
:10B3300085F86163204606F053FA4FF4187006F062
:10B340004EFA5549087095F82903FF2802D10520C7
:10B3500085F82903BDE8F88F1CB502460846843AF3
:10B360004E4CC1B2072A0ED2DFE802F0040E190DCE
:10B37000242F3900A1786278CDE900212378E27981
:10B38000A17906F038FB1CBDA1786278CDE90021D7
:10B390002378E279C1B2A08806F02DFB1CBDA1780C
:10B3A0006278CDE900212378A179C2B2A08806F0A5
:10B3B00022FB1CBDA1786278CDE90021E279C3B2FD
:10B3C000A179A08806F017FB1CBDA078CDE900107C
:10B3D0002378E279A179A08806F00DFB1CBD607886
:10B3E000CDE900012378E279A179A08806F003FB7A
:10B3F0001CBD10B501210F2006F0F2F9002110202C
:10B4000006F0EEF90121112006F0EAF90021BDE86D
:10B410001040122006F0E4B970B50024204D04F568
:10B42000B070295D06F0DCF9641CE4B2072CF6D399
:10B4300070BD70B500241B4D24F00100295C04F19F
:10B440001B0006F0CDF9A41CE4B2152CF4D30124A2
:10B4500024F00100285A010A04F11B0006F0C0F98B
:10B46000A41CE4B2162C1FE09616002094020020C3
:10B470000C030020170300200C000020368600205B
:10B48000088600206A0200206802002000007F4336
:10B4900048840020607F00208C0200208C11002056
:10B4A000A5FB020864FB0208D2D30024FE4D24F061
:10B4B0000100295C04F1310006F092F9A41CE4B209
:10B4C000152CF4D3012424F00100285A010A04F1B8
:10B4D000310006F085F9A41CE4B2162CF3D370BD3C
:10B4E0002DE9F0410025DFF8C4830024C5EBC50039
:10B4F00000EB080605EB85073819315D00F5A170F2
:10B5000006F06EF9641CE4B2052CF5D36D1CEDB2A7
:10B51000022DEAD3BDE8F08170B50024E44D04F2B9
:10B520002D10295D06F05CF9641CE4B2152CF6D3ED
:10B5300070BD2DE9F04107460024DE4D0126062F9F
:10B5400021D2DFE807F07F037F214462DA48015D02
:10B5500004F2031006F044F9012C07D10321A020C6
:10B5600006F03EF90321A12006F03AF9072C04D297
:10B57000002104F1B20006F033F901216F2006F03A
:10B580002FF985F86F605DE0CC48015D04F203108F
:10B5900006F026F9012C07D10221A02006F020F99F
:10B5A0000221A12006F01CF9072C04D2002104F18D
:10B5B000B20006F015F904219B2006F011F90321D1
:10B5C0006F2006F00DF9032085F86F003AE0BC48C3
:10B5D000015D04F2031006F003F9012C07D10221EA
:10B5E000A02006F0FDF80221A12006F0F9F8072CB2
:10B5F00004D2002104F1B20006F0F2F801216F201C
:10B6000006F0EEF885F86F601CE0AE48015D04F2CC
:10B61000031006F0E5F8012C07D10221A02006F066
:10B62000DFF80221A12006F0DBF8072C04D200216C
:10B6300004F1B20006F0D4F801216F2006F0D0F832
:10B6400085F86F60641CE4B22A2CFFF478AF61E7E0
:10B650002DE9F0415F249C4D964E4FF48177652C87
:10B6600019D096F86E0000EBC00101EB401005EB1D
:10B670008000204410F85F1C204606F0B1F896F8D0
:10B680006E0000EBC00101EB401005EB8000204490
:10B6900010F85F0C3055641CA4B2BC42DFD996F898
:10B6A0006E1040F259256C1C11B1012913D024E011
:10B6B000C821284606F094F80021204606F090F8AC
:10B6C000284606F08CF886F85902204606F087F8DE
:10B6D00086F85A0211E0A821284606F081F80221D6
:10B6E000204606F07DF8284606F079F886F85902DB
:10B6F000204606F074F886F85A0274480078FFF77E
:10B7000018FFFFF709FFFFF7EBFEFFF792FEFFF7C9
:10B7100083FEFFF76EFE4F2140F2813006F060F8A5
:10B72000662140F2823006F05BF8662140F28330F9
:10B7300006F056F800214FF4617006F051F8202110
:10B7400040F2853006F04CF8202140F2863006F0B9
:10B7500047F8202140F2873006F042F820214FF4CC
:10B76000627006F03DF84C2140F2893006F038F85E
:10B770006F2140F28A3006F033F8772140F28B30A7
:10B7800006F02EF800214FF4637006F029F820210E
:10B7900040F28D3006F024F8202140F28E3006F081
:10B7A0001FF8202140F28F3006F01AF820214FF4C4
:10B7B000647006F015F84D2140F2913006F010F853
:10B7C000652140F2923006F00BF8642140F293308C
:10B7D00006F006F800214FF4657006F001F820210C
:10B7E00040F2953005F0FCFF202140F2963005F044
:10B7F000F7FF202140F2973005F0F2FF20214FF4AF
:10B80000667005F0EDFF482140F2993005F0E8FF41
:10B81000692140F29A3005F0E3FF002140F29B30AD
:10B8200005F0DEFF20214FF4677005F0D9FF2021DD
:10B8300040F29D3005F0D4FF202140F29E3005F00B
:10B84000CFFF202140F29F3005F0CAFF20214FF4A6
:10B85000687005F0C5FF412140F2A13005F0C0FF3E
:10B86000752140F2A23005F0BBFF742140F2A330F5
:10B8700005F0B6FF6F214FF4697005F0B1FF0021AC
:10B8800040F2A53005F0ACFF202140F2A63005F0D3
:10B89000A7FF202140F2A73005F0A2FF20214FF49E
:10B8A0006A7005F09DFF13E07AFB02087A05030831
:10B8B00090FB0208607F0020D2040308FC04030808
:10B8C00026050308500503088A03030877000020B3
:10B8D0000021922005F084FF002448274FF04708FC
:10B8E00007EB4405A8B205F07AFFFF2809D108EB61
:10B8F000440080B2002105F073FFA8B2002105F0DA
:10B900006FFF641CA4B2082CEAD3012086F8B802A9
:10B9100001214FF42E7005F063FF0E2140F2BA2092
:10B9200005F05EFF0E2086F8BA0296F8480300255F
:10B93000FF2873D106F55276542030705321717070
:10B94000B0704121F170307138207071B571F571AE
:10B95000A6F5527654214FF4527005F041FF532161
:10B9600040F2493005F03CFF542140F24A3005F0E6
:10B9700037FF412140F24B3005F032FF54214FF4A4
:10B98000537005F02DFF382140F24D3005F028FFAF
:10B99000002140F24E3005F023FF002140F24F30ED
:10B9A00005F01EFF00214FF4547005F019FF00212F
:10B9B00040F2513005F014FF002140F2523005F002
:10B9C0000FFF002140F2533005F00AFF00214FF431
:10B9D000557005F005FF002140F2553005F000FFDD
:10B9E000002140F2563005F0FBFE002140F25730B6
:10B9F00005F0F6FE00214FF4567005F0F1FE00212F
:10BA000040F2593005F0ECFE002140F25A3005F0CA
:10BA1000E7FE002140F25B3005F0E2FEC82140F273
:10BA2000AA3005F0DDFE002140F2AB3005F0D8FE73
:10BA3000C8214FF46B7005F0D3FE002140F2AD3009
:10BA400005F0CEFE282140F2AE3005F0C9FE1021EF
:10BA500040F2AF3005F0C4FE1E214FF46C7005F0CB
:10BA6000BFFE0F2140F2B13005F0BAFE322140F2A4
:10BA7000B23005F0B5FE052140F2B33005F0B0FE5E
:10BA800006214FF4A87005F0ABFE1E2140F25110C4
:10BA900005F0A6FE08214FF4A97005F0A1FE1E21B5
:10BAA00040F2531005F09CFE12214FF4AA7005F0ED
:10BAB00097FE1E2140F2551005F092FE16214FF41C
:10BAC000AB7005F08DFE1E2140F2571005F088FE88
:10BAD000002140F2B92005F083FE96F89702FF2876
:10BAE0000DD196F89602FF2809D1002140F2972047
:10BAF00005F076FE012140F2962005F071FE40F23D
:10BB0000E1718420FFF728FC0024301990F86712B7
:10BB1000FF2907D180F8675204F2672080B2002124
:10BB200005F05EFE641CA4B2092CEED3002404F5DB
:10BB3000A17080B2002105F053FE641CA4B2072C52
:10BB4000F5D3002404F2491080B2002105F048FE2C
:10BB5000641CA4B2072CF5D3DCE42DE9F041FE4CC3
:10BB600040F25A26204694F86E10771E90F87E0018
:10BB700000297DD000EBC0000525B0FBF5F020309A
:10BB80007B34C1B2E1707E2005F02AFEA07800EB84
:10BB9000C000B0FBF5F02030C1B2A1707D2005F0EF
:10BBA0001FFE14F8040C00EBC000B0FBF5F02030D1
:10BBB000C1B204F8041C772005F012FE94F8660068
:10BBC00000EBC000B0FBF5F02030C1B284F8661085
:10BBD000E12005F005FE94F8DE0194F8DF1100EB9A
:10BBE000012080B200EBC000B0FBF5F000F5A070C2
:10BBF00082B2110A84F8DF1184F8DE21304605F0A4
:10BC0000EFFD94F8DE11384605F0EAFDA07EE17EF6
:10BC100000EB012080B200EBC000B0FBF5F000F5B6
:10BC2000A07080B2010AE176A076962005F0D8FDDA
:10BC3000A17E952005F0D4FD207F617F00EB0120DF
:10BC400080B200EBC000B0FBF5F000F5A07080B250
:10BC5000010A61772077982005F0C2FD217F9720A7
:10BC600005F0BEFDA07FE17F00EB012080B200E087
:10BC700041E000EBC000B0FBF5F000F5A07080B231
:10BC8000010AE177A0779A2005F0AAFDA17F99200B
:10BC900005F0A6FD14F8070D617800EB012080B2D5
:10BCA00000EBC000B0FBF5F000F5A07080B2010A17
:10BCB00061702070752005F093FD14F8071B742047
:10BCC00005F08EFD14F8090D617800EB012080B2BB
:10BCD00000EBC000B0FBF5F000F5A07080B2010AE7
:10BCE00061702070732005F07BFD2178BDE8F04184
:10BCF000722005F075BD2038C0B2092500EB800028
:10BD0000B0FBF5F07B34C1B2E1707E2005F068FD38
:10BD1000A0782038C0B200EB8000B0FBF5F0C1B2D3
:10BD2000A1707D2005F05CFD14F8040C2038C0B231
:10BD300000EB8000B0FBF5F0C1B204F8041C7720E2
:10BD400005F04EFD94F866002038C0B200EB80008C
:10BD5000B0FBF5F0C1B284F86610E12005F040FDBB
:10BD600094F8DE0194F8DF1100EB0120A0F5A0703B
:10BD700080B200EB8000B0FBF5F082B2110A84F8CB
:10BD8000DF1184F8DE21304605F02AFD94F8DE113B
:10BD9000384605F025FDA07EE17E00EB0120A0F5F0
:10BDA000A07080B200EB8000B0FBF5F080B2010A19
:10BDB000E176A076962005F013FDA17E952005F092
:10BDC0000FFD207F617F00EB0120A0F5A07080B205
:10BDD00000EB8000B0FBF5F080B2010A61772077BC
:10BDE000982005F0FDFC217F972005F0F9FCE17F0C
:10BDF0005A4EA07F06EB0121084480B200EB800080
:10BE0000B0FBF5F080B2010AE177A0779A2005F047
:10BE1000E7FCA17F992005F0E3FC14F8070D617899
:10BE200006EB0121084480B200EB8000B0FBF5F086
:10BE300080B2010A61702070752005F0D1FC14F801
:10BE4000071B742005F0CCFC14F8090D617806EB93
:10BE50000121084480B200EB8000B0FBF5F080B215
:10BE6000010A61702070732005F0BAFC2178BDE8EA
:10BE7000F041722005F0B4BC10B5374C012823D036
:10BE80009A2005F0ACFC703484F82A00992005F063
:10BE9000A6FC84F82900702005F0A1FC2070712018
:10BEA00005F09DFC6070752005F099FC60717420B0
:10BEB00005F095FC2071732005F091FCE070722074
:10BEC00005F08DFCA07010BD40F25A2005F087FCF3
:10BED000793484F8E10140F2592005F080FC84F8BF
:10BEE000E0016C2005F07BFC04F80D0C6D2005F0E2
:10BEF00076FC04F80C0C962005F071FC6077952018
:10BF000005F06DFC2077982005F069FCE07797201C
:10BF100005F065FCA07710BD2DE9F043DFF838800F
:10BF20000F4A414698F8B992D07C91F8615359EA8A
:10BF3000000991F87D000B4F00EB800300EB8000BF
:10BF400091F8C5104FEA400402F12C064FF0050CA1
:10BF500013D098F8590207E0607F0020C0FEFFFF71
:10BF6000280000200F03002098F85A8200EB0820D8
:10BF7000084400B250834DB32CE098F8990098F82B
:10BF80009A8000EB082000B250830A2903D00844AD
:10BF9000508385B115E00A2190FBF1F801FB1808E8
:10BFA000B8F1000FF5D090FBF1F801FB1801401A31
:10BFB0000A305083EDE7B2F91A00B0EB430F00DD11
:10BFC0005483508B308087F800C007E0B0EB430FFC
:10BFD00000DD5483508B3080062038700020D072F2
:10BFE00082F808C0BDE8F0832DE9F041DFF8FCC31A
:10BFF000FF4A9CF8B70090739CF8B982D07C6146E8
:10C0000058EA000891F87E0091F8615300EB800334
:10C0100000EB8000F74F91F8C5104FEA400402F1A1
:10C020002C060AD09CF859029CF85AC200EB0C204E
:10C03000401A00B250834DB32CE09CF899009CF854
:10C040009AC000EB0C2000B250830A2903D0401A9A
:10C05000508385B115E00A2190FBF1FC01FB1C0C1B
:10C06000BCF1000FF5D090FBF1FC01FB1C01401A64
:10C070000A385083EDE7B2F91A00B0EB430F00DA4B
:10C080005483508B30800720387007E0B0EB430FAB
:10C0900000DA5483508B3080082038700020D07232
:10C0A0000520107258E52DE9F041D14CCF4D012605
:10C0B0002179687A002914D040F001016972A674D0
:10C0C000092005F08DFB95F86300C0EB001080009F
:10C0D00060622179E17485F89B1095F8B902C8B1C6
:10C0E0001BE000F0FE0169720027A774092005F02B
:10C0F00077FBC148077067622179E17485F89B106E
:10C1000095F8B90210B99B2005F06AFBA7710420CD
:10C11000E07303E09B2005F063FBE673E07CE070D6
:10C12000B648067118E530B5B14A0123537110794C
:10C13000042801D2401C10711079AC4C0025042851
:10C140000DD90020211891F89E12022901D004294E
:10C1500000D15370401CC0B20828F3D3157194F875
:10C160006F1013790420994200D21071D572507269
:10C17000A348057030BD9E49012048710879002808
:10C1800001D0401E087199480A7990F86F009042DA
:10C1900000D208710020C87204224A7298490870BF
:10C1A000704710B59149002491F86B00002825D103
:10C1B00091F8A903022802D2401C81F8A90391F842
:10C1C000A00028B991F8A903022801D181F8A94358
:10C1D00091F8A10030B991F8A903012802D10220F9
:10C1E00081F8A90391F8A903022801D981F8A9438C
:10C1F00091F8A91340F2A93005F0F2FA7C48C47214
:10C200000421817210BD10B57849002491F86B00AB
:10C2100000281DD191F8A90310B1401E81F8A9038F
:10C2200091F8A00028B991F8A903022801D181F85A
:10C23000A94391F8A10028B991F8A903012801D1D7
:10C2400081F8A94391F8A91340F2A93005F0C8FA82
:10C250006748C4720421817210BD7CB5694843F6F9
:10C26000EF464FF6FF75007847F6196401281CD099
:10C27000022833D0032817D1CDE9005462A36C22E1
:10C280000A21012005F08EFECDE900545FA397221C
:10C290000A21012005F086FECDE900565CA3C222EA
:10C2A0000A21012005F07EFE7CBDCDE9005656A393
:10C2B0006C220A21012005F075FECDE9005453A33C
:10C2C00097220A21012005F06DFECDE9005450A30C
:10C2D000C2220A21012005F065FE7CBDCDE9005493
:10C2E00049A36C220A21012005F05CFECDE900562D
:10C2F00046A397220A21012005F054FECDE90054FF
:10C3000043A3C2220A21012005F04CFE7CBD7CB56E
:10C310003C4843F6EF464FF6FF75007847F6196440
:10C3200001281CD0022833D0032817D1CDE90054AE
:10C3300035A36C220A21012005F034FECDE900541A
:10C3400032A397220A21012005F02CFECDE90056E8
:10C350002FA3C2220A21012005F024FE7CBDCDE9D5
:10C36000005629A36C220A21012005F01BFECDE90D
:10C37000005426A397220A21012005F013FECDE9DF
:10C38000005423A3C2220A21012005F00BFE7CBD2C
:10C39000CDE900541CA36C220A21012005F002FE05
:10C3A000CDE9005619A397220A21012005F0FAFDD4
:10C3B000CDE9005416A3C2220A21012005F0F2FDA6
:10C3C0007CBD2DE9F041022006F0AEFB084E114B7A
:10C3D000064D308C06F11E04772825D07D2823D009
:10C3E00070285AD0712861D0822815E0607F002023
:10C3F000280000200F030020D80000209611002004
:10C4000010000020F00000205345540046414E002B
:10C4100053595300FA00030851D0002101226B2820
:10C4200054D05E2871D07FE0772819D095F8610349
:10C4300001282ED095F87E00B4F90010401C8142EE
:10C440000DDD95F86E0000EBC00202EB401003EB2F
:10C45000C00090F83C00814201DD491E2180C8E007
:10C4600095F86103012813D1B4F9001095F87E0006
:10C4700081420DDD95F86E0000EBC00202EB40102A
:10C4800003EBC00090F83000814201DD491E21809D
:10C49000AFE02088401E2080ABE021880A3921804F
:10C4A000C9B285F8701005F09BF9A2E021880A391D
:10C4B0002180C9B285F8711005F092F999E0B4F9BC
:10C4C0000000002801DD401E208092E0B4F9000049
:10C4D000032802DB401E20808BE0022802D00128C6
:10C4E0000AD086E095F87900032801D0012801D808
:10C4F00021807EE022807CE095F87900032801D03D
:10C50000012876D8218074E0FFE7377D67B1B4F960
:10C51000000095F8CF10884202DD401E208068E0C0
:10C5200095F8D100208064E05D2801D1377DD7B136
:10C53000572818D072281AD0652821D095F86E1087
:10C5400001EBC10707EB411103EBC103A0F15F0150
:10C5500013F81130B4F900108B424AD0491E2180E3
:10C56000E5283CD040E02088401E208041E0208823
:10C57000401E2080010A85F89A1085F8990038E05D
:10C58000B4F9000090B1072813D0012814D008286E
:10C5900015D0042815D0052816D0032817D0022856
:10C5A00018D0062818D0401E208022E007202080C6
:10C5B0001FE0062020801CE00820208019E0218058
:10C5C00017E00520208014E00320208011E00220E5
:10C5D00020800EE022800CE00420208009E095F805
:10C5E0005F10012900D122805F2802D1208800B984
:10C5F0002280308C642802D1207885F8640051E5CF
:10C6000070B5022006F090FAFD4BFE4CFE4A188CE5
:10C6100003F11E01772804D07E2802D05E2834D092
:10C6200042E092F861331BB10888401C088070BD5D
:10C63000772815D092F87D00B1F90030401E834272
:10C64000F5DA92F86E0000EBC00202EB401004EB4A
:10C65000C00090F83F008342E9DA5B1C0B8070BD9C
:10C66000B1F9003092F87D008342F8DA92F86E005A
:10C6700000EBC00202EB401004EBC00090F8310068
:10C680008342ECDA5B1C0B8070BD1D7D65B1B1F996
:10C69000000092F8D130984202DA401C088070BD48
:10C6A00092F8CF00088070BD02256B2802D05E286A
:10C6B00019D01AE0B1F900303BB992F8790003289B
:10C6C00001D0012801D80D8070BD92F86E0000EBFA
:10C6D000C00202EB401004EBC000407E9842F3DD44
:10C6E0005B1C0B8070BD1B7D13B3702824D0712898
:10C6F0002CD0722834D082283AD065283FD092F8C6
:10C700006E3003EBC30505EB431304EBC304A0F148
:10C710005F0304EB43035C78B1F900309C4201D025
:10C720005B1C0B806428DDD1087882F8640070BD42
:10C730000888401C088070BD0B880A330B80D9B272
:10C7400082F87010BDE8704005F04AB80B880A33D3
:10C750000B80D9B282F87110BDE8704005F040B886
:10C760000888401C0880010A99325170107070BD11
:10C77000B1F900000228FADA401C088070BDB1F956
:10C780000000062811D0072812D0A0B1082815D023
:10C79000012816D0022816D0032817D0052818D053
:10C7A0000428EBD10620088070BD0720088070BDEA
:10C7B0000020088070BD0820088070BD012008801E
:10C7C00070BD0D8070BD0320088070BD05200880FD
:10C7D00070BD0420088070BD4FF47A700BF078BEF5
:10C7E000FCF736BC2DE9F05FDFF814B2874E0BF191
:10C7F0001E05BBF820000127DFF814A2824CB5F912
:10C8000000104FF00208942806D0642809D05A4638
:10C810005E28127D0ED00EE0C80701D18AF8008094
:10C8200080E094F86410642004F0DAFF287884F83B
:10C83000640077E012B15E2820D034E094F85F0005
:10C84000022801D013286DD17248DFF8CC910088FE
:10C85000081AA9F80000C1B25B2004F0C1FFB9F8C2
:10C860000000C0F307215C2004F0BAFFB9F8000013
:10C8700084F85B00000A84F85C0053E09AB1C9B206
:10C88000062004F0ADFF2878A0715D4928310880AA
:10C8900001226248FBF793FE6149A07908700C20E1
:10C8A0008AF800003EE083280DD0554A1E32B2F9C6
:10C8B000002002EB82025200952814D09B281BD046
:10C8C000722826D02EE0C80706D00121832004F06C
:10C8D00087FF8BF8107025E00221832004F080FF91
:10C8E0008BF810801EE0D1B2C2F3072013F053FA88
:10C8F0000120FFF7C1FA15E0C9B28BF8131084F8D4
:10C900009B108BF804109B2004F06AFFB7703771FE
:10C9100008E02A80D1B2C2F3072013F0E2FA002027
:10C92000FFF7AAFABBF82000B5F90010225C8A4292
:10C930007AD021545E2802D0C9B204F051FFBBF86E
:10C9400020006A2807D1297804F04AFF2878FEF7EA
:10C95000F0FDFFF745FFBBF820006E2807D12978CE
:10C9600084F86E1004F03CFF3770FFF7F6F8BBF860
:10C970002000792803D1FFF733FFFFF72DFFBBF825
:10C9800020005F2804D1297884F85F1004F028FF84
:10C99000BBF820006B281AD12888042809D194F804
:10C9A000E500012805D0394684F8E570E52004F05B
:10C9B00017FF288805280AD194F8E600012806D038
:10C9C00084F8E67094F86210E62004F009FFBBF8E2
:10C9D0002000144E4FF00009652871D1297804F029
:10C9E000FFFEB5F9000030B301282FD0022838D05F
:10C9F000032841D004284BD0052855D0062814E040
:10CA000028000020FA000308607F00209611002013
:10CA10000F03002078020020640200200077000845
:10CA200017030020961600200DE14AD0072854D0A5
:10CA300008285ED068E084F865904FF416500BF03B
:10CA400057FC4FF41650C6F802005DE084F865709C
:10CA50004FF496400BF04CFC4FF49640C6F80200A1
:10CA600052E084F865804FF416400BF041FC4FF41F
:10CA70001640C6F8020047E0032084F865004FF432
:10CA800061400BF035FC4FF46140C6F802003BE01A
:10CA9000042084F865004FF4E1300BF029FC4FF4DA
:10CAA000E130C6F802002FE0052084F865004FF45D
:10CAB00096300BF01DFC4FF49630C6F8020023E0D0
:10CAC00024E0062084F865004FF496600BF010FC1B
:10CAD0004FF49660C6F8020016E0072084F865005F
:10CAE0004FF496500BF004FC4FF49650C6F8020039
:10CAF0000AE0082084F865004FF461500BF0F8FB61
:10CB00004FF46150C6F802000BF002FDBBF82000A4
:10CB100083280FD12878C00706D00121832004F094
:10CB20005FFE8BF8107005E00221832004F058FEB0
:10CB30008BF81080BBF820006C2801D06D2825D11F
:10CB40000A216C2827D094F86D20B5F9000002EB7B
:10CB50008202B0EB420F0DDB90FBF1F0401CC1B242
:10CB600084F86D106D2004F03BFE94F86D100220E7
:10CB700013F013FB0120FFF77FF99BF8110040F041
:10CB800001008BF81100F84880F80090BBF82000F5
:10CB9000602818D01DE094F86C20B5F9000002EB75
:10CBA0008202B0EB420FE5DB90FBF1F0401CC1B21A
:10CBB00084F86C106C2004F013FE94F86C100120C3
:10CBC00013F0EBFAD6E7297884F86010602004F0BF
:10CBD00007FEBBF820006F280DD194F86F009BF87A
:10CBE0001310884207D204218BF8131084F89B108D
:10CBF0009B2004F0F5FDBBF82000922810D1B5F978
:10CC00000000DA49084001281FD00320B07184F8E1
:10CC100092900021922004F0E3FD04208AF80000A5
:10CC2000BBF8200082280ED1B5F9000001281ED0E3
:10CC3000022823D00021822004F0D2FD84F88290C3
:10CC400009208AF80000BDE8F09F86F8069084F875
:10CC5000927012F0F2FA002018F0EEF90121922001
:10CC600004F0BEFD0021822004F0BAFDD8E70121C6
:10CC7000822004F0B5FD84F88270E1E70221822071
:10CC800004F0AEFD84F88280DAE770B586B005F076
:10CC90006AFFB74CB74D03AA218C6B465E2902D1BF
:10CCA000207D012820D095292BD09B2936D000202B
:10CCB0005E3901EB810105EB81010D5C15540D1806
:10CCC000AD7A1D54401CC0B20A28F6D3012005F0ED
:10CCD0002BFF694603A806F0E2F8A549208CA64A76
:10CCE0001E315E2827D037E00020291891F84C64C7
:10CCF000165491F856141954401CC0B20A28F4D3A3
:10CD0000E4E70020291891F86064165491F86A1439
:10CD10001954401CC0B20A28F4D3D7E700202918C0
:10CD200091F87464165491F87E141954401CC0B2E2
:10CD30000A28F4D3CAE7237D73B1937992F8D150CE
:10CD4000AB4201D9957104E092F8CF50AB4200D2CA
:10CD5000957192790A800CE0832814D00A237228F6
:10CD600014D095281CD0822825D0922827D0125C78
:10CD70000A805E2805D1207D002802D17F480088E6
:10CD8000088006B070BD227C0A80F2E712F8995F35
:10CD9000527805EB022212B292FBF3F20A80E8E726
:10CDA00092F8595292F85A2205EB022212B292FBE3
:10CDB000F3F20A80DDE792F882200A80D9E7704A10
:10CDC000927912B100220A80D3E701220A80D0E7CB
:10CDD00067485E21027B002A0AD00184664991F8E7
:10CDE0007F10032901D1952101840021017502E002
:10CDF00001840121017548E770B5012005F094FE1A
:10CE0000022005F091FE5A49088C942801D10A7B32
:10CE100042B10D7B00246323574A012D07D05E28C1
:10CE200016D019E05E2008840120087525E092F8EC
:10CE30007F20032A02D00B840C751EE0952804D0B5
:10CE40009B28F9D195200884F6E79B200884F3E716
:10CE50000D7D0DB10C7510E092F87F40042C0FD0C1
:10CE6000602831D09223822830D0832836D072288F
:10CE700036D0922837D0401C0884BDE8704004E7C3
:10CE80005E2806D0A0F16802022A05D2401C088460
:10CE9000F3E769200884F0E76A2806D0A0F16C0265
:10CEA000022A05D2401C0884E7E76C200884E4E7E6
:10CEB000822801D10A7C22B16E28DED19420088418
:10CEC000DBE784200884D8E70B84D6E792F8830058
:10CED00010B183200884D0E70B84CEE70B84CCE725
:10CEE00076200884C9E793200884C6E72DE9F0413D
:10CEF000012005F019FE022005F016FE1C491E4E09
:10CF00005E22087B88B196F87F00032801D00A844E
:10CF100027E0088C952802D09B2803D021E09B2095
:10CF200008841EE0952008841BE0088C00235E28FE
:10CF300005D10C7D1CB1942008840B7511E05E288E
:10CF400001D10C7DF4B196F87F7082248325042FE3
:10CF50001BD063283ED092283FD0762845D0401E73
:10CF60000884BDE8F04190E67300002001000080D5
:10CF7000280000205EFC0208607F00205E02002086
:10CF80009616002001200875EBE7682806D0A0F16E
:10CF90006902012A05D8401E0884E2E70A840B755D
:10CFA000DFE76C2806D0A0F16D02012A05D8401EEB
:10CFB0000884D6E76A200884D3E7942805D092280D
:10CFC000CFD1087C20B10D84CBE76E200884C8E760
:10CFD0000C84C6E760200884C3E796F88300012824
:10CFE00001D00C84BDE70D84BBE774200884B8E74A
:10CFF0007CB5FB4A47F6196402F11E01108CB1F9A9
:10D0000000104FF6FF75772867D012DCA0F15E00A4
:10D0100019282DD2DFE800F03361612C2C6193F7E1
:10D0200061612C2C61612C2C4E616868612C612C33
:10D030006100802851D009DCA0F17800082817D2BF
:10D04000DFE800F04B5D4B4B4B4B4BF994285FD026
:10D0500008DC822870D0832835D092286DD09328A0
:10D0600006D155E09B2873D0E52836D0E62834D089
:10D0700002B02022BDE87040002005F095BD107D73
:10D0800030B102B02022BDE87040002005F08CBD18
:10D09000D44890F86E0030B102B04622BDE870402E
:10D0A000002005F081BD02B04322BDE870400020A1
:10D0B00005F07ABD41B1CDE90054CBA3C2220021D5
:10D0C000012004F06FFF7CBDCDE90054C8A3C2224B
:10D0D0000021012004F066FF7CBD02B02022BDE8E3
:10D0E0007040002005F060BD0A2091FBF0F002B016
:10D0F00001B2BDE870402022002005F055BDCDE909
:10D100000054BDA3C2220021012004F04BFF7CBDCE
:10D11000C80708D0CDE90054B8A3C22200210120DD
:10D1200004F040FF7CBDCDE90054B5A3C22200212C
:10D13000012004F037FF7CBD46E065E008E0CDE962
:10D140000054B0A3C2220021012004F02BFFF2E71B
:10D150000529F0D2DFE801F0030C151E2700CDE908
:10D160000054AAA3C2220021012004F01BFFE2E721
:10D17000CDE90054A6A3C2220021012004F012FF31
:10D18000D9E7CDE90054A4A3C2220021012004F074
:10D1900009FFD0E7CDE90054A1A3C222002101205C
:10D1A00004F000FFC7E7CDE900549FA3C22200218D
:10D1B000012004F0F7FECDE900549BA3C222002118
:10D1C000012004F0EFFEB6E701290AD0022911D0B0
:10D1D000CDE9005496A3C2220021012004F0E2FE12
:10D1E000A9E7CDE9005494A3C2220021012004F054
:10D1F000D9FEA0E7CDE9005491A3C222002101206D
:10D2000004F0D0FE97E71DE08F480140012909D0C6
:10D21000CDE900548DA3C2220021012004F0C2FEFA
:10D2200089E708E0CDE900548AA3C2220021012049
:10D2300004F0B8FE7FE702B02022BDE870405A201B
:10D2400005F0B2BCC1B101291FD0022926D00329A3
:10D250002DD0042934D005293BD0062942D00729F6
:10D2600049D008298CD1CDE900547CA3C2220021E9
:10D27000012004F097FE5EE7CDE9005479A3C222B5
:10D280000021012004F08EFE55E7CDE9005477A37C
:10D29000C2220021012004F085FE4CE7CDE90054B4
:10D2A00074A3C2220021012004F07CFE43E7CDE9F3
:10D2B000005472A3C2220021012004F073FE3AE759
:10D2C000CDE900546FA3C2220021012004F06AFEC0
:10D2D00031E7CDE900546DA3C2220021012004F002
:10D2E00061FE28E7CDE900546AA3C2220021012093
:10D2F00004F058FE1FE7CDE9005468A3C2220021C4
:10D30000012004F04FFE16E770B5664D354C00263F
:10D31000297894F87F000939122951D2DFE801F009
:10D32000090C505015180F1B122025503F4245483C
:10D330004B4EFEF7F1FD43E0FEF756FE40E0FEF7F0
:10D34000F2FE3DE0FEF717FF3AE0FEF786FF37E01A
:10D35000FEF7DDFF34E0052832D0FEF722FF2FE094
:10D3600005282DD0FEF74FFF2AE005F0FCFBFFF764
:10D370002FFD94F87F001A4C40B1042806D00228F3
:10D3800008D0032806D0052804D019E02673FFF73B
:10D390001FFD15E0FFF71CFD0120207310E0FFF7D3
:10D3A0002BFD0DE0FFF7A2FD0AE0FFF729F907E0EA
:10D3B000FFF707F804E0FFF715FA01E0FFF712FAAC
:10D3C0002E7070BD00218438374A072879D2DFE8F3
:10D3D00000F0046D716F73757700918871E0000043
:10D3E00028000020607F00202D462D200000000036
:10D3F0002D432D2000000000344100004E4F00005E
:10D400005945530031303020200000004F6666003F
:10D410004D6F6465310000004D6F6465320000009F
:10D420004D6F6465330000004175746F00000000AB
:10D4300052533438350000005A49474245450000F0
:10D44000204155544F000000010000804D4F4442E0
:10D45000555300004241434E4554000031343430AE
:10D460003020000039363030202000003139323091
:10D47000302000003338343030200000353736306B
:10D48000302000003131353230302000373638302E
:10D49000302000003132303020000000343830308D
:10D4A00020000000F80000208C110020917908E095
:10D4B000117A06E0D17904E0117802E0517800E0B9
:10D4C000917808B2704710B503F0EDFF802004F0AA
:10D4D00064F804F015F808B1002010BDFE2004F037
:10D4E0005CF804F00DF808B1002010BD03F0F1FF66
:10D4F000012010BD10B5044603F0D5FF802004F0D4
:10D500004CF803F0FDFF08B1002010BD3CB1F52040
:10D5100004F043F803F0F4FF28B1002010BDF3201D
:10D5200004F03BF8F6E703F0D4FF012010BD70B51E
:10D530000E4603F0B8FF812004F02FF803F0E0FF5F
:10D54000012004F04BF84FF6FF7101EA002501209D
:10D5500004F044F840EA0504002004F03FF803F02A
:10D56000B8FF3480012070BD01F00203834201D076
:10D570000020704721F0030150B140F2E2404143E6
:10D58000C81701EB104000143C3810800120704790
:10D5900044F2A4404143C81701EB10400014A0F529
:10D5A00090504D3800B20A2190FBF1F01080EDE769
:10D5B00070B5054603F077FF812003F0EEFF03F01E
:10D5C0009FFF08B1002070BD012004F007F84FF65E
:10D5D000FF7101EA0024012004F000F8204484B225
:10D5E000002003F0FBFF03F074FF022D0AD044F289
:10D5F000A4404443FA480A2100EB244090FBF1F098
:10D6000080B270BD40F2E24044436FF03B0000EB5B
:10D610002440F5E710B503F046FF802003F0BDFF7E
:10D6200003F06EFF08B1002010BDE72003F0B5FF46
:10D6300003F066FF08B1002010BD03F034FF812025
:10D6400003F0ABFF03F05CFF08B1002010BD002029
:10D6500003F0C4FF044603F03CFFE0B210BD70B518
:10D660000646C1F1FA0021F002FC4FF03332DD4BE7
:10D6700021F050FC04460D46304621F0F8FB2246CE
:10D680002B4621F075F921F0C3FB00B270BD2DE9E6
:10D69000F0470446084622F033F8D34921F0FEFE55
:10D6A00021F062FE20F04AFF21F030F906462046C4
:10D6B00021F0DDFBCD4F0D46044600223B4621F014
:10D6C00029FC21F023F98146DFF82483DFF824A325
:10D6D000204629464246534621F04AF904460D4663
:10D6E000484621F041FE22462B4621F0FDF921F06B
:10D6F0000DF90146304621F063FE21F035FE8946E2
:10D70000064600223B4621F039FD04460D463046D0
:10D7100049464246534621F0FDFB22462B4621F066
:10D72000E3F921F075FB00B2BDE8F08763214FF407
:10D73000607004F055B8B0498A8892070BD08A7996
:10D740000D2A15D2DFE802F014393B3E4144474A26
:10D750004D5053575B008A790D2A09D2DFE802F059
:10D760000807090C0F1215181B1E21252900C8795E
:10D770007047C8791F307047C8793B307047C87907
:10D780005A307047C87978307047C87997307047F9
:10D79000C879B5307047C879D4307047C879F3304C
:10D7A0007047C87900F211107047C87900F5987079
:10D7B0007047C87900F5A7707047C8797047C87975
:10D7C0001F307047C8793C307047C8795B3070476C
:10D7D000C87979307047C87998307047C879B630C1
:10D7E0007047C879D5307047C879F4307047C87928
:10D7F00000F589707047C87900F231107047C87918
:10D8000000F24F10704700B5FFF795FF7B49888302
:10D81000C0F3C70200F007017948104400F22D4020
:10D82000FDF75EF908B1012000BD002000BD2DE923
:10D83000F043734D714901266A7A724FCB7C4FF0E9
:10D84000040C02F0FE044FF0000805280FD2DFE8B8
:10D8500000F00E03101E2100CE7342F0010068722A
:10D860008E7481F813C081F804C0BE71BE70BDE82B
:10D87000F08381F80FC06C7281F81280002BF6D013
:10D8800081F8138081F80480BE71BE70EFE70A2032
:10D89000C873ECE70C20C8736C7281F81280002BFF
:10D8A000E5D081F8138081F80480BE71BE70DEE798
:10D8B00010B5514A147A002C03D0127A012902D0F3
:10D8C00002E00722FAE708224D4907283AD2DFE8AA
:10D8D00000F039040D161F283100521E02EB4200E1
:10D8E000084490F8150400F007032BE0521E02EBE9
:10D8F0004200084490F81504C0F3C20322E0521E0F
:10D9000002EB4200084490F8160400F0070319E007
:10D91000521E02EB4200084490F81604C0F3C20302
:10D9200010E0521E02EB4200084490F8170400F089
:10D93000070307E0521E02EB4200084490F8170468
:10D94000C0F3C20358B210BD2DE9FC5F002611F0F0
:10D9500074FC2948007AE0B32748007A401E00F0A2
:10D96000FF09FFF750FF2849284ADFF894E0002814
:10D970007ED00EF2094003784478C3EB031304EB26
:10D9800083030B808378C478C3EB031304EB830316
:10D990004B8003794479C3EB031304EB83038B803F
:10D9A0008379C479C3EB031304EB8303CB80037A3D
:10D9B000447AC3EB031304EB83030B81C37A807AAD
:10D9C000C0EB001003EB80004881002409EB4908FC
:10D9D00000E01DE002EB4807385DFF281BD051E056
:10D9E000B3EDFFFF3333C3BF00007A4400A03140E2
:10D9F000CDCCCCCCCCFCA2408C1100202800002047
:10DA0000607F00209611002048090020E883002054
:10DA10004FF00609A5E7FF484FF6FF7120F81410F4
:10DA200008EB5400FC4A01901044009090F8150453
:10DA3000E10741D0C10801F0030119B3E1073ED06D
:10DA400000F0C70AFF2109EB4900800000EB440BFE
:10DA50000BEB020080F8B51380F8B6130BF2B5306B
:10DA600003F0BEFE0BF2B630FF2103F0B9FE00E07A
:10DA7000D9E0009880F815A40198514600F21540AD
:10DA800003F0AEFE641CE4B2062CA5D3DFF88C9341
:10DA900099F80000E8B30020DE4901F10E0231F8E8
:10DAA000103022F81030401CC0B20628F7D30524ED
:10DAB0004FF0000C00201FE000F00301BDE700F074
:10DAC000F80ABFE7411C32F8103032F811A0534574
:10DAD00011D90126938132F8113022F81030938940
:10DAE00022F8113017F800A03B1893F801B007F89E
:10DAF00000B083F801A0C8B2A042E3D3641EE4B230
:10DB00000CF1010C0CF0FF0CBCF1060FD2D300207D
:10DB100000E001E089F80000CEB30024BE4E08EB1F
:10DB20005402931993F81514E00706D0385D0128C4
:10DB300017D0D8B1FF281ED01FE0385D012803D0D0
:10DB400038B1FF280AD018E001F0F80040F00101D8
:10DB500013E001F0F80040F002010EE001F0F801DE
:10DB60000BE001F0C70040F0080106E001F0C7003B
:10DB700040F0100101E001F0C70183F8151402F232
:10DB8000154003F02DFE641CE4B2062CC7D3A44854
:10DB900041780078C0EB001001EB80049D4E0E36FA
:10DBA0003088A04207D87088A04204D901210846D5
:10DBB000FFF77EFEC5B27088A04207D8B088A042A9
:10DBC00004D901210220FFF773FEC5B2B088A0423C
:10DBD00007D8F088A04204D901210320FFF768FE8E
:10DBE000C5B2F088A04207D83089A04204D90121EB
:10DBF0000420FFF75DFEC5B23089A04207D87089C6
:10DC0000A04204D901210520FFF752FEC5B2708958
:10DC1000A04204D801210620FFF74AFEC5B22846DB
:10DC2000BDE8FC5F03E609EB49070EEB870000F255
:10DC3000B53003784478C3EB031304EB83030B8004
:10DC40008378C478C3EB031304EB83034B8003791D
:10DC50004479C3EB031304EB83038B808379C4798A
:10DC6000C3EB031304EB8303CB80037A447AC3EB47
:10DC7000031304EB83030B81C37A807AC0EB00109B
:10DC800003EB80004881002002EB4704225CFF2A5E
:10DC900019D0401CC0B20628F8D3DFF8808198F86C
:10DCA0000000E0B30020DFF86CB10BF10E0B31F88F
:10DCB00010202BF81020401CC0B20628F7D30522F4
:10DCC0000023002121E05548807CBDE8FC5FAEE5E3
:10DCD000481C3BF811C03BF81090CC4514D90126E4
:10DCE000ABF80CC03BF810C02BF811C0BBF80CC04F
:10DCF0002BF810C014F8019004EB010C9CF801A063
:10DD000004F801A08CF80190C1B29142E0D3521EF8
:10DD1000D2B25B1CDBB2062BD3D3002000E001E0C3
:10DD200088F80000D6B30026F14607EB560202EB56
:10DD3000090393F81514F00706D0A05D012817D049
:10DD4000D8B1FF281ED01FE0A05D012803D038B154
:10DD5000FF280AD018E001F0F80040F0010113E0BC
:10DD600001F0F80040F002010EE001F0F8010BE0D4
:10DD700001F0C70040F0080106E001F0C70040F0E4
:10DD8000100101E001F0C70183F8151402F21540FB
:10DD900003F026FD761CF6B2062EC6D32048417845
:10DDA0000078C0EB001001EB80041A4E0E3630886C
:10DDB000A04207D87088A04204D900210120FFF7B3
:10DDC00077FDC5B27088A04207D8B088A04204D9B8
:10DDD00000210220FFF76CFDC5B2B088A04207D831
:10DDE000F088A04204D900210320FFF761FDC5B2ED
:10DDF000F088A04207D83089A04204D9002104202D
:10DE0000FFF756FDC5B23089A04210D87089A042F4
:10DE10000DD907E048090020607F0020280000207D
:10DE20008C11002000210520FFF742FDC5B270894A
:10DE3000A04204D800210620FFF73AFDC5B22846CB
:10DE4000FFF7F5FC98F80200854204D01E49012036
:10DE500008718870487088F80250BDE8FC9FF0B5E2
:10DE600003461A481A4CC51895F86702FF2824D0B3
:10DE7000002658B1411E012705290BD2C9B2154809
:10DE8000FCF72EFE012803D0E65416E0E65414E019
:10DE9000E75412E01049062806D1B1F90020002A03
:10DEA00001DDE75400E0E654072806D1B1F902008D
:10DEB000002801DDE75400E0E65495F867020028E9
:10DEC00001D16420E054F0BD96110020607F002055
:10DED0006409002090020020BE0000202DE9F041DE
:10DEE000FB4C0023A370E370FB4D3C24F94F182634
:10DEF00005EB8203002904D0012939D0022968D119
:10DF000057E0B0FBF4F104FB110197F802C0614443
:10DF1000C9B2B1FBF4FCB1FBF4F804FB1811D970E1
:10DF2000B0FBF4F104FB1101401A80B2B0FBF4F035
:10DF3000B0FBF4F104FB1101614497F801C06144A6
:10DF4000C9B2B1FBF4FCB1FBF4F804FB18119970F1
:10DF5000B0FBF4F0397860440844C0B2B0FBF6F18D
:10DF6000B0FBF6F406FB1400587005F8221030E000
:10DF7000B978D970B0FBF4F104FB110197F801C036
:10DF80006144C9B2B1FBF4FCB1FBF4F804FB181115
:10DF90009970B0FBF4F0397860440844C0B2B0FB2B
:10DFA000F6F1B0FBF6F406FB1400587005F82210E9
:10DFB0000FE0B978D9707978997039780844C0B28F
:10DFC000B0FBF6F1B0FBF6F406FB1400587005F850
:10DFD0002210D8783B2801D13A20D870BDE8F081D2
:10DFE00010B5BB4BBC49BB4A002814D011F82040E7
:10DFF000DB789C422FD101EB800013784178994265
:10E0000027D181785378994221D1C078917888427C
:10E010001BD8012010BD08789B78984213D148780E
:10E02000137898420DD188785378984207D1C878F0
:10E030009178884201D8012010BD002010BD002039
:10E0400010BD002010BD002010BD002010BD00201C
:10E0500010BD002010BD002010BD2DE9F14FDFF8EC
:10E06000708298F80C0001285AD10024814608F1EA
:10E070003E0B4FF0000A08F11A06984F4DE0651C60
:10E08000E8B2FFF7ADFF012801D1315D11B10128E0
:10E090002CD041E097F8DB00032813D017F8CB0F02
:10E0A000797800EB012080B2A8F8240006F80490EB
:10E0B000397ACB3F0122FFF711FF97F8DB000228E6
:10E0C0000DD029E006F80490EAB23BF814000021D4
:10E0D000FFF704FF7E483B3000F80490EDE706F8B8
:10E0E00004A088F80AA088F80CA015E0305D01288B
:10E0F00012D197F8DB00032814D017F8CD0F7978E8
:10E1000000EB012080B2A8F8240006F804A0B97939
:10E11000CD3F0122FFF7E2FEECB200988442AED37D
:10E12000BDE8F88F6A48423030F8140030B106F884
:10E1300004A0EAB20021FFF7D1FEEDE7EAB23BF816
:10E1400014000021FFF7CAFEE6E7D21C884205D181
:10E15000D1B25F4800221830FCF7B5BCD1B25C48A0
:10E1600001221830FCF7AFBC10B50446002903D0DB
:10E1700057490020323108555548012221461830B0
:10E18000FCF7A1FCE41CE1B251480022BDE81040BC
:10E190001830FCF798BC10B504464D482630015D98
:10E1A0004F48005D821C91420DD94948002221460A
:10E1B0001030FCF788FC214645480122BDE810409C
:10E1C0001230FCF780BC801E81420DDA40480122EB
:10E1D00021461030FCF777FC21463D480022BDE87F
:10E1E00010401230FCF76FBC394800222146103035
:10E1F000FCF769FC214636480022BDE81040123089
:10E20000FCF761BC2DE9F04F89B00446334EDFF8CE
:10E21000C09096F86B00002807D0012844D0314FF9
:10E2200002287ED0032810D1AAE099F8050006281C
:10E230000CD096F8A903022815D0012813D0204647
:10E24000FFF7A9FF0120FFF7A6FFC1E02048012248
:10E2500000211030FCF737FC1D4800221146123017
:10E26000FCF731FCB4E00120FFF795FF96F8A90315
:10E2700002280CD01648012200211030FCF723FCA4
:10E280001348002211461230FCF71DFCDAE7104853
:10E29000002211461030FCF716FC0D480122002127
:10E2A0001230FCF710FCCDE70120FFF774FF99F85E
:10E2B0000400C8B10648002211461030FCF703FCE8
:10E2C0000348012200211230FCF7FDFB17E028E093
:10E2D000720000208C1100206D090020607F00205A
:10E2E000AE030020B803002001220021FE48FCF705
:10E2F000EAFBFD4800221146801CFCF7E4FB99F87C
:10E300000B0070B3401E89F80B0000221146F6483E
:10E31000FCF7D9FBF44800221146801CFCF7D3FB24
:10E3200056E096F89F02052804D096F89E0205282C
:10E3300007D00AE07888012801D0002505E00125F2
:10E3400003E0388801280DD000256DB10022114668
:10E35000E548FCF7B8FBE44801220021801CFCF7EB
:10E36000B2FB35E00125F0E701220021DE48FCF791
:10E37000AAFBDD4800221146801CFCF7A4FB27E025
:10E380000221DA48FCF7ACFB10B9012089F807003C
:10E3900096F89F02052804D096F89E02052807D01B
:10E3A0000AE07888012801D0002505E0012503E076
:10E3B000388801285DD00025F5B301220021CA4824
:10E3C000FCF781FBC84800221146801CFCF77BFB50
:10E3D000A020A0EB4407C548C349D438C44AC05D57
:10E3E000253104EB440B02EB4B08002628B306282A
:10E3F00056D010F808000855C81C12F81B2002550A
:10E40000DFF8E4A20AF1160A0AF10F011AF8040073
:10E41000095D0AF10905884204D305F10901095D86
:10E42000884224D9B148D43890F87900022801D024
:10E4300004283DD8214601E01DE028E0B9F812008B
:10E44000FCF730FB30B1A8481AF804102830005D02
:10E4500081420CD32146B9F81000FCF723FB38B3F6
:10E46000A1481AF804102530005D814220D92E55AC
:10E4700069E10125A0E7002211469B48FCF723FB38
:10E48000994801220021801CFCF71DFBA0E796485B
:10E49000642228300255964810F81B000855AFE753
:10E4A0000E55934810F81B208F4828300255A7E7D7
:10E4B0002146B9F81000FCF7F5FAD0B30021A120ED
:10E4C0008A4AA0EB4400D43ADFF824E2105C05ABA2
:10E4D00008E0D25D01EB4B0C724412F80C205A5448
:10E4E000491CC9B2814AD43A8842F2D80022C0F10C
:10E4F000060C06E003EB020B022100F80B10521C85
:10E50000D2B29445F6DC1AF804004FF0030E03284B
:10E5100002D802460AF804E01AF804009DF819C06F
:10E52000CDF820C0ACF1020C604503DA0621295574
:10E530001BE06FE09DF81410884201D92E5514E0BD
:10E54000002103EB010B9BF801B0584509D913F8E2
:10E5500001B0ABF1020B584503DA01F1010B05F8EC
:10E5600004B0491CC9B20429EBD39DF814108B1ECA
:10E57000984207DB884205D8295D012902D009B1FC
:10E58000012129559DF815108B1E984208DB884201
:10E5900006D8295D012903D0022901D0022129557D
:10E5A0009DF816108B1E984208DB884206D8295D1C
:10E5B000022903D0032901D005F804E09DF81710C3
:10E5C0008B1E984208DB884206D8295D032903D0B8
:10E5D000042901D0042129559DF818108B1E98425A
:10E5E00008DB884206D8295D042903D0052901D01B
:10E5F00005212955604509DB0899884206D8295D1F
:10E60000052903D0062901D006212955032801D167
:10E610000AF804202146B9F81200FCF743FAE8B3DF
:10E620000020324905AAD439C95D04E018F8003049
:10E630001354401CC0B28142F8D800206623C1F1B7
:10E64000060705E002EB000C01F80C30401CC0B2DC
:10E650008742F7DC9DF819701AF8040007F1020CE4
:10E66000604502D90C21295514E09DF81410884208
:10E6700001D22E550EE0002153185B78984205D246
:10E68000535C9B1C984201D9CB1D2B55491CC9B228
:10E690000429F1D39DF81410884200E053E008D318
:10E6A000891C884205D8295D072902D009B10721B4
:10E6B00029559DF81510884209D3891C884206D82F
:10E6C000295D072903D0082901D0082129559DF883
:10E6D0001610884210D3891C88420DD8295D08295C
:10E6E0000AD0092908D005E08200002034800020EB
:10E6F00079090020092129559DF81710884209D36E
:10E70000891C884206D8295D092903D00A2901D02D
:10E710000A2129559DF81810884209D3891C88427E
:10E7200006D8295D0A2903D00B2901D00B212955D0
:10E73000B84208D3604506D8285D0B2803D00C28C2
:10E7400001D00C202855FE4F0DF11C0A385D0AF847
:10E7500004002146B9F81800FCF7A4F978B1214665
:10E76000B9F80E00FCF79EF948B9385DB8B1401C05
:10E770003855F348002221461A38FCF7A4F904F171
:10E78000030808F0FF01B9F81800FCF78BF970B323
:10E790002146B9F80E00FCF785F9D8B127E0285DCD
:10E7A000062805D92146B9F81600FCF77BF970B1A7
:10E7B000285D401E0628DCD22146B9F81400FCF77B
:10E7C00071F90028D5D1385D401C3855D1E70720B4
:10E7D0003855CEE7385D072815D008B1401E3855AA
:10E7E000D74808F0FF0100221A38FCF76CF9285DC1
:10E7F0000D286ED2DFE800F06D091E3A586E8BA42A
:10E80000B8D5F6EFEE003E55EAE7385D401E062823
:10E810000BD2CB48002221461A38FCF754F9385D58
:10E8200022460121FFF791FC2EE101212046FFF74E
:10E830009BFC29E1385D811E05290BD2C0480022CE
:10E8400021461A38FCF73FF9385D22460221FFF7CE
:10E850007CFC19E1012804D001212046FFF784FC4B
:10E8600012E100212046FFF77FFC0DE1385DC11E5B
:10E8700004290BD2B248002221461A38FCF723F9AA
:10E88000385D22460321FFF760FCFDE0022806D038
:10E89000012804D001212046FFF766FCF4E00021A6
:10E8A0002046FFF761FCEFE0385D011F03290BD222
:10E8B000A348002221461A38FCF705F9385D2246A4
:10E8C0000421FFF742FCDFE001212046FFF74CFC6A
:10E8D000DAE0C0E0385D411F02290BD298480022DF
:10E8E00021461A38FCF7EFF8385D22460521FFF77C
:10E8F0002CFCC9E0401E032804D800212046FFF765
:10E9000033FCC1E001212046FFF72EFCBCE0385D5E
:10E91000062807D0401E04280DD800212046FFF706
:10E9200023FCB1E08648002221461A38FCF7CBF8D8
:10E9300006203855A8E001212046FFF715FCA3E08A
:10E94000385D06280BD97E48002221461A38FCF78C
:10E95000BAF8385D22460721FFF7F7FB94E0012162
:10E960002046FFF701FC8FE0385D07280DD9744879
:10E970004FF000022146A0F11A00FCF7A4F8385D20
:10E9800022460821FFF7E1FB7EE005D14FF00001B0
:10E990002046FFF7E9FB77E001212046FFF7E4FB83
:10E9A00072E0385D08280DD965484FF00002214615
:10E9B000A0F11A00FCF787F8385D22460921FFF71D
:10E9C000C4FB61E009D0072807D001212046FFF7EA
:10E9D000CBFB59E02EE019E004E000212046FFF7D0
:10E9E000C3FB51E0385D09280BD955480022214668
:10E9F0001A38FCF768F8385D22460A21FFF7A5FBB4
:10EA000042E000212046FFF7AFFB3DE0385D0A28D9
:10EA10000BD94B48002221461A38FCF754F8385DD0
:10EA200022460B21FFF791FB2EE000212046FFF745
:10EA30009BFB29E0385D0B2808D94148002221467C
:10EA40001A38FCF740F80C2038551DE0002120460C
:10EA5000FFF78AFB18E03A48002221461A38FCF7F3
:10EA600032F8385D38B1364808F0FF0101221A3813
:10EA7000FCF729F808E0285D3855314808F0FF0117
:10EA800000221A38FCF71FF81AF80400395D884292
:10EA900019D02B4901200931087048708870284826
:10EAA000012221462438FCF70EF80A2089F80000DC
:10EAB0000220CDE9000602960023642221A1244809
:10EAC000039608F050FF385D30BB1AF80400DFF8F9
:10EAD0007080411EA8F10608A8F1030A06291CD27D
:10EAE000DFF870B09BF8660048B101222146A8F11A
:10EAF0001800FBF7E8FF9BF8660008F804009BF895
:10EB0000670048B10E48012221461C38FBF7DBFFA5
:10EB10009BF867000AF804002AE0072828D3DFF8EA
:10EB200034B09BF8660048B10548012221461C38E4
:10EB3000FBF7C9FF9BF866000AF804000CE0000030
:10EB4000A40000205374617465537769746368008E
:10EB50009DA90008607F00209BF8670040B101225A
:10EB60002146F948FBF7AFFF9BF8670008F804005F
:10EB700099F8010000280ED1A9F81860A9F81460CE
:10EB8000A9F816602878072800D32E70285D38551C
:10EB9000012089F8010009B0BDE8F08F2DE9FF4F91
:10EBA00081B081464D460024DFF8A083DFF898B39A
:10EBB00008F1D6000BF1270BA246009084B198F81B
:10EBC000CD0098F8CE1000EB0126049800F00F015C
:10EBD0000398052919D2DFE801F00D0F1113170072
:10EBE00098F8CB0098F8CC1000EB012602980109A8
:10EBF0004846EEE7002508E0642506E0054604E007
:10EC0000322101EB500500E04508CF48083005559A
:10EC1000002739460098FBF763FF012807D108EB6E
:10EC2000070090F8B910032901D190F88B511CB15D
:10EC30007F1CFFB2052FECD398F8D310012902D026
:10EC4000022904D006E0C6EB0610860002E04FF46D
:10EC500061604643642206FB05F0B0FBF2F0BA4F58
:10EC600080B22A3727F81400C5F164037343B3FB5D
:10EC7000F2F23B1D23F8142088B185B11BF8042063
:10EC8000012A0CD1A3F1420201261673621CD2B2F2
:10EC9000FFF724F9A7F1240006550BF804A037F874
:10ECA000140000B11DB9A848801D00F804A0641C20
:10ECB000E4B2022C82D305B06EE72DE9F34F81B0A8
:10ECC0000027DFF884A2DFF88892DFF880B20AF12B
:10ECD0001E0A0BEB0700009010F8B74F007B0728C7
:10ECE00014D002987900005DC84000F00300022CA7
:10ECF0000ED24FF0A001A1EB44011BF801604FF0D0
:10ED0000A101A1EB44011BF8018006E00198EEE7A8
:10ED100003D19BF89C609BF89D808E49097801295E
:10ED20000CD19BF8B710012901D107B902209BF83B
:10ED3000B810012902D1012F00D1022030B10128E1
:10ED40007ED0022804D0032801D164E00025CDE064
:10ED50007D487D4912302131005D095D884235D200
:10ED600016B91AF80410E9B11AF8041004EB4405B6
:10ED7000494406EB4502114411F8011C081A4FF4EE
:10ED80007A71FBF78DFE09EB450106EB0802114491
:10ED900011F8011C90FBF1F54FF47A70854200D90F
:10EDA0000546A3E004EB440508EB4501494411F88E
:10EDB000011C081A4FF47A71FBF772FE09EB45014A
:10EDC000414411F8011C90FBF1F5E5E75E4924315F
:10EDD000095D88421DD91AF8041004EB44056FF050
:10EDE0000602494402EB4502895C401A4FF47A71ED
:10EDF000FBF756FE09EB4501314411F8011CC1F146
:10EE0000640190FBF1F5B5F57A7F6FD94FF47A750F
:10EE10006CE000256AE04C484B4912302131005D1E
:10EE2000095D884239D20EB31AF8041004EB440588
:10EE3000494406EB4502114411F8011C081A00E090
:10EE400052E04FF47A71FBF72BFE09EB450106EB1C
:10EE50000802114411F8011C90FBF1F505F5FA7553
:10EE60004FF47A70854241D905463FE01AF8041004
:10EE700004EB4405494408EB4502114411F8011C18
:10EE8000081A4FF47A71FBF70BFE09EB4501414478
:10EE900011F8011C90FBF1F5E0E72B492431095DE5
:10EEA00088421FD91AF8041004EB44056FF00602DB
:10EEB000494402EB4502895C401A4FF4FA71FBF7B2
:10EEC000EFFD09EB4501314411F8011CC1F164016A
:10EED00090FBF1F505F5FA754FF47A70854205D986
:10EEE000054603E0002501E04FF47A75009890F89C
:10EEF000C300072830D002984021B940005D084087
:10EF000000B31148104912302131005D095D88427B
:10EF10003BD2C6B11AF8041004EB4404494406EB92
:10EF20004402114411F8011C081A4FF4FA71FBF75E
:10EF3000B7FD09EB440108EB0602114411F8011C6E
:10EF400090FBF1F545E009E086000020607F00209D
:10EF5000790900203F0200200020D1E71AF80410B0
:10EF600004EB4404494408EB4402114411F8011C29
:10EF7000081A4FF47A71FBF793FD09EB4401414401
:10EF800011F8011C90FBF1F523E0F749095D884277
:10EF90001ED91AF8041004EB44056FF00602494428
:10EFA00002EB4502895C401A4FF4FA71FBF778FDD9
:10EFB000A021A1EB44014FF0FF321BF8011002EB3E
:10EFC00045024944895CC1F1640190FBF1F500E020
:10EFD00000254FF47A70854200D90546009890F8D4
:10EFE0007B0011280DD0022817D003281FD0042839
:10EFF0002FD0284620F09CFBDC497A1D01EB8211C2
:10F0000048627F1CFFB2022FFFF463AE9BF8C3007F
:10F010000022D749022826D027E0680820F088FB84
:10F020000146D24A781D02EB80104162E9E705EB08
:10F0300085000621B0FBF1F0C83020F079FBCB4908
:10F040007A1D01EB82114862CA4A9042D9DD4A62B8
:10F05000D7E7C5F57A7020F06BFBC4497A1D01EB48
:10F0600082114862CDE70B881BB1032804D1488880
:10F0700010B9BE48C0F864219BF8C400022801D131
:10F080000B8823B1032805D14888002802D1B7484E
:10F09000C0F8A421BDE8FE8F30B5B749062813D0CB
:10F0A00091F87C10B44A4C1F642392F85E0392F8E6
:10F0B0005D23801A0C2C32D2DFE804F009111919F3
:10F0C000191919191919222691F87B10EAE7AB4989
:10F0D000B1F90010484390FBF3F000B230BDA849ED
:10F0E000B1F90010484390FBF3F000B230BDA04AE4
:10F0F000C91F32F91110484390FBF3F000B230BD44
:10F10000A048B0F9000030BD9F49098809B2891AAA
:10F110004FF47A72514391FBF0F000B230BD002001
:10F1200030BD2DE9F04F8BB00025019597489949E6
:10F13000914F02789648002A06D097F86C200280FA
:10F1400097F86D00088005E097F87120028097F825
:10F150007000088000242046FFF754F8641CE4B2D5
:10F16000032CF8D38048DFF800A23838AAF1060A49
:10F17000007A01280BD197F8A0008AF8000097F8D0
:10F18000C800C0EB00108100AAF1320041847A4926
:10F190009AF8000001F51C72734E01F5B0710E363D
:10F1A000CDE90912DFF8F091DFF8F0B1A6F12008FF
:10F1B000062828D899F80010C319C1EBC10202F241
:10F1C00003129A5C3280D1B10999415C059117F81C
:10F1D000A01F084498F8001010F80B00401A642192
:10F1E000FBF75EFC797817F8A029114411F80B1091
:10F1F00090FBF1F0C4B2642C2ED964242CE00A995F
:10F20000415C0591E3E799F80010C1EBC1021318C6
:10F2100097F8A120C2F106029B1A3B4493F80331F0
:10F220003380E9B3811A394491F8601105915B4943
:10F2300098F80020891F405C6421101AFBF730FC0D
:10F2400097F8A01011F80B10C1F1640190FBF1F0D8
:10F25000C4B2642C00D964244348DFF840A1801F65
:10F260000AF1060A4078062832D899F8001041B30E
:10F270004B49415C71800999415C039117F89E1FCD
:10F28000084498F8011010F80A00401A6421FBF7AE
:10F2900007FC797817F89E29114411F80A1000E04C
:10F2A00009E090FBF1F000F0FF0BBBF1640F35D9E2
:10F2B0004FF0640B32E0811A394491F870120591D5
:10F2C000B5E73849415C71800A99415C0391D5E703
:10F2D00099F80010F1B397F89F10C1F10601411A97
:10F2E000394491F82621728091F86011039198F8C1
:10F2F000011010F80B00081A6421FBF7D1FB97F8F6
:10F300009E1011F80A10C1F1640190FBF1F000F0B9
:10F31000FF0BBBF1640F01D94FF0640B12481F497A
:10F32000801F0C318078089106284ED899F800107B
:10F33000C9B11C493331415CB18017F89C1F0144AD
:10F340000898085C98F80210401A6421FBF7A8FBA3
:10F35000387800E028E079789C3F01440898085C00
:10F36000B4FBF0F04DE02CE0AA000020488400201F
:10F370001812002000007A44607F00205E02002006
:10F38000540000205C020020580200203A000020B7
:10F39000B4030020B60300203B00002078090020C1
:10F3A000868000203F82002097F89F10C1F106015F
:10F3B000411A394491F8DF22728091F8701203915A
:10F3C00095E7FC49415CB180B7E799F8001041B37B
:10F3D00097F89D10C1F10601411A394491F81213B2
:10F3E000B18098F8021010F80A00081A6421FBF79F
:10F3F00057FB97F89C200899515CC1F1640190FB80
:10F40000F1F097F8DB00DFF8B0A3C0B301210020D2
:10F4100002AA052816DA3B1893F8B930032B0AD054
:10F4200019E097F89D10C1F10601411A394491F88D
:10F430002013B180D5E7012902D0012150540AE000
:10F440000021FBE73B1893F87630112B03D10129FB
:10F4500065D001215054401C00B20728D9DB9DF82B
:10F4600008001AF80000E8B39DF809001AF8000037
:10F47000C8B3039B5A4619465846FFF78FFB002432
:10F48000DFF834B34FF0010A0BF1070BCA48005DF7
:10F49000032861D004286BD00BF804001BF804008B
:10F4A000214636F81000FBF7FDFA0246C248214615
:10F4B0003238FBF708FB641CE4B2072CE6D3BE48E5
:10F4C000BE4E52388079C0B3BB48523890F8200005
:10F4D00001900024381990F8B90001280DD00228B5
:10F4E0000BD001E01DE030E0214601A8FBF7F8FA5F
:10F4F00020F01EF906EB84114862641CE4B2052C6E
:10F50000E8D301210020DFF8B0B2ABF1380B0528B9
:10F5100060D23A1892F8B920032A48D068E0002156
:10F5200098E79DF809001AF8000038B15A462046BD
:10F53000039B0599FFF732FBA1E725E0059B2246D7
:10F5400019462046FFF72AFB99E722465846059BB5
:10F550000399FFF723FB92E798F8000098F8011051
:10F56000884202D20BF8045098E70BF804A095E704
:10F5700098F8000098F80110884202D90BF804505E
:10F580008CE70BF804A089E700248B485238B0F8C8
:10F5900020B02BFA04F000F0010020F0C9F806EBCF
:10F5A00084114862641CE4B2052CF2D3A9E7012956
:10F5B00008D001211BF80120012A05D006EB80129A
:10F5C000556215E00021F5E706EB80134FF07E52FF
:10F5D0005A620DE03A1892F87620112A08D1C9B182
:10F5E00000211BF80120012A16D006EB801255627B
:10F5F000401CC0B207288AD3002404F1B70007904A
:10F6000002F0EDF803280DD0079802F0E8F804287E
:10F6100016D022E00121E4E706EB80134FF07E5282
:10F620005A62E5E798F8000098F80110884203D282
:10F63000381980F8B75010E0381980F8B7A00CE0FE
:10F6400098F8000098F80110884203D9381980F81A
:10F65000B75002E0381980F8B7A0641CE4B2022C5D
:10F66000CBD35548DFF850A15238AAF1060A4079A9
:10F6700080B1062829D0AAF11A021178062953D898
:10F6800099F80000E0B34E48085C8DF8100004F0D3
:10F690000F0058E0BAF80000323000B2AAF80000BB
:10F6A0004FF47A71884201DDAAF80050BAF80200DE
:10F6B000323800B2AAF80200002801DAAAF80210D3
:10F6C0004FF4FA7008F004FF1AE197F8A602042834
:10F6D00017D0AAF8005097F8A702042817D0AAF864
:10F6E0000250BAF900104FF47A70814201DDAAF895
:10F6F0000000BAF90210814201DDAAF80200FFE021
:10F700000BE00620FFF7C8FCAAF80000E3E707209B
:10F71000FFF7C2FCAAF80200E3E729480E30085CB4
:10F720008DF8100020090EE099F80000E0B197F87C
:10F73000A100C0F10600081A384490F82D018DF898
:10F74000100004F00F0097F89F305178C3F10603C2
:10F75000CB1A06291AD899F800308BB1184BDB1D4B
:10F76000C95C8DF8111019E0200997F8A130C3F198
:10F770000603C91A394491F83B118DF81010E2E7DD
:10F780000C4B3A3BC95C8DF8111007E099F800105A
:10F79000C1B1D91991F834118DF811109178062959
:10F7A0001BD899F800209AB1024A1A3A895C8DF860
:10F7B00012101FE080820020C40000204884002036
:10F7C0008D800020D91991F8E6128DF81110E5E727
:10F7D000B94A895C8DF812100CE099F80020F2B15A
:10F7E00097F89D20C2F10602891A394491F8061350
:10F7F0008DF8121004A9FFF760FAB04805210690B1
:10F80000FBF76EF9B0B197F8620397F86313000243
:10F8100000B208441FF074FFC6F85C010DE097F8D1
:10F820009D20C2F10602891A394491F819138DF806
:10F830001210DFE7A248C6F85C0106210698FBF724
:10F840004FF958B197F8640397F86513000200B2B6
:10F8500008441FF055FFC6F89C0102E09848C6F81E
:10F860009C01984CA07901284AD197F8B70004A9C7
:10F870004FF06409095CC1F3011149B101292CD091
:10F8800004F13503DA1C022904D0032927D114E03E
:10F89000E58324E018F80010125C914203D9881A1D
:10F8A0004000E0831BE0185C814204D2C1F13200C9
:10F8B0004000E08313E0E58311E018F80010125CCB
:10F8C000914201D9E1830AE0185C814203D2C1F17F
:10F8D0006400E08303E0E58301E0A4F81E900721C3
:10F8E0000698FBF7FDF808B1607BE083B4F91E00D1
:10F8F000052801DAE58303E05F2801DDA4F81E9006
:10F900000024DFF8C481381990F8BE00012802D124
:10F910006E49097861B1022802D1B8F8001039B1F6
:10F92000032802D1B8F8021011B1042804D006E06F
:10F9300006EB841045622DE097F8DB1011B1052825
:10F940000AD00CE09BF80000012823D106EB8411BB
:10F950004FF07E5048621DE097F8DB1011B1062889
:10F960000DD017E021465A48FBF7BAF89BF8001073
:10F9700008401FF0DDFE06EB841148620AE097F8AC
:10F98000DB00022806D14F48807A012802D106EB1D
:10F9900084104562641CE4B2052CB4D30020DFF867
:10F9A00024914FF07E5899F809103A1892F8DC200B
:10F9B000022A04D101291CD006EB80125562401C9A
:10F9C000C0B20528F1D300243D4D002006EB841180
:10F9D00051F82020AA4217D051F8200010F0FF4F14
:10F9E0000CD0404514D1012221463948FBF75EF87E
:10F9F0000EE006EB8012C2F82480E0E700222146E8
:10FA00003348FBF753F803E0401CC0B21028DFD3A3
:10FA1000641CE4B2052CD8D399F80500002817D04F
:10FA20000524002006EB841151F82020AA4207D0BB
:10FA300051F820001FF028FE611F2AF8110003E092
:10FA4000401CC0B21028EFD3641CE4B2072CE8D3EA
:10FA50000BB0BDE8F08F1B4832300078011F02293F
:10FA600002D80A30C0B27047C11F022902D8C01E96
:10FA7000C0B27047A0F10A010229FAD8C01DC0B275
:10FA8000704770B50F4E0021308AFBF70BF8044623
:10FA90000A4DD63D95F8A10000B900240021708AD6
:10FAA000FBF700F828B1A41CE4B295F8A00000B957
:10FAB0000024204670BD000079820020368000209E
:10FAC00000007F4372000020181200203A0000203E
:10FAD000900200200D49086070470C49486070474B
:10FAE0000A498860704709494AF6AA2008607047A9
:10FAF00006494CF6CC400860704701460020034A96
:10FB0000D2680A4200D00120704700000030004057
:10FB1000B448016841F0010101604168B24A1140F6
:10FB200041600168B14A11400160016821F48021FF
:10FB30000160416821F4FE0141604FF41F018160C2
:10FB40007047A8490A6822F480320A600A6822F4E1
:10FB500080220A60B0F5803F07D0B0F5802F03D136
:10FB6000086840F4A02008607047086840F48030BE
:10FB7000086070470346002059099A4A01290AD0B3
:10FB800002290AD0516A03F01F02012393400B425D
:10FB900000D0012070471168F5E7116AF3E718B546
:10FBA000002000904FF4A0643120FFF7E3FF00999C
:10FBB000491C00910099A14201D00028F4D03120C5
:10FBC000FFF7D8FF08B1012018BD002018BD854AF5
:10FBD000116821F0F80141EAC000106070478449C3
:10FBE000086070477F4B5A6822F47C120843104328
:10FBF000586070477E49086670477A4A516821F01C
:10FC000003010143516070477648406800F00C00E2
:10FC10007047744A516821F0F00101435160704708
:10FC2000704A516821F4E0610143516070476D4AA8
:10FC3000516821F4605141EAC00050607047694A40
:10FC4000002903D0517A014351727047517A8143A0
:10FC5000517270476649D83108607047614A5168EF
:10FC600021F440410143516070475E490022203138
:10FC70000A7001F82029012805D0042802D10520A6
:10FC800081F820007047012081F820007047594911
:10FC90000860704753490A6A02430A62704755492F
:10FCA00044390860704710B54E4A516801F00C01A4
:10FCB000514B002927D0042927D0082927D00360D9
:10FCC000516801F0F00109094C4B5C5C0168E140AE
:10FCD0004160546804F4E064240A1C5D21FA04F4D1
:10FCE0008460546804F46054E40A1B5DD940C16028
:10FCF000526802F44042920B404B1B1F9A5CB1FBCE
:10FD0000F2F1016110BD0360DAE70360D8E75168E2
:10FD100001F47011536803F48033022404EB914121
:10FD200033B153689B0307D5354B59430160C7E78F
:10FD3000334B59430160C3E72F4B59430160BFE781
:10FD4000284A002903D05169014351617047516924
:10FD5000814351617047234A002903D091690143CF
:10FD60009161704791698143916170471D4A0029F3
:10FD700003D0D1690143D1617047D1698143D16119
:10FD80007047184A002903D0D1680143D1607047F9
:10FD9000D1688143D1607047124A002903D01169AC
:10FDA0000143116170471169814311617047114925
:10FDB0004039086070470E49C86470470949C871E6
:10FDC00070470848416A41F08071416270470146BE
:10FDD0000020044A92680A4200D00120704701497D
:10FDE00088727047001002400000FFF8FFFFF6FE27
:10FDF000000042428004424200127A00DE000020ED
:10FE000000093D004D4A002903D0118801431180AB
:10FE1000704711888143118070474848001D018850
:10FE200041F01001018070474448001D018821F015
:10FE300010010180704741481C3000883F4918314B
:10FE4000098840EA0140704700B50246FFF7E5FF28
:10FE50003A49100C18310880081D02805DF804EB47
:10FE6000E2E700B50246FFF7D8FF3449C2F303408A
:10FE700008310880081D02805DF804EBD4E700B566
:10FE80000246FFF7CAFF2D49100C20310880081DDB
:10FE900002805DF804EBC7E72848103000880007AF
:10FEA000010B2648143000880843704770B50024C1
:10FEB000224D2D1D06E0641CE4B2642008F008FB0E
:10FEC0001E2C02D828888006F5D570BD70B5002498
:10FED0001A4D2D1D288820F00800288006E0641C9B
:10FEE000E4B2642008F0F4FA1E2C02D82888000737
:10FEF000F5D570BD01460020104A121D12880A4235
:10FF000000D0012070470D49091D0A8882430A80EC
:10FF100070470A49091D0988C2B21140074A128870
:10FF2000024202D009B10120704700207047034906
:10FF3000091D0A8882430A8070470000002800409B
:10FF400010B5FE4988420AD1C41401212046FFF7AA
:10FF500018FF2046BDE810400021FFF712BFB0F1A6
:10FF6000804F0CD0F649884213D101210220FFF7BF
:10FF700013FF0021BDE810400220FFF70DBF012153
:10FF80000846FFF709FF0021BDE810400120FFF7F8
:10FF900003BFEC49884209D101210420FFF7FCFE90
:10FFA0000021BDE810400420FFF7F6BEE649884274
:10FFB00009D101210820FFF7EFFE0021BDE8104024
:10FFC0000820FFF7E9BEE149884209D1012110204C
:10FFD000FFF7E2FE0021BDE810401020FFF7DCBE75
:10FFE000DB49884209D101212020FFF7D5FE0021FD
:10FFF000BDE810402020FFF7CFBED64988420AD185
:020000040801F1
:10000000441401212046FFF7BCFE2046BDE8104005
:100010000021FFF7B6BED04988420AD10121CC04A5
:100020002046FFF7AEFE2046BDE810400021FFF756
:10003000A8BECA4988420AD101210C052046FFF713
:10004000A0FE2046BDE810400021FFF79ABEC4493B
:1000500088420AD101214C052046FFF792FE204636
:10006000BDE810400021FFF78CBEBE49884209D18F
:1000700001214020FFF790FE0021BDE81040402004
:10008000FFF78ABEB849884209D101218020FFF7D5
:1000900083FE0021BDE810408020FFF77DBEB349FC
:1000A00088420AD1841501212046FFF775FE2046BB
:1000B000BDE810400021FFF76FBEAD4988420AD16C
:1000C00001210C042046FFF75CFE2046BDE81040ED
:1000D0000021FFF756BEA74988420AD101214C04EE
:1000E0002046FFF74EFE2046BDE810400021FFF7F6
:1000F00048BEA14988420AD101218C042046FFF75D
:1001000040FE2046BDE810400021FFF73ABE10BD7A
:1001100030B50288894C8F4DA0420DD0A8420BD03B
:10012000B0F1804F08D0864B984205D0854B98425D
:1001300002D0854B984203D122F070034A881A43BB
:10014000824B984206D0824B984203D022F44073EF
:10015000CA881A4302808A8882850A880285A0425A
:100160000AD0A84208D0824A904205D0814A9042E3
:1001700002D0814A904201D1097A0186012181820F
:1001800030BD30B5028C22F001020284028C8388DB
:10019000048B24F0700424F003050C882C4322F017
:1001A00002020D8915434A882A43644DA8420BD0A8
:1001B000684DA84208D06E4DA84205D06D4DA842AA
:1001C00002D06D4DA8420FD122F008054A892A437A
:1001D00022F004058A882A4323F4807323F40073F1
:1001E0008D891D43CB892B4383800483C9888186F5
:1001F000028430BD70B5028C22F010020284028CA1
:100200008388048B24F4E04424F440760D884FF670
:10021000FF7404EA0525354322F020020E8904EA22
:10022000061616434A8804EA02123243434EB0428D
:1002300002D0484EB04217D122F080024E8904EA23
:100240000616164326F040068A8804EA0212324354
:1002500023F4806323F400638E8904EA86061E4338
:10026000CB8904EA8303334383800583C9880187EC
:10027000028470BD70B5028C22F480720284028CFC
:100280008388848B24F0700424F003040D882543B4
:1002900022F400720E894FF6FF7404EA0626164314
:1002A0004A8804EA02223243244EB04202D0294E48
:1002B000B04217D122F400664A8904EA022232438E
:1002C00022F480668A8804EA0222324323F48053AF
:1002D00023F400538E8904EA06161E43CB8904EAF0
:1002E0000313334383808583C9888187028470BD6B
:1002F00070B5028C22F480520284058C8288838B34
:1003000023F4E04323F440760C884FF6FF7303EAAE
:100310000424344325F400550E8903EA06362E439F
:100320004D8803EA05353543044EB04202D0094EEC
:10033000B04226D122F480468A891FE0002C014079
:100340000004004000080040000C00400010004085
:100350000014004000340140004C014000500140B6
:100360000054014000180040001C004000200040E4
:1003700000400140004401400048014003EA82126D
:10038000324382808483C988A0F84010058470BD00
:10039000828B22F440628283828B4FF6FF7303EAE2
:1003A00001210A4382837047F0B5048C24F4805401
:1003B0000484868B048C4FF6FF7505EA013726F41A
:1003C000734605EA0222324305EA03331343F74A30
:1003D00090420ED0F64A90420BD0B0F1804F08D038
:1003E000F44A904205D0F44A904202D0F34A904237
:1003F00005D124F40051394341F4805104E024F440
:1004000002420A4342F4805183830184F0BD828B0F
:1004100022F00C028283828B0A4382837047F0B5FC
:10042000048C24F480740484858B048C4FF6FF774D
:1004300007EA012625F0F30507EA031313432B43CC
:10044000DA4A90420ED0DA4A90420BD0B0F1804F97
:1004500008D0D84A904205D0D74A904202D0D74A15
:10046000904205D124F40071314341F4807104E0DD
:1004700024F420620A4342F4807183830184F0BD36
:10048000028B22F440620283028B4FF6FF7303EA71
:1004900001210A4302837047F0B5048C24F0100454
:1004A0000484068B048C4FF6FF7505EA011726F4C9
:1004B000734605EA0333334305EA02221A43BB4B72
:1004C00098420ED0BA4B98420BD0B0F1804F08D072
:1004D000B84B984205D0B84B984202D0B74B9842DF
:1004E00005D124F02001394341F0100104E024F04B
:1004F000A0030B4343F0100102830184F0BD028B83
:1005000022F00C020283028B0A430283704770B50B
:10051000048C24F001040484058B048C25F0F3057D
:100520004FF6FF7606EA031313432B439F4A90428C
:100530000ED09F4A90420BD0B0F1804F08D09D4A18
:10054000904205D09C4A904202D09C4A904205D1EC
:1005500024F002020A4342F0010104E024F00A02FE
:100560000A4342F001010383018470BD70B5054662
:100570000C468E48854209D08D48854206D0B5F19B
:10058000804F03D08B48854200D08B4820886188FB
:10059000A288238958B1042811D0082817D02846EA
:1005A000FFF702FFE1882846BDE87040F0E62846E4
:1005B000FFF7ADFFE1882846BDE870409FE7284679
:1005C000FFF76AFFE1882846BDE8704058E72846F3
:1005D000FFF725FFE1882846BDE8704017E72DE9C1
:1005E000F04107460C46002501266188002900D10C
:1005F0000225A288012A00D102262088238988B1F9
:100600003846FFF749FFE1883846FFF739FF23896D
:10061000324629463846FFF77AFFE1883846BDE87A
:10062000F0416CE73846FFF772FFE1883846FFF784
:1006300066FF2389324629463846FFF72DFFE188B9
:100640003846BDE8F0411BE710B50A884B88CC88D6
:100650001A438B8823431A430B891A434B89898990
:100660001A430A43A0F8442010BD4FF6FF71818061
:1006700000210180C180418001727047002101800A
:1006800041808180C180018141818181C181704728
:1006900000210180418001228280C1800181704758
:1006A0000021018041808180C1800181418181815F
:1006B0007047002904D0018841F001010180704792
:1006C000018821F0010101807047002905D030F830
:1006D000441F41F400410180704730F8441FC1F3CA
:1006E0000E0101807047002A03D082890A4382816B
:1006F000704782898A4382817047818270471143A3
:10070000A0F848107047002A03D082890A438281EA
:10071000704782898A4382817047018921F00701ED
:1007200001817047028922F070020A4302817047FA
:1007300000B503461846FFF7F5FF188940F007009B
:10074000188100BD70B50D4604461146602D0CD0D1
:1007500001222046FFF7DBFE29462046FFF7E2FF95
:10076000208940F00700208170BD01222046FFF75C
:1007700093FEF1E730B50489E4B24FF6FF7505EA60
:10078000032313430B432343038130BD10B50446B9
:100790002046FFF7EFFF208920F0070040F0070018
:1007A00020F0700040F07000208110BD002C01404E
:1007B000003401400004004000080040000C0040EC
:1007C00010B504462046FFF7D5FF208940F480404D
:1007D0002081EAE7018582827047028822F0700258
:1007E0000A430280704770B50589048B068C25F09A
:1007F00007050D434FF6FC410C4040F201110C433C
:1008000026F022064FF6FF7101EA0311114331432E
:1008100005810483018470BD028B22F070020A43BB
:1008200002837047028B22F4E0424FF6FF7303EA23
:100830000121114301837047828B22F070020A4329
:1008400082837047828B22F4E0424FF6FF7303EA03
:100850000121114381837047002904D0018841F0B0
:10086000800101807047018821F08001018070477C
:10087000002904D0818841F004018180704781887B
:1008800021F0040181807047002904D0818841F063
:10089000080181807047818821F0080181807047BC
:1008A000002904D0818841F001018180704781884E
:1008B00021F0010181807047028B22F008020A4377
:1008C00002837047028B22F400624FF6FF7303EA43
:1008D0000121114301837047828B22F008020A43F1
:1008E00082837047828B22F400624FF6FF7303EA23
:1008F0000121114381837047028B22F004020A43D5
:1009000002837047028B22F480624FF6FF7303EA82
:100910000121114301837047828B22F004020A43B4
:1009200082837047828B22F480624FF6FF7303EA62
:100930000121114381837047028B22F080020A4318
:1009400002837047028BC2F30E024FF6FF7303EA75
:100950000121114301837047828B22F080020A43F8
:1009600082837047828BC2F30E024FF6FF7303EA55
:100970000121114381837047028C22F002020A4355
:1009800002847047028C22F008020A4302847047F6
:10099000028C22F020024FF6FF7303EA011111438B
:1009A00001847047028C22F080024FF6FF7303EA45
:1009B0000111114301847047028C22F400724FF63A
:1009C000FF7303EA0121114301847047028C22F472
:1009D00000624FF6FF7303EA01211143018470475F
:1009E000028C22F400524FF6FF7303EA01311143E7
:1009F0000184704710B501238B40048C9C43048410
:100A0000038C8A4013430384CFE610B504238B4044
:100A1000048C9C430484038C8A4013430384C4E6FF
:100A200030B500F1180301248C40058CA5430584E2
:100A3000002911D008290FD0091FC1F34E00184416
:100A4000016821F4E041016001684FF6FF7303EA99
:100A500002221143016030BD03EB5100016821F017
:100A60007001016001681143016030BD002904D0AC
:100A7000018841F0020101807047018821F00201E4
:100A800001807047002904D0018841F004010180F1
:100A90007047018821F0040101807047002904D0CB
:100AA000818841F0800181807047818821F0800138
:100AB00081807047028822F00802028002880A437F
:100AC00002807047828822F07002828082880A4306
:100AD00082807047028922F00702028102890A435C
:100AE00002817047028922F08002028102890A4352
:100AF0000281704781847047818570478186704785
:100B00000187704781877047A0F8401070470288BE
:100B100022F44072028002880A4302807047808E6D
:100B20007047008F7047808F7047B0F84000704763
:100B3000808C7047008D704702460020128A0A425E
:100B400000D001207047C94301827047024600204F
:100B5000138A0B4092890A40002B02D0002A00D051
:100B600001207047C94301827047000010B5E14978
:100B700088420AD101218C032046FFF702F9204662
:100B8000BDE810400021FFF7FCB8DB4988420AD1DC
:100B900001214C042046FFF7FFF82046BDE8104035
:100BA0000021FFF7F9B8D54988420AD101218C0408
:100BB0002046FFF7F1F82046BDE810400021FFF77E
:100BC000EBB8CF4988420AD10121CC042046FFF777
:100BD000E3F82046BDE810400021FFF7DDB8C94921
:100BE00088420AD101210C052046FFF7D5F820469E
:100BF000BDE810400021FFF7CFB810BD30B585B07B
:100C000004460D46208A4CF6FF710840E9880143EE
:100C10002182A0894EF6F3110840A9882A89114340
:100C20006A8902431143A181A08A4FF6FF4108401F
:100C3000A9890143A1826846FFF735F8AD4884428F
:100C400001D1039800E00298A189090408D500EBBE
:100C5000C00101EB001029684900B0FBF1F007E08A
:100C600000EBC00101EB001029688900B0FBF1F036
:100C70006422B0FBF2F109010B096FF018056B4318
:100C800000EB8300A3891D044FF0320307D503EB6B
:100C9000C000B0FBF2F000F00700084306E003EBF1
:100CA0000010B0FBF2F000F00F000843208105B007
:100CB00030BD4FF41651016000218180C180018157
:100CC0000C2242818181704710B5038A4FF2FF02E6
:100CD00013400A884C8822438C88C9880C432243DD
:100CE0001A43028210BD0021018041808180C180B1
:100CF0007047002904D0818941F4005181817047F7
:100D0000818921F400518181704710B540F66A1342
:100D1000C1F3421301F01F040121A140012B07D0B0
:100D2000022B07D014303AB102680A43026010BDAA
:100D30000C30F8E71030F6E702688A43026010BD15
:100D4000002A03D0828A0A4382827047828A8A43B9
:100D500082827047028A22F00F020282028A0A43CC
:100D600002827047828922F40062828182890A436A
:100D700082817047002904D0818941F0020181817C
:100D80007047818921F0020181817047028A22F037
:100D900020020282028A0A4302827047002904D09C
:100DA000018A41F4804101827047018A21F4804127
:100DB00001827047C1F30801818070478088C0F3C9
:100DC00008007047818941F0010181817047028BE1
:100DD000D2B20283028B42EA012101837047028B67
:100DE00002F47F420283028B0A4302837047002988
:100DF00004D0818A41F0200181827047818A21F0EC
:100E0000200181827047002904D0818A41F01001BD
:100E100081827047818A21F0100181827047002908
:100E200004D0818A41F0080181827047818A21F0D3
:100E3000080181827047002904D0818941F4004172
:100E4000818170478189C1F30E018181704700293A
:100E500004D0818A41F4006181827047818A21F443
:100E6000006181827047828A22F004028282828A33
:100E70000A4382827047002904D0818A41F002012E
:100E800081827047818A21F0020181827047024687
:100E9000002012880A4200D0012070478A05C94309
:100EA0000180704770B5002440F66A12C1F3421306
:100EB00001F01F05012606FA05F2012B0CD0022BCA
:100EC0000DD0838A1340090A8E40008830400BB150
:100ED00000B10124204670BD83891340F3E7038AE3
:100EE0001340F0E740F66A120A0A01219140C94313
:100EF0000180704700380140004400400048004035
:100F0000004C00400050004010B50120FEF74FFF9C
:100F1000BDE810400020FEF74ABF20490860704736
:100F20001E49091F086070471C49843108607047DA
:100F30001B4A118821F46071014311807047184ADF
:100F4000118821F07F0101431180704708B5144AD0
:100F50002C3A104400900098016008BD08B5104973
:100F60002C39084400900098008808BD0B489C303C
:100F70000068C0B270470A480830018841F001019A
:100F8000018070470548A0300068C0B2704704482F
:100F90000830018841F002010180704704860D424B
:100FA0002C6C004010B501210C072046FEF7F4FE22
:100FB0002046BDE810400021FEF7EEBE2149086240
:100FC00070472049086170471F4A116821F0E0010D
:100FD0000143116070471B49A031086070471A4BEC
:100FE0001A6822F0030202431A601848026842F0AD
:100FF00004020260012905D020BF016821F004012C
:101000000160704730BFF8E70F48016841F0040104
:101010000160016841F0020101600C48016841F083
:101020000401016030BF704701460020064A526843
:101030000A4200D00120704703490A6842EA800052
:101040000860704700000E420070004010ED00E0A4
:101050000948804709480047FEE7FEE7FEE7FEE74C
:10106000FEE7FEE7FEE7FEE7FEE7FEE70448054988
:10107000054A064B70470000D583000831810008FF
:1010800020D8002020DE002020DA002020DA0020F6
:101090007FB5B24CA088ADF80C0048258DF80F50F4
:1010A00002268DF80E6003A92068F7F7B2FE208AA9
:1010B000ADF808008DF80B508DF80A6002A9E068C1
:1010C000F7F7A7FEA08BADF804008DF807508DF858
:1010D000066001A9A069F7F79CFE208DADF800001D
:1010E0008DF803508DF802606946606AF7F791FE4B
:1010F0007FBD70B5994D583DB5F85C10A86DF7F7F8
:10110000E3FE974C18B3207820F004002070B5F867
:101110006810686EF7F7D8FEF0B1207820F0020072
:101120002070B5F87410286FF7F7CEFEC8B120789C
:1011300020F001002070B5F88010E86FF7F7C4FECA
:10114000A0B1207820F008002070207870BD2078B1
:1011500040F004002070DAE7207840F002002070B0
:10116000DFE7207840F001002070E4E7207840F0CD
:1011700008002070E9E72DE9F047012007F088F921
:10118000FFF7B7FF044677484480754EDFF8D881F3
:10119000093E4FF0000770794FF0010534EA000076
:1011A00015D098F87F00032811D0F5706F480770AC
:1011B00098F8ED006E49C0EB00104FF6FF7202EA9E
:1011C0008000088018B101216A48F7F791FEF07895
:1011D000694B012876D1717931EA040072D098F810
:1011E0007A0002286ED0F77064480570644A642063
:1011F0001070B17163480770187801280FD07278A9
:101200004FF00D0C05204FF00E0962B3012951D0AB
:1012100002293DD0042960D0082976D169E03079CF
:10122000172801D0182803D108290AD0042908D08A
:1012300001290DD0022908D004290CD008290FD18A
:101240000CE01920B07237715FE01820B07207E02F
:101250001720B07204E01620B07201E01520B072C1
:10126000B07A307151E001294FD002294DD00429C4
:1012700002D0082949D105E086F80AC07570B5701A
:10128000307042E086F80A907570B57030703CE0BE
:10129000B278012A04D0022A05D0032A06D007E03A
:1012A0000A22B27204E01122B27201E01222B2727A
:1012B00030702AE0B278012A05D0022A06D0032A2B
:1012C00007D008E032E00922B27204E00F22B272C5
:1012D00001E01022B272307017E086F80AC0757013
:1012E000B278032A02D2521CB27000E0B57030709E
:1012F0000BE086F80A907570B278012A02D9521E66
:10130000B27001E00322B2703070042908D00829BD
:1013100006D0022904D0012902D098F8790028B912
:1013200019480770F571B5811848077074710C2C55
:1013300011D1187878B998F87F0001280BD00328CC
:1013400009D0307A411C31721E2802D91320B072A4
:101350001D70BDE8F0873772FBE70000F805030851
:10136000F700002036120020607F00206600002079
:101370003E000020000801406900002067000020B6
:101380006F000020700000206A0000207100002023
:1013900038B5A54C208FADF8000048208DF803002B
:1013A0006946606BF7F735FD218F606BF7F7A0FD9D
:1013B00038BD38B59C4C208FADF8000010208DF85A
:1013C000030003208DF802006946606BF7F721FDEA
:1013D000218F606BF7F78CFD38BD08B50820ADF89C
:1013E000000010208DF8030003208DF802006946EC
:1013F0008E48F7F70EFD08BD08B50820ADF80000CF
:1014000048208DF8030069468848F7F702FD08BDBB
:10141000854A002803D0918D906AF7F769BD918DB8
:10142000906AF7F767BD804A002803D0118F506B90
:10143000F7F75EBD118F506BF7F75CBD7A48018FEF
:10144000406BF7F741BD7848818D806AF7F73CBD66
:10145000F8B5754C0121606AFEF77DFCA08DADF8F2
:10146000000010258DF8035003268DF802606946B0
:10147000A06AF7F7CEFCA18DA06AF7F739FD01212C
:10148000206BFEF768FC208FADF800008DF803504C
:101490008DF802606946606BF7F7BBFC218F606BCB
:1014A000F7F726FDF8BD10B5FFF783FF0120FFF722
:1014B000BAFF0120FFF7ACFF042006F0E9FF00208F
:1014C000FFF7B1FF042006F0E3FFBDE81040002065
:1014D0009EE710B5FFF76DFF0020FFF799FF002092
:1014E000FFF7A1FF042006F0D3FF0120FFF790FFD4
:1014F0000120FFF798FFBDE81040042006F0C8BFA8
:1015000010B500240120FFF78EFFFFF741FF0120F7
:1015100006F0BEFF0120FFF77BFF012006F0B8FFB9
:1015200007E0641CA4B2FA2C03D9FFF7D2FF012014
:1015300010BDFFF783FF0028F3D1FFF769FF0020FC
:1015400010BD10B50020FFF763FFFFF732FF00204A
:10155000FFF769FF022006F09BFF0120FFF758FF0D
:10156000022006F095FFBDE81040002050E710B5BE
:101570000020FFF74DFFFFF71CFF0120FFF753FF8F
:10158000022006F085FF0120FFF742FF022006F04F
:101590007FFFBDE8104000203AE770B50546FFF731
:1015A00008FF0020FFF734FF0024E809FFF73BFFA6
:1015B0006806050E022006F06BFF0120FFF728FFEA
:1015C000022006F065FF0020FFF722FF022006F050
:1015D0005FFF641CE4B2082CE7D370BD70B506460B
:1015E0000024FFF7D5FE00250020FFF711FF0220A1
:1015F00006F04EFF0120FFF70BFF6006040EFFF719
:101600001DFF08B1641CE4B2012006F041FF6D1C0F
:10161000EDB2082DE8D31EB1FFF793FF204670BD51
:10162000FFF7A5FFFAE70000A00503080008014046
:1016300038B5704CE06B002815D054F83C0F0121F0
:10164000FEF789FB2089ADF8000010208DF803001B
:1016500003208DF8020069466068F7F7DAFB2189FC
:101660006068F7F745FC38BD624AD16B00290AD0A3
:1016700020B1B2F84410106CF7F73ABCB2F844103D
:10168000106CF7F737BC704710B5FFF7E1FEBDE807
:101690001040CDE710B50446FFF705FF200AA02152
:1016A00001EB4000C0B2FFF778FFFFF729FFE0B27F
:1016B000FFF773FFFFF724FFFFF7F5FEA120FFF709
:1016C0006CFFFFF71DFF0020FFF788FF0446FFF7C0
:1016D00000FF204610BD70B504460D460020FFF700
:1016E000C3FFFFF7E0FE200AA02101EB4000C0B2DB
:1016F000FFF753FFFFF704FFE0B2FFF74EFFFFF7DE
:10170000FFFE2846FFF749FFFFF7FAFEFFF7E1FE6D
:101710000120FFF7A9FFBDE87040052006F0D8BE04
:101720002DE9F04106460D461746002409E0E00089
:1017300025FA00F0C1B2301980B2FFF7CCFF641C6B
:10174000E4B2BC42F3D3BDE8F0812DE9F04102469A
:101750000E4600200024971908E00502381B401EA1
:1017600080B2FFF797FF2844641CE4B2B442F4D37C
:10177000E9E710B5FF20FFF78DFF55280AD0552166
:10178000FF20FFF7A8FFFF20FFF784FF552803D0B5
:10179000012010BD002010BD002010BD70B5044612
:1017A0000E46154608E02046641CA4B2FFF772FFFF
:1017B00006F8010B6D1EADB2002DF4D170BD70B5F1
:1017C00006460D46144606E029783046FFF783FFAB
:1017D000761CB6B26D1C641EA4B2F5D270BD59E77A
:1017E000054A1278012A03D0B72802D0B82800D0C1
:1017F00071E77047A0050308FD000020704730B571
:101800006423B0FBF3F4E4B2B0FBF3F503FB150083
:10181000132C01D96430C0B200EB90030724B3FB52
:10182000F4F504FB1533A44D1A440D4415F8015C7E
:101830002A4492B2800703D1032901D2521E92B2E8
:10184000B2FBF4F004FB102030BD810701D0002072
:1018500070476421B0FBF1F201FB120109B10120D4
:1018600070474FF4C871B0FBF1F201FB120008B1F0
:1018700000207047012070472DE9F047FEF7DBFAA2
:1018800006468E4FB6FBF7F38D488E4D0188994280
:1018900033D0038040F2B2744FF4B7784FF4B67986
:1018A0000FE02046FFF7D1FF38B1434502D3A3F53F
:1018B000B77304E0641CA4B205E0A3F26D13641CCA
:1018C000A4B24B45EDD8AC800024DFF8EC8108F1E0
:1018D0000C080CE0A888FFF7B8FF08B1012C2FD046
:1018E00018F80400984204D81B1A641CA4B21C2BDC
:1018F000F0D2641CAC715B1CEB71B6FBF7F007FB1C
:1019000010604FF46161B0FBF1F22A70B0FBF1F2AC
:1019100001FB12033C22B3FBF2F36B70B0FBF1F35B
:1019200001FB1300B0FBF2F102FB1100A870EA7991
:10193000A979A888FFF763FF28720020BDE8F08727
:101940001D2BD6D31D3BD0E770B500240420FFF734
:1019500005FB45F25005A8423FD001214FF0C05091
:10196000FEF704FA0120FFF729FBFFF7CDFA01206B
:10197000FEF77BF908E0641CE4B20A2006F0A8FD3B
:10198000C82C01D3012070BD4120FEF7F3F80028D8
:10199000F1D0FA2C01D3012070BD4FF48070FEF716
:1019A00079F90120FEF77BF9FEF780FAFEF78EFA4F
:1019B00001210846FEF726FAFEF778FAFEF72DFA1F
:1019C00047F6FF70FEF74DFAFEF770FAFEF72CFAB5
:1019D00029460420FFF7BAFA07E0FEF777FA01215B
:1019E0000846FEF70FFAFEF761FAFFF707FFFFF769
:1019F00043FF002070BD2DE9F05F0646DDF828A00A
:101A0000894690460024A6F2B270822802D30120B3
:101A1000BDE8F09F40F2B2752B4FDFF8B0B008E0A0
:101A20002846FFF712FF08B13C4400E05C446D1CFF
:101A3000ADB2B542F4D3A9F1010909F0FF070025C1
:101A4000DFF87490DFF874B009F10C090FE019F8B1
:101A5000050040F2A321484304EBC0143046FFF7D1
:101A6000F4FE10B1012D00D15C446D1CADB2BD423D
:101A7000EDD3A8F1010840F2A32008FB00F804EB25
:101A8000C810C3EB4311C1EB032100EB0110CAEBFB
:101A90000A1100EB81000B99441801214FF0C0504E
:101AA000FEF764F90120FFF789FA2046FEF7CCF92A
:101AB000FEF7FCF90020ABE7880503088051010020
:101AC000FE0000208C1100200085E2018033E1013E
:101AD00070B5FA4B0024C3F88041F94A0125127A07
:101AE000042A02D3F74A156001E0C3F888510022A6
:101AF000C3F88441060602D5C3F88C5101E0C3F84F
:101B00008C41C3F884514006000E521CD2B2082A00
:101B1000EED30020C3F884410A0602D5C3F88C51E5
:101B200001E0C3F88C41C3F884514906090E401CFA
:101B3000C0B20828EED3C3F8805170BDC0F30722AD
:101B4000C1B21046C4E730B5DC4A0023C2F8803188
:101B5000DB49097A042902D3DA490B6001E0C2F8B3
:101B6000883100210124C2F88431050602D5C2F86B
:101B70008C4101E0C2F88C31C2F884414006000E6D
:101B8000491CC9B20829EED3C2F8804130BD30B536
:101B9000CA4A0024C2F88041C9490123097A0429AC
:101BA00002D3C8490B6001E0C2F888310021C2F8B5
:101BB0008441050602D5C2F88C3101E0C2F88C419F
:101BC000C2F884314006000E491CC9B20829EED380
:101BD000C2F8803130BD2DE9F04381468846C2F31A
:101BE0000724D5B2C3F30726DFB22A20FFF7ABFFE5
:101BF0000020FFF7CCFF4846FFF7C9FF0020FFF7A2
:101C0000C6FF4046FFF7C3FF2B20FFF79CFF20468F
:101C1000FFF7BDFF2846FFF7BAFF3046FFF7B7FFD3
:101C20003846FFF7B4FFBDE8F0432C208BE72DE9E1
:101C3000F0410746002240F23F13EF211046FFF724
:101C4000CAFF00254FF4A07600243846FFF776FF40
:101C5000641CF02CF9D36D1CB542F5D3BDE8F081BE
:101C600000B52820FFF76FFF10205DF804EB6AE74E
:101C700010B51120FFF767FF782006F029FCBDE8BA
:101C8000104029205FE770B58F4C012525600520A5
:101C900006F01EFC0020E0630A2006F019FCE56354
:101CA000782006F015FC1120FFF74DFF782006F094
:101CB0000FFCCF20FFF747FF0020FFF768FFC3208E
:101CC000FFF765FF3020FFF762FFED20FFF73BFFD6
:101CD0006420FFF75CFF0320FFF759FF1220FFF796
:101CE00056FF8120FFF753FFE820FFF72CFF8520E8
:101CF000FFF74DFF1020FFF74AFF7920FFF747FF5E
:101D0000CB20FFF720FF3920FFF741FF2C20FFF702
:101D10003EFF0020FFF73BFF3420FFF738FF022093
:101D2000FFF735FFF720FFF70EFF2020FFF72FFF0B
:101D3000EA20FFF708FF0020FFF729FF0020FFF748
:101D400026FFC020FFF7FFFE2220FFF720FFC12063
:101D5000FFF7F9FE1120FFF71AFFC520FFF7F3FE8A
:101D60003D20FFF714FF2020FFF711FFC720FFF7EA
:101D7000EAFEAA20FFF70BFF3620FFF7E4FEC8209B
:101D8000FFF705FF3A20FFF7DEFE5520FFF7FFFEC5
:101D9000B120FFF7D8FE0020FFF7F9FE1320FFF770
:101DA000F6FEB620FFF7CFFE0A20FFF7F0FEA220D6
:101DB000FFF7EDFEF620FFF7C6FE0120FFF7E7FE76
:101DC0003020FFF7E4FEF220FFF7BDFE0020FFF712
:101DD000DEFE2620FFF7B7FE0120FFF7D8FEE02049
:101DE000FFF7B1FE0F20FFF7D2FE3F20FFF7CFFE37
:101DF0002F20FFF7CCFE0C20FFF7C9FE1020FFF7C5
:101E0000C6FE0A20FFF7C3FE5320FFF7C0FED52011
:101E1000FFF7BDFE4020FFF7BAFE0A20FFF7B7FE2E
:101E20001320FFF7B4FE0320FFF7B1FE0820FFF7F1
:101E3000AEFE0320FFF7ABFE0020FFF7A8FEE12077
:101E4000FFF781FE0020FFF7A2FE0020FFF79FFEB4
:101E50001020FFF79CFE0320FFF799FE0F20FFF7ED
:101E600096FE0520FFF793FE2C20FFF790FEA220A0
:101E7000FFF78DFE3F20FFF78AFE0520FFF787FE64
:101E80000E20FFF784FE0C20FFF781FE3720FFF7BE
:101E90007EFE3C20FFF77BFE0F20FFF778FE11202F
:101EA000FFF751FE782006F013FB2920FFF74BFEC9
:101EB000BDE87040322006F00BBB000000802242DB
:101EC000607F0020988121428081224210B5FB482A
:101ED000002101604160C160C163A0F5C070F84A93
:101EE000127A042A02D3F748016001E0C0F8881191
:101EF000FFF7C9FEBDE8104047F6196097E62DE9E7
:101F0000F05FDDE90A7800281BD0EF4D1826242465
:101F1000203B03EBC30000EB400005EB8005881974
:101F2000401E00F0FF0C1319C8B25B1E6146FFF79C
:101F300052FE7443E01704EB5070C0F3CF09002643
:101F40002CE0E24D302660242D2B07D0202B08D02A
:101F5000303B03EBC30005EB8015E0E705F5B45516
:101F6000DDE705F5C655DAE700244FEA182A4FEAFF
:101F7000172B2878E040C00704D0F9B25846FFF785
:101F8000A7FD04E008F0FF015046FFF7A1FD641C27
:101F9000A4B2082CEDD36D1C761CB6B24E45E3D32B
:101FA000BDE8F09F2DE9FC470746DDE90A890C46AC
:101FB00016461D4609E0B2B2A1B23846CDE9008905
:101FC000FFF79DFF37B117346D1C2B78002BF2D132
:101FD000BDE8FC871F34F7E770B51646049A01FB8D
:101FE00000F4A5B254181844401EC1B2641ED8B201
:101FF0002346FFF7F0FD002407E036F81400C1B2D5
:10200000000AFFF765FD641CA4B2AC42F5D370BDB5
:102010002DE9F041089E069A01FB00F4A5B2541880
:102020001844401EC1B2641ED8B22346FFF7D3FD48
:102030000024370A05E0F1B23846FFF749FD641C79
:10204000A4B2AC42F7D309E62DE9FF5FA04F79783F
:1020500001297AD19A4991F86E200AB1462200E00E
:10206000432291F8C5B00A236426DFF868E22025F0
:10207000002441424FF0300A4FF02D0C4FF02E0853
:102080004FF47A79BBF10A0F26D0002870DB48455F
:102090006FDB90FBF9F130318DF8081090FBF9F10E
:1020A00009FB110191FBF6F130318DF8091090FB1D
:1020B000F6F106FB110191FBF3F130318DF80A10B6
:1020C0008DF80B8090FBF3F103FB110030308DF89D
:1020D0000C008DF80D4074E1002858DB48451BDBEF
:1020E00090FBF9F130318DF8081090FBF9F109FB04
:1020F000110191FBF6F130318DF8091090FBF6F1EA
:1021000006FB110090FBF3F030308DF80A008DF8DB
:102110000B208DF80C4054E1642817DB90FBF6F19E
:1021200030318DF8081090FBF6F106FB110090FBA2
:10213000F3F030308DF809008DF80A208DF80B503F
:102140008DF80C508DF80D403BE15EE10A2811DB63
:1021500090FBF3F030308DF808008DF809208DF8F1
:102160000A508DF80B508DF80C508DF80D4028E179
:10217000C4E070E08DF808A08DF809208DF80A50B1
:102180008DF80B508DF80C508DF80D4019E170450D
:102190001BDC8DF808C091FBF9F030308DF8090098
:1021A00091FBF9F009FB101090FBF6F030308DF840
:1021B0000A0091FBF6F006FB101090FBF3F03030B4
:1021C0008DF80B008DF80C40FBE010F1640F14DC6F
:1021D0008DF808C091FBF6F030308DF8090091FBC6
:1021E000F6F006FB101090FBF3F030308DF80A008B
:1021F0008DF80B208DF80C40E3E010F10A0F16DC8F
:102200008DF808C091FBF3F030308DF809008DF89F
:102210000A8091FBF3F003FB101030308DF80B00B7
:102220008DF80C208DF80D408DF80E50C9E08DF81A
:1022300008C08DF809A08DF80A8091FBF3F003FB2C
:10224000101030308DF80B008DF80C208DF80D40FB
:102250008DF80E50B5E064281BDB90FBF6F13031B1
:102260008DF8081090FBF6F106FB110191FBF3F1DC
:1022700030318DF809108DF80A8090FBF3F103FBE3
:10228000110030308DF80B008DF80C208DF80D40CA
:1022900097E00A2820DB90FBF3F130318DF808102D
:1022A0008DF8098090FBF3F103FB110030308DF8BD
:1022B0000A008DF80C208DF80D4082E080812242CA
:1022C000607F00209881214270C70308340703080B
:1022D0009611002018FCFFFF8DF808A08DF80980EA
:1022E00090FBF3F103FB110030308DF80A008DF8FC
:1022F0000B208DF80C408DF80D5062E070451BDC12
:102300008DF808C091FBF9F030308DF8090091FB91
:10231000F9F009FB101090FBF6F030308DF80A0050
:1023200091FBF6F006FB101090FBF3F030308DF8C7
:102330000B008DF80C4044E010F1640F14DC8DF8B4
:1023400008C091FBF6F030308DF8090091FBF6F0F3
:1023500006FB101090FBF3F030308DF80A008DF87A
:102360000B208DF80C402CE010F10A0F16DC8DF8D4
:1023700008C091FBF3F030308DF809008DF80A8029
:1023800091FBF3F003FB101030308DF80B008DF84B
:102390000C208DF80D408DF80E5012E08DF808C01D
:1023A0008DF809A08DF80A8091FBF3F003FB101063
:1023B00030308DF80B008DF80C208DF80D408DF825
:1023C0000E50FB4E307880B1FA48007868B18DF835
:1023D00008508DF809508DF80A508DF80B508DF883
:1023E0000C508DF80D408DF80E5047F617604FF6E3
:1023F000FF71CDE9001002AB6C226A210120FFF7CA
:10240000D1FD3078002800D17C70BDE8FF9F70B509
:1024100086B0E94DA978012941D10021E74B20245C
:1024200003AE01EBC0021A4492F8812352B17254F8
:10243000491CC9B20529F4D393F86F00002601287E
:1024400002D010E07454F3E7DD48007858B903F285
:1024500089334F2018706E2058709E70DC701C718C
:102460005C719C71DC71D74C207830B1D148007818
:1024700018B1D5A103A81AF09BF98DF8116047F6A1
:1024800017604FF6FF71CDE9001003AB97226A2168
:102490000120FFF787FD2078002800D1AE7006B03C
:1024A00070BD7FB5C44DE878002830D0C34890F89F
:1024B000A903022803D0012806D050B10DE0C4A121
:1024C00002A81AF075F908E0C3A102A81AF070F981
:1024D00003E0C3A102A81AF06BF9C34C207830B115
:1024E000B448007818B1C1A102A81AF061F947F602
:1024F00017604FF6FF71CDE9001002ABC2226A21CE
:102500000120FFF74FFD2078002800D1E8707FBD43
:10251000FEB5B84F387800284BD000203870FDF752
:102520009AFAB54947F619644FF6FF7509784FF4E2
:102530008976C1B3B8B33878012847D0AF4ACDE91E
:102540000065B6232D2128200294FFF745FDAC48F5
:102550000178427880781144C14225D1A948007899
:1025600098B3012846D002284ED0032856D004281C
:1025700018D1FDF770FA01285AD0042858D0022843
:1025800060D005285ED0032866D0062864D00028D5
:1025900008D19D4ACDE90065DE232D210F2002944C
:1025A000FFF71AFDFEBD06E0984A907901285DD03C
:1025B0006CE00120B2E7964ACDE90065B6232D21F3
:1025C00028200294FFF708FDC1E709E0904ACDE911
:1025D0000065B6232D2128200294FFF7FDFCB6E705
:1025E000894ACDE90065DE232D210F200294FFF7F3
:1025F000F3FCD7E7874ACDE90065DE232D210F20C4
:102600000294FFF7E9FCCDE7834ACDE90065DE23BC
:102610002D210F200294FFF7DFFCC3E77F4ACDE9AD
:102620000065DE232D210F200294FFF7D5FCB9E7CA
:10263000784ACDE90065DE232D210F200294FFF7B3
:10264000CBFCAFE7744ACDE90065DE232D210F20D6
:102650000294FFF7C1FCA5E7704ACDE90065DE23CF
:102660002D210F200294FFF7B7FC9BE7D1790129B8
:102670000CD0117A012909D0CDE90065DE23654A25
:102680002D210F200294FFF7A7FC8BE7D1790129B8
:102690000ED101280CD0137A012B09D0CDE90065A9
:1026A000DE235D4A2D210F200294FFF795FC79E788
:1026B000127A012A0DD101280BD0012909D0CDE9C8
:1026C0000065DE23554A2D210F200294FFF784FC7C
:1026D00068E7CDE90065DE234B4A2D210F200294E7
:1026E000FFF77AFC5EE72DE9FE4FFDF7CAF90746D2
:1026F0004B48DFF8C4800178B94203D0012188F843
:1027000005100770DFF8B4904FF6FF764FF0000A1F
:1027100099F8670299F8681299F86A22084499F8BA
:10272000691247F619641144C8424FF489753ED0C6
:10273000DFF8D8B09BF8000001280DD19BF80110FC
:10274000012909D0CDE900560223364A2D21372030
:102750000294FFF741FC18E09BF8011001290BD10E
:10276000012809D0CDE9005602232F4A2D21372018
:102770000294FFF731FC08E0CDE900540223002267
:102780002D2137200294FFF743FC9BF8020001281B
:102790004ED19BF8031001294AD0CDE900563E23C3
:1027A000224A2D2137200294FFF716FC23E159E03D
:1027B000300000203300002096110020607F0020B0
:1027C0002F00002031000020202020202020200089
:1027D0004865617420000000436F6F6C20000000AA
:1027E0004175746F2000000032000020202020205E
:1027F00020000000000100202C000020086C0308CD
:10280000CD8100203B000020E0480308640900203F
:10281000F85D0308264E03086C530308B2580308FA
:102820005E000020187A03086E8D03083422030826
:102830009BF8031001290BD1012809D0CDE90056DE
:102840003E23FD4A2D2137200294FFF7C5FBD2E03D
:10285000CDE900543E2300222D2137200294FFF7BA
:10286000D7FBC8E099F8B912F448012919D098F8B3
:10287000041000299AD00068002877D0CDE90054D0
:102880000223EF4A2D2137200294FFF7A5FBCDE963
:1028900000563E23EB4A2D2137200294FFF79CFB84
:1028A000A7E00068C0B198F80400002813D0CDE973
:1028B0000054022300222D2137200294FFF7A8FBA9
:1028C000CDE900563E23DF4A2D2137200294FFF741
:1028D00083FB88F804A08EE0DFF86CB39BF800005F
:1028E000092830D004DC012807D0042864D117E07F
:1028F0000A283CD00B285FD14CE0CDE900560223DA
:10290000CF4A2D2137200294FFF766FBCDE9005610
:102910003E23CC4A2D2137200294FFF75DFB4BE08C
:10292000CDE900560223C64A2D2137200294FFF735
:1029300053FBCDE900563E23BF4A2D213720029498
:10294000FFF74AFB38E0CDE900560223BF4A2D21AC
:1029500037200294FFF740FBCDE900563E23B94AE9
:102960002D2137200294FFF737FB25E029E0CDE940
:1029700000560223B54A2D2137200294FFF72CFB85
:10298000CDE900563E23AC4A2D2137200294FFF7B3
:1029900023FB11E0CDE90054022300222D21372032
:1029A0000294FFF735FBCDE900543E2300222D2190
:1029B00037200294FFF72CFBA5499BF80000087014
:1029C00019E0A448007818B399F87600B0B3CDE9BF
:1029D000005402239D4A2D2137200294FFF7FCFA70
:1029E000CDE900563E23974A2D2137200294FFF768
:1029F000F3FA88F804A099F86B0299F86C12C842AF
:102A000068D0DFF8549299F8040001282BD039E0FF
:102A100099F8760098B1CDE900540223884A2D2117
:102A200037200294FFF7D8FACDE900563E23824AB8
:102A30002D2137200294FFF7CFFADAE709E0CDE93C
:102A400000540223814A2D2137200294FFF7C4FA53
:102A5000EAE7CDE900540223794A2D213720029478
:102A6000FFF7BAFABCE799F8051001290AD0CDE9B9
:102A700000567A23794A2D2137200294FFF7ACFAC9
:102A8000BDE8FE8F99F8051001290BD1012809D066
:102A9000CDE900567A23724A2D2137200294FFF7A0
:102AA0009BFAEDE7012801D1012901D048B941B9CC
:102AB000CDE900547A2300222D2137200294FFF71C
:102AC000A7FA99F80400642808D099F8050064284A
:102AD00004D0D5E798F805000128D1D127B1012FFE
:102AE0000CD0022F1DD113E0CDE900547A2300222F
:102AF0002D2137200294FFF78BFA12E0CDE9005622
:102B00007A23574A2D2137200294FFF765FA08E00F
:102B1000CDE900567A23514A2D2137200294FFF740
:102B20005BFA88F805A0ABE71CB547F619640128E5
:102B300008D000944BA3C222002101200194FFF78A
:102B400031FA1CBD009447A36C220021012001949E
:102B5000FFF728FA009443A3972200210120019453
:102B6000FFF720FA1CBD3EB547F619654FF6FF7416
:102B700067208DE8310000231A462D21EF20FFF752
:102B800047FA92208DE8310000231A462D21EF20CC
:102B9000FFF73EFABD208DE8310000231A462D21B3
:102BA000EF20FFF735FA3EBD2DE9FF4764250A23E4
:102BB00020244FF0000C4FF47A77202A29D02E26BB
:102BC0004FF0300900297DDBB9427CDB91FBF7F047
:102BD00030308DF8080091FBF7F007FB101090FBE8
:102BE000F5F030308DF8090091FBF5F005FB101081
:102BF00090FBF3F030308DF80A008DF80B6091FBFC
:102C0000F3F003FB101030308DF80C008DF80D2020
:102C1000D3E0B9423FDB91FBF7F030308DF808008C
:102C200091FBF7F007FB101090FBF5F030308DF8BA
:102C3000090091FBF5F01FE08A3503084C000020E5
:102C4000187A030834220308370000206E8D030829
:102C50002E0000203B000020640900201AB4030865
:102C6000C4A0030820202020202020202020202075
:102C7000202020200000000005FB101090FBF3F046
:102C800030308DF80A0091FBF3F003FB1010303068
:102C90008DF80B0046E064291EDB91FBF7F007FB83
:102CA000101090FBF5F030308DF8080091FBF5F036
:102CB00005FB101090FBF3F030308DF8090091FB0C
:102CC000F3F001E07CE034E003FB101030308DF8CD
:102CD0000A008DF80B4025E00A2914DB8DF8084026
:102CE00091FBF5F005FB101090FBF3F030308DF800
:102CF000090091FBF3F003FB101030308DF80A004F
:102D00008DF80B400EE000290CDB8DF8084091FB9C
:102D1000F3F003FB101030308DF809008DF80A40F5
:102D20008DF80B408DF80C408DF80D408DF80EC0DD
:102D3000A7E064291BDB91FBF5F030308DF808002B
:102D400091FBF5F005FB101090FBF3F030308DF89F
:102D500009008DF80A6091FBF3F003FB101030308E
:102D60008DF80B008DF80C208DF80D4025E00A2918
:102D700012DB91FBF3F030308DF808008DF809601C
:102D800091FBF3F003FB101030308DF80A008DF842
:102D90000C208DF80D4010E08DF808908DF809603A
:102DA00091FBF3F003FB101030308DF80A008DF822
:102DB0000B208DF80C408DF80D408DF80EC060E0B2
:102DC00048424FF02D0811F57A7F24DC8DF80880F9
:102DD00090FBF7F130318DF8091090FBF7F107FB0C
:102DE000110191FBF5F130318DF80A1090FBF5F1EE
:102DF00005FB110191FBF3F130318DF80B108DF8CB
:102E00000C6090FBF3F103FB110030308DF80D00E6
:102E10008DF80E2033E011F1640F1DDC8DF8088071
:102E200090FBF5F130318DF8091090FBF5F105FBC1
:102E3000110191FBF3F130318DF80A108DF80B6020
:102E400090FBF3F103FB110030308DF80C008DF88E
:102E50000D208DF80E4012E08DF808808DF8099055
:102E60008DF80A6090FBF3F103FB110030308DF810
:102E70000B008DF80C208DF80D408DF80E408DF86C
:102E80000FC047F619604FF6FF71CDE9001002AB95
:102E9000C22200210120FFF785F8BDE8FF877CB53D
:102EA0000E4647F619654FF6FF7403466C22002163
:102EB0000120CDE90045FFF775F833469722002140
:102EC0000120CDE90045FFF76DF87CBD2DE9FE4FEF
:102ED00005460C4647F619694FF6FF768DE8500215
:102EE00008212B46FC4A0846FFF776F8A01C47F657
:102EF000176A80B28DE84104AB1D002201217120C8
:102F0000FFF786F804F10800CDE9016A87B2AB1C2F
:102F100000221C2102200097FFF77AF804F122001A
:102F2000CDE901691FFA80F8EB4A08212B4680326F
:102F30000846CDF80080FFF74FF804F1270080B273
:102F40008DE84104AB1D002201217120FFF760F8DC
:102F5000CDE9016905F17303CDF800800821984699
:102F6000DE4A0846FFF738F8DC4A8DE850020821AF
:102F7000434680320846FFF72FF8CDE9016A05F194
:102F8000780300221C2101200097FFF741F804F18B
:102F900028004BF69C6780B28DE8C1006B1D0022B3
:102FA00002217320FFF734F88DE8D0006B1D00225A
:102FB00002217320FFF72CF8A41DA4B28DE8D000E5
:102FC0002B46002220210220FFF722F88DE8D000B6
:102FD00005F17903002220210220FFF719F84FE5BF
:102FE000F0B5BF4D2E2764230A242026C2EB02121F
:102FF0002A44002816DA2D215172404290FBF3F149
:103000003031917290FBF3F103FB110191FBF4F16C
:103010003031D172177390FBF4F104FB11003030A2
:10302000507358E0DFF8BCC24FF47A7561444FF03A
:10303000250CA84237DB91F8E51002291BD090FB44
:10304000F5F13031517290FBF5F105FB110191FB67
:10305000F3F13031917290FBF3F103FB110191FB1D
:10306000F4F13031D172177390FBF4F104FB1100CD
:10307000303050732FE090FBF5F13031517290FBFE
:10308000F5F105FB110191FBF3F13031917290FBE9
:10309000F3F103FB110090FBF4F03030D07282F8B2
:1030A0000CC0567317E090FBF3F53035557290FB6A
:1030B000F3F503FB150393FBF4F330339372D772EC
:1030C00090FBF4F304FB13003030107391F8E5002B
:1030D000022802D056739673F0BD82F80DC0FAE74D
:1030E0002DE9F05F7F4890F8B812092902D909212B
:1030F00080F8B81290F8B812002973D000243A274B
:10310000DFF8E4814FF00A094FF0640A2025744E7D
:1031100012E2081990F8BA02C01E0E281CD2DFE88D
:1031200000F0071E354C647B92A9C0FAE7E6E5DAA9
:103130000020C4EB041232440B1893F8A93163B198
:103140001354401CC0B20828F6D31772B8F9000017
:1031500022460021FFF744FFECE11554F1E700207F
:10316000C4EB041232440B1893F8B13163B1135419
:10317000401CC0B20828F6D31772B8F902002246E4
:103180000021FFF72DFFD5E11554F1E70020C4EB36
:10319000041232440B1893F8B93163B11354401C34
:1031A000C0B20828F6D31772B8F9040022460021ED
:1031B000FFF716FFBEE11554F1E70020C4EB04123F
:1031C00032440B1893F8C1316BB11354401CC0B298
:1031D0000828F6D31772B8F9060022460021FFF737
:1031E000FFFEA7E1AEE11554F0E70020C4EB0412A6
:1031F00032440B1893F8C93163B11354401CC0B268
:103200000828F6D31772B8F9080022460021FFF704
:10321000E7FE8FE11554F1E70020C4EB04123244BD
:103220000B1893F8D13163B11354401CC0B2082875
:10323000F6D31772B8F90A0022460021FFF7D0FE34
:1032400078E11554F1E70020C4EB041232440B1866
:1032500093F8D93163B11354401CC0B20828F6D397
:103260001772B8F90C0022460021FFF7B9FE61E1A0
:103270001554F1E70020C4EB041232440B1893F804
:10328000E13163B11354401CC0B20828F6D3177261
:10329000B8F90E0022460021FFF7A2FE4AE11554BC
:1032A000F1E7FCF7EEFBC4EB04105321315400EBC3
:1032B000060B74218BF8011061208BF80200672047
:1032C0008BF8030065208BF804008BF80570FCF781
:1032D000C2FB00210EE0F4E084EF030884F0030851
:1032E00008010020607F002018120020B3E074E085
:1032F00022E010E0FB4AC0EBC00010440BEB0103DE
:10330000425C9A71491CC9B20729F7D38BF80D505A
:103310008BF80E500EE10020C4EB041232440B185F
:1033200093F8913133B11354401CC0B20E28F6D338
:103330009573FFE01554F7E7EB498879EB4B401E96
:1033400000EB800003EB40004278C4EB04103254E1
:103350008A793044521E02EB820203EB42029278D9
:1033600042708A79521E02EB820203EB4202D2784B
:103370008270C570CA79B2FBF9F230320271CA7933
:10338000B2FBF9F309FB1322303242712C22827115
:103390008B884FF47A72B3FBF2F33033C3718B88AE
:1033A000B3FBF2FC02FB1C32B2FBFAF230320272C7
:1033B0008A88B2FBFAF30AFB1322B2FBF9F230322D
:1033C00042728988B1FBF9F209FB12113031817226
:1033D000C572057345738573ACE0C4EB04105421CA
:1033E00031543044692141706D2181706521C17073
:1033F0000571BF49097803291FD0BB4A1178B1FB79
:10340000F9F1303141711178B1FBF9F309FB131176
:1034100030318171C7715178B1FBF9F130310172EE
:103420005178B1FBF9F209FB12113031417285720A
:10343000C5720573457385737CE045214171722126
:103440008171C1716F22027241728572C5720573FA
:10345000457385736EE0C4EB04104321315430444E
:103460004F21417032218170C770A2494FF47A72A6
:103470000988914204D3B1FBF2F33033037100E0C9
:103480000571B1FBF2F302FB1312B2FBFAF2303218
:103490004271B1FBFAF20AFB1212B2FBF9F23032BE
:1034A0008271B1FBF9F209FB12113031C171702147
:1034B000017241726D218172C57205734573857306
:1034C00038E0C4EB04104821315430447521417078
:1034D0006D2181706921C17080F804A0417174214F
:1034E00081717921C17107728349B1F90010B1F579
:1034F0007A7F08DB3121417230218172C17225212E
:103500000173457315E091FBFAF23032427291FB80
:10351000FAF20AFB121292FBF9F2303282722E2278
:10352000C27291FBF9F209FB1211303101732521AE
:1035300041738573641CE4B2704991F8B802A042EB
:103540003FF6E7ADBDE8F09F2DE9FC5FFFF7C8FD52
:10355000DFF8A8816A4C6B4D98F8B812002647F640
:1035600017674FF6FF7B99B90020491EC1EB011187
:1035700029440A5C2254401CC0B20A28F9D3A6721E
:10358000CDE900B75E4BED2200210120FEF70AFDD8
:1035900098F8B802002842D0DFF86891401EA9F1DF
:1035A0000809C0EB00104219D9F80410501C8842D9
:1035B0001CD80020531A03F10F0C05E011F800800D
:1035C00004F80080401CC0B28445F7DC0020A1EB69
:1035D000020808E003EB000AA24415F800C08AF8CC
:1035E0000FC0401CC0B28045F4DC06E000200B5C3C
:1035F0002354401CC0B20A28F9D30E328A4202D1A9
:10360000C9F8045002E0491CC9F80410A672CDE9BB
:1036100000B73B4BED221E210120FEF7C3FCBDE8A5
:10362000FC9FF0B587B0044647F617664FF478471D
:10363000CDE90176ED20002300901A461E21EF20EF
:10364000FEF7E6FC0021274A2E4D8C3204A802F139
:103650001E03083D14B1012C08D00EE095F801C0FE
:103660008C4412F80CC000F801C006E095F801C0C7
:103670008C4413F80CC000F801C0491CC9B20A29D7
:10368000E8D300248DF81A40CDE9007604ABED2292
:103690001E210120FEF786FC6878192803D2401C01
:1036A000687007B0F0BD6C70FBE70EB555224FF6A1
:1036B000FF71002809D0CDE90021029108218B2358
:1036C00000220846FEF7A4FC0EBDCDE9002147F616
:1036D0001960029008218B2300220846FEF798FC0F
:1036E0000EBD00006C0603088C110020E6FB0208EA
:1036F0000F030020580200205C020020607F0020A1
:103700009F110020080100202DE9F04F87B00D46E1
:103710004FF0270B052104915721069105210391B4
:1037200097210591052102914FF47A7A47F619669F
:103730004FF6FF7700287AD14FF00A094FF064085E
:10374000002D76DB2C46AFF67473CDE9007620228F
:1037500006210120FEF726FC554534DB94FBF9F0E9
:1037600004B2642C0BDB94FBF8F03030CDE900762A
:10377000C3B259460020049AFEF7C1FB07E0CDE929
:103780000076202359460020049AFEF7B8FB94FBEC
:10379000F8F008FB104090FBF9F0CDE900763030EE
:1037A000C3B20020039A0699FEF7A9FB94FBF9F037
:1037B00009FB1040CDE900763030C3B20020029AF8
:1037C0000599FEF79CFB554531DA642D0BDB94FB24
:1037D000F8F03030CDE90076C3B259460020049AA3
:1037E000FEF78DFB07E0CDE9007620235946002047
:1037F000049AFEF784FB94FBF8F008FB104090FB62
:10380000F9F0CDE900763030C3B20020039A069972
:10381000FEF775FB94FBF9F009FB1040CDE900764B
:103820003030C3B20020029A0599FEF768FB68E0C9
:10383000FFE7684204B2642C2FDB94FBF8F03030D1
:10384000CDE90076C3B259460020049AFEF757FB33
:1038500094FBF8F008FB104090FBF9F0CDE90076FE
:103860003030C3B20020039A0699FEF748FB94FB60
:10387000F9F009FB1040CDE900763030C3B20020EA
:10388000029A0599FEF73BFBCDE9007630A3202292
:1038900006210120FEF786FB33E0CDE900762023E8
:1038A00059460020049AFEF72AFB94FBF8F008FB27
:1038B000104090FBF9F0CDE900763030C3B2002023
:1038C000039A0699FEF71BFB94FBF9F009FB1040E5
:1038D000CDE900763030C3B20020029A0599FEF798
:1038E0000EFBCDE900761BA3202206210120FEF766
:1038F00059FBCDE9007616A3202228210120FEF7EE
:1039000051FB554503DD0020FFF7CFFE02E001200B
:10391000FFF7CBFE104C207801280DD10F4890F80E
:103920006E0060B1CDE900760DA33822D6210120CA
:10393000FEF738FB0020207007B0BDE8F08FCDE91E
:10394000007608A33822D6210120FEF72BFBF1E7F1
:103950002D0000002000000096110020607F002054
:10396000460000004300000010B5254C0121204610
:10397000FDF7E2F8012803D122490A68521C0A60C7
:103980002149088841F28832904203D20A88521CA9
:103990000A8001E0002008802046BDE81040012197
:1039A000FDF7D1B87FB504460D4601211020FCF784
:1039B000DDF9ADF80840ADF804500020ADF80A007C
:1039C000ADF806000E4C01A92046FCF7A1FB3621FC
:1039D0008DF8001001218DF8011003228DF80220CE
:1039E0008DF803106846F4F79CFE0122114620462C
:1039F000FCF779FE01212046FCF75BFE7FBD00004D
:103A0000001000403802002096060020FE49097A86
:103A100005290BD2FD4A20B1883291881068F5F74C
:103A200067BA883291881068F5F764BAF84A18B115
:103A300002211046F5F75CBA02211046F5F75ABA92
:103A4000F149097A05290BD2F04A20B194329188C4
:103A50001068F5F74DBA943291881068F5F74ABAB4
:103A6000EB4A18B101211046F5F742BA0121104680
:103A7000F5F740BAE449097A05290BD2E34A20B1A7
:103A8000A03291881068F5F733BAA0329188106897
:103A9000F5F730BADE4A18B110211046F5F728BA0A
:103AA00010211046F5F726BAD749097A05290BD215
:103AB000D64A20B1AC3291881068F5F719BAAC3209
:103AC00091881068F5F716BAD14A18B10821104646
:103AD000F5F70EBA08211046F5F70CBACA49097A6B
:103AE00005290BD2C94A20B1B83291881068F5F780
:103AF000FFB9B83291881068F5F7FCB9C44A18B11B
:103B000004211046F5F7F4B904211046F5F7F2B98F
:103B1000BD49097A05290BD2BC4A20B1C43291882B
:103B20001068F5F7E5B9C43291881068F5F7E2B985
:103B3000B74A18B120211046F5F7DAB9202110460E
:103B4000F5F7D8B92DE9FC41F220ADF804000025C5
:103B50008DF8075002248DF80640AE4E01A930467C
:103B6000F5F757F94FF00308ADF804808DF80750CA
:103B70008DF80640A84F01A93846F5F74AF9ADF887
:103B800004808DF807508DF80640DFF8908201A977
:103B90004046F5F73EF99C481025007A052816D2D4
:103BA0001C20ADF804008DF807508DF8064001A9DF
:103BB0004046F5F72EF9E020ADF804008DF80750E7
:103BC0008DF8064001A93046F5F723F915E03F20AE
:103BD000ADF804008DF807508DF8064001A98C4817
:103BE000F5F717F90C20ADF804008DF807508DF8A3
:103BF000064001A94046F5F70CF94FF40076ADF800
:103C000000608DF803508DF8024069463846F5F79C
:103C100000F901213046FCF79EF8BDE8FC8110B5A3
:103C200086B04FF40040FCF719F801214802FCF778
:103C300092F8002001908DF808008DF809004FF4EB
:103C400060210391049001208DF81400744C01A9A7
:103C50002046F4F7E9FD01212046F4F70DFE204649
:103C6000F4F72DFE2046F4F72FFE0128FAD0204667
:103C7000F4F731FE2046F4F733FE0128FAD006B0FF
:103C800010BD2DE9F0470546042B06D0062B04D0C5
:103C9000842B05D0862B03D004E04FF4FA7001E0AA
:103CA0004FF47A70DFF860C105F114036344DC7EE1
:103CB0001B7F04EB032340F2FF345A4FA14203DB86
:103CC000BB6418B2BDE8F08701EB81014E0096FBA2
:103CD000F0F10CB2CAB1611C05EB41016144CA7E2E
:103CE000097F02EB012305EB44016144CA7E097F91
:103CF00002EB01255D1B00FB14636B4393FBF0F0AB
:103D000000EB01201044B86433E005EB440161444A
:103D100011F8312F497802EB0122611C05EB4101BA
:103D2000614491F8315091F8328005EB0821A2EB03
:103D300001091BF0FDFC824648461BF0E1FC814670
:103D400030461BF0DDFC0646601C1BF0D9FC5146DA
:103D50001BF036FD31461BF009FE49461BF030FDD5
:103D600051461BF09BFB1BF08FFC00EB0820284406
:103D7000B864B7F8480000B2A4E770B5224C294BEC
:103D80000A281FD00A220B282BD0274D231835F9DB
:103D9000106093F8F73006FB031101EB8101490035
:103DA0005B1C91FBF3F191FBF2F302FB1313052B68
:103DB00000DB0A3191FBF2F325F8103091FBF2F0B1
:103DC00000B270BD187A052800D2598394F86000BB
:103DD000B3F91A2002FB0011401C91FBF0F058834C
:103DE000EEE794F829035C8D04FB001101EB8101DF
:103DF0004900401C91FBF0F090FBF2F102FB110135
:103E0000052900DB0A3011E0607F0020A0050308CF
:103E10000018014000080140000C01400010014062
:103E2000002401403C020020F011002090FBF2F140
:103E3000598590FBF2F0C3E710B512224FF4E1640C
:103E4000132907D0142932D0FE4B997C814251DDD1
:103E5000204610BDFC4B997C814201DD204610BDFF
:103E6000521E52B29C5C214481421DDD081A64211D
:103E70004843995C90FBF1F0042A09DB121F02EB26
:103E8000C20101EB021100EB8100C0F30E0009E05A
:103E900002EBC20101EB021100EB8100C0F5C8701A
:103EA00040F4004000B210BD002AD9D148E00921F9
:103EB000E64B5A8A824202DD4FF4AF7010BD491EB4
:103EC00049B233F811402244824210DD101AC0EB8F
:103ED0000010400033F8112090FBF2F0C1EB01110B
:103EE00000EB4100C0F30E00463000B210BD0029C7
:103EF000E5D125E0521E52B29C5C214481421DDD79
:103F0000081A64214843995C90FBF1F0042A09DB0C
:103F1000121F02EBC20101EB021100EB8100C0F3A2
:103F20000E0009E002EBC20101EB021100EB81007F
:103F3000C0F5C87040F4004000B210BD002AD9D1CD
:103F4000C34810BD2DE9F0410746C248B0F92C50D6
:103F5000B0F92E40281B1BF0D3FBBF4E31461BF09F
:103F60009DFA8046C8204443684200EB800004EB81
:103F7000C0001BF0C5FB31461BF090FAB74C214640
:103F80001BF01EFC054638461BF0D2FB41461BF0D9
:103F900017FC29461BF014FA21461BF07FFA1BF090
:103FA00073FB00B2BDE8F0812DE9F0471D46AC4E31
:103FB00040F2062301FB03F796F878344FF47A7841
:103FC0004FF0640900283AD00E2838D063283CD03E
:103FD0004FF4966A01FB0AFC40F2FF3A802836D083
:103FE0008B2834D0012835D00B2833D00D2831D080
:103FF000022855D082285ED0032867D0052865D0D6
:10400000072863D0082861D009285FD00A285DD02E
:10401000832873D0852871D087286FD088286DD0E9
:1040200089286BD08A2869D0042873D0842871D05D
:10403000062870D086286ED00C286DD0D5E097FB6E
:10404000F8F0434393FBF9F2CFE00A46CDE09CFB46
:10405000FAF2CAE0012816D00D2819D088B213212F
:10406000FFF7EAFE010402D5C0F30E00404296F8C5
:104070006E1031B100EBC000052190FBF1F000F5AE
:10408000A0704219B1E088B20221FFF7D5FEE9E73E
:1040900088B21421FFF7D0FE4628E3DA4620E1E794
:1040A00008461AF0E4FE6F4A6F4B1AF033FF1AF01D
:1040B000AFFE024699E008461AF0D9FE6B4A6C4BF7
:1040C0001AF028FF1AF0A4FE02468EE0B1F5F17F47
:1040D00009DC052805D0082803D00A2801D00122D0
:1040E00083E0002281E0032806D0072804D00928B5
:1040F00002D0012279E001E0002276E04FF4FA7369
:1041000099420CDC852808D0882806D08A2804D05B
:1041100001226AE00FE032E055E0002265E09942BA
:1041200063DD832805D0872803D0892801D00122A8
:104130005BE0002259E0042802D0842803D004E088
:1041400097FBF8F201E09CFBFAF2534393FBF9F181
:10415000404A38320428127802D0842807D00CE074
:10416000042309B20020FFF78CFD044605E08423F8
:1041700009B20020FFF785FD0446621935E00628E4
:1041800002D0862803D004E097FBF8F201E09CFB04
:10419000FAF2534393FBF9F12E4A3832062852784B
:1041A00002D0862807D00CE0062309B20020FFF7D2
:1041B00068FD044605E0862309B20020FFF761FD93
:1041C0000446621911E008461AF051FE294A2A4BAA
:1041D0001AF0A0FE1AF01CFE4FF4C871884200DAF3
:1041E000084680B2FFF7AEFE024610B26AE5811EB5
:1041F0000B2910D2DFE801F00B0F0F0606060606AA
:10420000060606001D49401F31F91000704711488D
:10421000B0F93C007047002070478008704770B5C7
:1042200005460C4602212846F4F775FC05230122B9
:1042300021462846F4F782FB01212846F4F757FB74
:1042400002211DE0ACFB0208BFFB0208D2FB020802
:10425000E883FFFF3C0200200000204300002041D3
:10426000607F002039B4C876BE9FBA3FC1CAA1455D
:10427000B6F3BD3F5C8FC2F5285CDF3F181200200B
:104280002846F4F741FC0028DAD02846BDE8704003
:10429000F4F79ABB70B50F21F948FFF7C0FF80B261
:1042A000FFF7BBFF01B20A20FFF767FDF54D95F858
:1042B0005F10132915D0142918D080B20221FFF7FE
:1042C000BBFDF14CA08400EBC001052291FBF2F193
:1042D00001F5A07109B2E18495F86E205AB1A18769
:1042E0000AE080B21321FFF7A7FDEAE780B21421AC
:1042F000FFF7A2FDE5E7A087A08FE087218D0844A6
:10430000A087E0480021D530F6F7EAFB38B195F8F0
:104310007B0395F87A1300EB0120608470BD95F85B
:104320005F00A8B1022816D0132814D0042815D095
:10433000D649032818D010281ED0112824D01228BE
:104340002FD0421F072A3DD831F8120060843FE089
:10435000A08F60843CE0A08F608439E0E08E94F907
:1043600000100844608433E0B1F90000B4F93C1057
:104370000844401060842BE0B1F90000B1F902104C
:1043800008444010608423E0B1F90000B1F9022034
:10439000B1F9041010440844032190FBF1F060844B
:1043A00016E0B1F90000B1F902201044B1F904207F
:1043B000B1F9061011440844C11700EB9170801048
:1043C000608405E0012808D0152809D0A08F6084FA
:1043D00095F8A20015280FD019E008886084F7E747
:1043E00095F82703FFF703FF034695F82803FFF727
:1043F000FEFE181A6084EBE795F82703FFF7F7FE37
:10440000034695F82803FFF7F2FE181A6087B4F9FF
:1044100022109F48814200DA6084B4F9221040F6ED
:10442000B83081427FF77AAF608470BD10B50D2837
:1044300027D009DC3DD2DFE800F02C242C242C24EA
:104440002424242424243400862812D00EDC83283B
:104450000FD006DC0E281CD080280AD0822828D154
:1044600007E0842805D0852823D102E08738042876
:104470001FD80120FFF7E4FABDE810400020FFF745
:10448000C5BA0120FFF7DCFABDE810400120FFF7B4
:10449000BDBA0020FFF7D4FABDE810400120FFF7B5
:1044A000B5BA0020FFF7CCFABDE810400020FFF7B6
:1044B000ADBA10BD10B508285DD2DFE800F0040FDA
:1044C0001A25303B46510020FFF708FB0020FFF77C
:1044D000EBFABDE810400020FFF7CCBA0020FFF750
:1044E000FDFA0020FFF7E0FABDE810400120FFF7D9
:1044F000C1BA0020FFF7F2FA0120FFF7D5FABDE8B4
:1045000010400020FFF7B6BA0020FFF7E7FA0120BD
:10451000FFF7CAFABDE810400120FFF7ABBA01204F
:10452000FFF7DCFA0020FFF7BFFABDE810400020DB
:10453000FFF7A0BA0120FFF7D1FA0020FFF7B4FA85
:10454000BDE810400120FFF795BA0120FFF7C6FA39
:104550000120FFF7A9FABDE810400020FFF78ABA52
:104560000120FFF7BBFA0120FFF79EFABDE81040DB
:104570000120FFF77FBA10BD02464249092A08D23E
:10458000DFE802F00705080B0E1114171A0091F866
:104590009E02704791F89F02704791F8A002704701
:1045A00091F8A102704791F8A202704791F8A30216
:1045B000704791F8A402704791F8A50270472DE961
:1045C000F84F00242F4FDFF8C480DFF8B4A0DFF8E5
:1045D000B89007F1D40BA8F114060120FFF798FA60
:1045E00021465846F6F77CFA50B107EB440090F8A4
:1045F0006B1390F86A0301EB002028F8140065E0C3
:10460000601CC0B2FFF7B8FF062843D03D1995F8EB
:10461000E500FFF70BFF2046FFF74CFF0A2003F0F1
:1046200057FF0B215046FFF7FAFD26F8140095F8C6
:10463000E5000C2805D036F81400FFF7EEFD26F84B
:10464000140095F8E500032812D0052810D0C11FEA
:1046500003290DD983280BD0852809D08738032852
:1046600006D936F914102046FFF787FB26F8140008
:1046700095F8E500042812D0842810D018E0000036
:1046800000240140607F00203C020020181200201E
:104690000CFEFFFFB9F8120028F8140016E099F894
:1046A0000910082902D289F80A4001E089F8094076
:1046B00036F9141000232246FFF776FC26F8140082
:1046C000F84931F81410084428F81400641CE4B2C6
:1046D000082C82D30A215046FFF7A1FDA9F80C004F
:1046E00099F8010001287DD00220F8F703FF14207B
:1046F00003F0EEFE0220F8F75BFF30820020F8F7AF
:10470000F9FE322003F0E4FE0020F8F751FFA9F88B
:10471000360097F8D902002865D040F2DB20FDF77B
:104720005EF80002A9F8200040F2DA20FDF757F801
:10473000B9F820100844A9F82000B9F920004FF476
:104740007A76B04201DDA9F82060B9F9200000278F
:10475000002801DAA9F82070B9F92010B9F936005B
:10476000F8F795FFA9F81800002500240821504605
:10477000FFF755FD0544032003F0AAFE641CE4B2D4
:104780001E2CF3D31E20B5FBF0F01AF0D1FF044627
:1047900020461AF095FFA9F81400C34920461BF0E3
:1047A0000FF8C2491AF07AFEC1491BF009F8C14955
:1047B0001AF074FE1AF068FF01460B20FFF7DDFACD
:1047C000A9F814000025002409215046FFF727FD11
:1047D0000544012003F07CFE641CE4B2142CF3D3E6
:1047E000142001E04CE05FE0B5FBF0F064214843A9
:1047F000000B00EB4000A9F8160001215046FFF71E
:104800000EFD00B243F6D00148430014A9F8300071
:1048100004215046FFF703FD00B243F6D0014843A0
:104820000014A9F832000C215046FFF7F8FCC0EB49
:10483000C0004000B0FBF6F0A9F80E000D21504674
:10484000FFF7EDFCC0EBC0004000B0FBF6F080B21B
:10485000A9F81000B9F80E100F2901D80F2859D95E
:1048600099F80B000A2802D2401D89F80B0099F82C
:104870000B000A2802D3012089F80200BDE8F88F56
:1048800032208D49009001230022081F01F0C3F956
:10489000D9F840001AF0F8FEA9F83600D9F844001B
:1048A0001AF0F2FE308234E797F80001834C50B3DF
:1048B000B6F910100920FFF760FA2080B9F81E1031
:1048C0000820FFF75AFAB9F83410084480B2A9F862
:1048D0001C004FF4C871884201D2A9F81C1099F845
:1048E0000100012812D0B9F93610B4F90000F8F728
:1048F000B6FEA9F820007249B9F8200009880844DA
:10490000A9F8200019E7308A2080D7E72088A9F885
:104910002000F0E799F80B0010B1401E89F80B0059
:1049200099F80B000028A9D189F80270A6E710B504
:10493000FFF708F9BDE81040FFF771B90146002004
:104940008A1E0B2A0CD2DFE802F00C0B0B060606BF
:1049500006060606060053483830491F30F9110094
:10496000704755484438B0F93C0070472DE9F04194
:10497000514A0020443A10714A4E0121323E3578A6
:10498000002D06D173880C2B02D93172117100E011
:1049900030724C4B012D93F86E400CD193F86C544F
:1049A000A54202D03172117100E03072B5790DB1BB
:1049B000307200E031723B4F283F3E463D787688AA
:1049C0002DB90C2E02D93972117100E03872012D07
:1049D0000FD193F86DC4A44502D03972117100E073
:1049E000387297F806C0BCF1000F01D0387200E0B1
:1049F0003972DFF8B0C0ACF11E0C9CF8007057B9EA
:104A0000BCF80280B8F1020F03D98CF808101171BC
:104A100001E08CF80800012F11D193F86E74A742C1
:104A200003D08CF80810117101E08CF808009CF894
:104A3000064014B18CF8080001E08CF80810DFF88B
:104A400064C0ACF10A0C64469CF8007064883FB9FD
:104A50000E2C03D08CF80810117101E08CF80800BE
:104A6000012F0FD1152C03D08CF80810117101E023
:104A70008CF808009CF8064014B18CF8080001E09E
:104A80008CF80810DFF81CC0ACF1140C64469CF8DC
:104A900000706488D7B90E2C16D08CF808101171EC
:104AA00014E00000E011002000803B4500F07F454D
:104AB0000000204100007C42800200206C000020A9
:104AC00040000020607F00208CF80800012F0FD1EB
:104AD000152C03D08CF80810117101E08CF8080037
:104AE0009CF8064014B18CF8080001E08CF808101E
:104AF00054793CB993F8B770022F02D091711171BB
:104B000000E09071012C07D193F8B840022C02D03C
:104B10009171117100E09071002D05D193F8A230D0
:104B2000B34203D0D1711171BDE8F081D071FBE7C0
:104B300070B5FFF71BFF3A4E96F86A04012837D18B
:104B4000384C3949A4F11405B4F90400B5F904301E
:104B5000364A984203DA04200870107002E0002000
:104B600008701070287818B9A878FFF7E7FEA880B9
:104B70002C4D0A3D287818B9A878FFF7DFFEA880E9
:104B8000207818B9A078FFF7D9FEA08096F86B04BA
:104B900001280DD1234926480A310A780AB9028C26
:104BA0008A80204914310A78002A01D1008C88803B
:104BB00070BDF0B51A4C0125002194F86A241C48F8
:104BC000012A0AD0C170C078012805D1194802888D
:104BD000428004F89E1F6570F0BD02790AB1C17071
:104BE000F1E70F4BDFF83CC00E4F5A7C9B7CACF1D9
:104BF000140C02EB0322BCF9043094F86B649A1A8B
:104C0000B7F904301EB19A4207DDC570DBE79A425E
:104C100001DDC570D7E7C170D5E7C170D3E70000EB
:104C2000607F0020C21100203B0000202C000020EB
:104C30003C020020540000202DE9F04FA1B00121DA
:104C40001020FBF788F801212020FBF784F80121D0
:104C50000820FBF780F8FC4C4FF40050217A04291F
:104C60000BD30121FBF777F801211120FBF773F833
:104C700001210220FBF77AF806E00121FBF76BF82F
:104C800001211120FBF767F8217AF04818274FF02F
:104C90000308042908D34FF0C001ADF860104FF0AD
:104CA0003001ADF8201003E04FF47071ADF8401002
:104CB0000FD38DF863708DF8628018A9F4F7A9F806
:104CC0008DF823708DF8228008A9E148F4F7A1F847
:104CD00006E08DF843708DF8428010A9F4F799F83A
:104CE000207A04280BD301210920FBF734F8012195
:104CF000D848F4F71FF90121D748F4F71BF9D24837
:104D000000250224007AD54E4FF001094FF47A7B3A
:104D10004FF0700A042824D3ADF858B0ADF85440D1
:104D2000ADF85A50ADF8565015A93046FBF7F0F9DA
:104D3000ADF844A0ADF84690ADF84C40ADF818B0D1
:104D4000ADF81440ADF81A50ADF8165005A9C44896
:104D5000FBF7DEF9ADF804A0ADF80690ADF80C4015
:104D600011E0ADF838B0ADF83440ADF83A50ADF8D8
:104D700036500DA93046FBF7CBF9ADF824A0ADF8BD
:104D80002690ADF82C40B048007A042810D311A921
:104D90003046FBF7F6F911A93046FBF72BFA01A9CB
:104DA000AF48FBF7EEF901A9AD48FBF723FA0FE096
:104DB00009A93046FBF7E5F909A93046FBF71AFACD
:104DC00009A93046FBF756FA09A93046FBF790FAD5
:104DD00008213046FBF770FD08213046FBF772FDD5
:104DE0009948007A042808D308219D48FBF764FD00
:104DF00008219B48FBF766FD0FE008213046FBF7D2
:104E00005BFD08213046FBF75DFD08213046FBF7CE
:104E100063FD08213046FBF765FD01213046FBF7B5
:104E200048FC01213046FBF750FC01210420FAF731
:104E30009DFF8548007A042807D301210220FAF754
:104E400095FF01218648FBF734FC01212120FAF768
:104E500082FF01210803F4F76DF84FF4E040ADF84C
:104E600080008DF883708DF8828020A97D48F3F74B
:104E7000D0FFADF878B0ADF87440ADF87A50ADF829
:104E80007650794D1DA92846FBF742F9ADF864A08C
:104E9000ADF86690ADF86C4019A92846FBF771F99A
:104EA00019A92846FBF7A6F919A92846FBF7E2F944
:104EB00008212846FBF700FD08212846FBF702FDE4
:104EC00008212846FBF708FD01212846FBF7F1FBE6
:104ED00021B0BDE8F08F0B461146012B07D0022B05
:104EE00007D0032B07D0042B07D1FBF70DBEFBF730
:104EF00005BEFBF705BEFBF705BE704730B40346A1
:104F0000514A574C5548127A062B27D2DFE803F056
:104F100026191D030E21042A04D320460A4630BC5C
:104F20000121D8E70A4630BC0321D4E7042A04D380
:104F300020460A4630BC0221CDE70A4630BC042197
:104F4000C9E70A4630BC0121C5E70A4630BC022148
:104F5000C1E70A4630BC01214348BCE730BC70477A
:104F6000414B002804D04FF47A7203211846B2E76F
:104F7000002203211846AEE73B4B002804D04FF433
:104F80007A7202211846A6E7002202211846A2E7FB
:104F90002DE9F84F83463548421C02F1010A00789A
:104FA0009AF800101278BBF1080F6CD2DFE80BF012
:104FB0006B040F1B27333F60002500F0010601F052
:104FC000010402F00107A8464FF001095BE001254A
:104FD000C0F34006C1F34004C2F340074FF002089B
:104FE0004FF003094FE00225C0F38006C1F38004AF
:104FF000C2F380074FF004084FF0050943E0032592
:10500000C0F3C006C1F3C004C2F3C0074FF00608E6
:105010004FF0070937E00425C0F30016C1F3001470
:10502000C2F300174FF008084FF009092BE00525DF
:10503000C0F34016C1F34014C2F340174FF00A0802
:105040004FF00B091FE00000607F002000100140BE
:10505000000C01400004300000081A000034014038
:1050600000040040001401400008004090020020AD
:105070000625C0F38016C1F38014C2F380174FF0E9
:105080000C084FF00D09B74245D1FF484146008951
:10509000F5F708FD0090A6B100200099884220D0C5
:1050A0008EB10022F84841460830F5F70CFDF6486D
:1050B000F649009A0A3042B1294491F8421141550B
:1050C00007E00120E9E70122ECE7294491F84911C2
:1050D0004155405D28B1EC48012249460830F5F7BA
:1050E000F2FCE94D49462889F5F7DCFC002812D18D
:1050F00085F801B007B90124BBF1080F0BD2DFE836
:105100000BF00A040C131A21282F9AF8000064F3FC
:1051100000008AF80000BDE8F88F9AF8000064F3F8
:1051200041008AF80000F6E79AF8000064F3820074
:105130008AF80000EFE79AF8000064F3C3008AF8E9
:105140000000E8E79AF8000064F304108AF8000011
:10515000E1E79AF8000064F345108AF80000DAE706
:105160009AF8000064F386108AF80000D3E72DE96E
:10517000F84FC748DFF81C830078002823D00124AB
:10518000DFF804A34FF000090AF1040AAAF10106AE
:10519000F51EAF1C2046FFF7FBFE6878002877D08D
:1051A000012803D09AF80010CA0772D038783178F5
:1051B000401C60F3000131709AF8000020F00100FB
:1051C0008AF80000CDE0B8F90000C82815DA4FF4DD
:1051D0007A710120FFF792FE00210220FFF78EFE78
:1051E00000210320FFF78AFE00210420FFF786FE3E
:1051F00000210520FFF782FE61E0B0F5C87F15DAD7
:1052000000210120FFF77AFE4FF47A710220FFF7A8
:1052100075FE00210320FFF771FE00210420FFF737
:105220006DFE00210520FFF769FE48E0B0F5167F0E
:1052300015DA00210120FFF761FE00210220FFF7AF
:105240005DFE4FF47A710320FFF758FE0021042021
:10525000FFF754FE00210520FFF750FE2FE0B0F5C8
:10526000487F17DA00210120FFF748FE00210220C5
:10527000FFF744FE00210320FFF740FE4FF47A7150
:105280000420FFF73BFE00210520FFF737FE16E064
:1052900069E027E000210120FFF730FE0021022015
:1052A000FFF72CFE00210320FFF728FE0021042039
:1052B000FFF724FE4FF47A710520FFF71FFE764CAE
:1052C000B8F8002002212046FFF705FEB8F80220BA
:1052D00003212046FFF7FFFDBDE8F84F4FF4FA70B9
:1052E00003F0F6B8022801D08A070BD53878327857
:1052F0004010401C60F34102327021F002008AF835
:1053000000002EE0032801D04A070BD53878327808
:105310008010401C60F38202327021F004008AF891
:1053200000001EE0042801D00A070BD53878327837
:10533000C010401C60F3C302327021F008008AF8EC
:1053400000000EE0052801D0C8060AD5387832786A
:105350000011401C60F30412327021F010008AF832
:10536000000085F80190641CE4B2062CFFF412AF33
:10537000DFF818A1DFF824B10AF1D6009AF86A1014
:105380000090062917D0002421460098F5F7A8FBC5
:1053900078B30AEB040090F8B900032831D0214615
:1053A0003F48F5F79DFB28B3002237482146C01C33
:1053B000F5F77CFB25E03B48007838B12878C0073A
:1053C0000DD0E9880120FFF799FD7BE00021012045
:1053D000FFF794FD287800F0FE00287072E04FF48B
:1053E0007A710120FFF78AFD297841F001012970C7
:1053F00068E001E00122D8E72C482B4900EB84103B
:10540000C1619BF80000012820D19AF853020228BC
:1054100002D001280ED014E021462548F5F760FBA4
:1054200030B1002218482146C01CF5F73FFB08E0C8
:105430000122F7E72CB98AF8D6900021D620FCF794
:10544000CFF9042C02D103208BF80000641CE4B2D5
:10545000052C99D396F80090164809F001010180B7
:105460000024124850F824001AF02AF91149A21C0D
:1054700021F81200641CE4B2092CF2D35FEAC9706F
:1054800030D00021012017E08E020020607F002034
:1054900077000020BE000020000800405A000020D5
:1054A000C68200203B00002000007F43488400208B
:1054B000B481002036120020FFF720FD287800F08C
:1054C000FE0028703078800723D4287880071BD40A
:1054D0004FF47A710220FFF711FD297841F00201A3
:1054E00029701EE02878C00704D0E9880120FFF762
:1054F00005FDE7E74FF47A710120FFF7FFFC2978FB
:1055000041F001012970DDE7E9880220FFF7F6FC90
:1055100007E000210220FFF7F1FC287800F0FD00F1
:1055200028703078400711D42878400709D44FF408
:105530007A710320FFF7E2FC297841F00401297019
:105540000CE0E9880320FFF7D9FC07E000210320E5
:10555000FFF7D4FC287800F0FB00287030780007B3
:1055600011D42878000709D44FF47A710420FFF78A
:10557000C5FC297841F0080129700CE0E988042075
:10558000FFF7BCFC07E000210420FFF7B7FC2878F8
:1055900000F0F70028703078C00611D42878C006D3
:1055A00009D44FF47A710520FFF7A8FC287840F061
:1055B000100028700CE0E9880520FFF79FFC07E049
:1055C00000210520FFF79AFC287800F0EF002870F2
:1055D0009BF8000001280DD19AF85302022809D146
:1055E000012205210098F5F761FA012206210098B1
:1055F000F5F75CFA05210098F5F772FA80B39BF88D
:105600000000012803D19AF85302022811D09AF819
:10561000620300029AF86313084400B29AF87B1000
:1056200079B111290DD082B202215848FFF753FCFD
:1056300026E09AF8560200029AF85512084400B281
:10564000ECE7012805D0002202215048FFF743FC77
:1056500016E04FF47A7202214C48FFF73CFC0FE051
:10566000FFE79AF87B00A8B101281ED004281CD0BF
:1056700011280FD0B8F8002002214448FFF72BFC76
:1056800006210098F5F72CFAF0B39BF800000128EA
:1056900024D027E03878800603D50120FFF76CFC82
:1056A000EEE70020FFF768FCEAE79AF86A040128B1
:1056B0000DD19AF86F04B8F9001000EB8002B1EB3D
:1056C000420F04DA00EB80004000A8F80000B8F8B0
:1056D000002002212D48FFF7FEFBD1E79AF8530284
:1056E000022816D09AF8640300029AF86513084459
:1056F00000B29AF87C1091B19AF87B1011290ED063
:1057000082B20321214800E01AE0BDE8F84FFFF71C
:10571000E2BB9AF857020102084400B2E9E7012807
:1057200006D0BDE8F84F002203211848FFF7D3BB8D
:10573000BDE8F84F4FF47A7203211448FFF7CBBB52
:105740009AF87C0068B1012818D0042816D01128D6
:1057500007D0B8F80220BDE8F84F03210B48FFF747
:10576000BABB3878400604D5BDE8F84F0120FFF7F2
:10577000F7BBBDE8F84F0020FFF7F2BBB8F80220F6
:10578000BDE8F84F03210148FFF7A5BB0008004022
:1057900010B5FBF70EFE0120FBF745FE012002F0DD
:1057A00077FE0120FBF734FE012002F071FE00209D
:1057B000FBF739FE0A2002F06BFE0020FBF728FE03
:1057C000BDE810400A2002F063BE10B5FBF7F1FD02
:1057D0000020FBF71DFE012002F05AFE0020FBF71F
:1057E00022FE012002F054FE0120FBF711FE0A20E8
:1057F00002F04EFE0120FBF716FEBDE810400A2025
:1058000002F046BE70B50546FBF7D3FD80242C425E
:1058100003D10020FBF707FE02E00120FBF703FEA7
:10582000052002F035FE0120FBF7F2FD052002F015
:105830002FFE0020FBF7ECFD012002F029FE64089A
:10584000002CE4D1BDE87040FBF75ABE70B50446A9
:105850000025FBF7D1FD4FF47A7607E0641EE4B231
:1058600001D2042070BD304602F012FEFBF7EBFDC2
:105870000028F3D0284670BD2DE9F04105460E46BC
:105880001746002028700120FBF7CDFDFBF780FDB7
:1058900080240120FBF7BCFD012002F0F9FD384611
:1058A000FFF7D4FF8046032002F0F2FDFBF795FDE1
:1058B000FBF7C4FD10B12878204328700020FBF7C7
:1058C000A7FD012002F0E4FD6408002CE1D1FBF704
:1058D00070FDBEB10120FBF7A6FD012002F0D8FD4E
:1058E0000120FBF795FD052002F0D2FD0020FBF71B
:1058F0008FFD0120FBF797FD142002F0C9FD404603
:10590000BDE8F0810020FBF78EFDE6E710B5FFF75C
:105910003FFF0020FFF776FF002803D1BDE81040CD
:1059200006206FE710BD0000F9494000087040F004
:10593000010048707047F7E7FFF747BF70B50546AD
:10594000FF20002340F2311410E0EA5C50400822AE
:10595000060603D584EA4000C0B201E04006000E0E
:10596000521ED2B2002AF3D15B1CDBB28B42ECD3C5
:1059700070BD10B51446FFF7E1FFA04201D0022030
:1059800010BD002010BD7CB504460D46002101A8C5
:10599000FFF772FF28B9002211460DF10500FFF74D
:1059A0006BFF20B9002229466846FFF765FF28B93A
:1059B0009DF80020022101A8FFF7DBFF9DF80510EC
:1059C0009DF8042041EA022121807CBD10B5FFF73B
:1059D000DFFECF484078BDE81040FFF713BF70B539
:1059E0000446200AFFF70EFF0546E0B2FFF70AFF64
:1059F000284370BD10B5FFF7CBFEC5480078BDE861
:105A00001040FFF7FFBEF8B50646FFF7F3FF054667
:105A10004FF45E50FFF7E3FF40EA050414B9FFF7C7
:105A2000D5FF04462CB9642200216846FFF7ABFF7E
:105A3000044634B9002201210DF10200FFF7A3FF53
:105A40000446FFF779FF34B9BDF80200BDF8001035
:105A500040EA014030602046F8BD70B50546FFF7CA
:105A6000C9FF044624B94FF22D30FFF7B8FF0446B2
:105A700014B9FFF7ABFF04462CB9002201212846D8
:105A8000FFF781FF0446FFF757FF204670BD10B5B2
:105A9000FFF7B0FF044624B943F24100FFF79FFF30
:105AA0000446FFF749FF204610BD10B519F040FE2F
:105AB000984919F085FE984919F082FEBDE810401A
:105AC000964919F0EBBC10B519F032FE944919F063
:105AD00077FE914919F074FE904919F0DFFCBDE89A
:105AE0001040904919F042BF2DE9FC410746884615
:105AF00016461D46FFF77EFF0446200005D196B1ED
:105B0000012E0AD0022E02D0802494B120E042F26D
:105B10001640FFF764FF0446F7E742F20B40FFF739
:105B20005EFF0446F1E74FF41050FFF758FF0446BC
:105B3000EBE74FF47A7606E0FFF748FF04462CB116
:105B4000304602F0A5FC6D1EEDB2F5D205B9042475
:105B500064B90022114601A8FFF715FF054600228F
:105B600001216846FFF70FFF40EA0504FFF7E4FE56
:105B700054B9BDF80400FFF7A6FF3860BDF8000077
:105B8000FFF793FFC8F800002046BDE8FC812DE92F
:105B9000FC4106460F4615469846FFF72BFF044684
:105BA0002CB995B1012D0AD0022D02D0802494B1D8
:105BB00014E042F61040FFF712FF0446F7E742F602
:105BC0000D40FFF70CFF0446F1E742F60640FFF7F1
:105BD00006FF0446EBE7FFF7F9FE04462CB9424600
:105BE000002101A8FFF7CFFE04462CB900220121B5
:105BF0006846FFF7C8FE0446FFF79EFE4CB9BDF8A5
:105C00000400FFF760FF3060BDF80000FFF74DFFB4
:105C100038602046B9E730B4029C002B04D0012B39
:105C200005D0802030BC7047234630BCAFE7234608
:105C300030BC59E770B505460E46FFF7DBFE04465B
:105C40002CB97DB3012D2ED0022D04D08024FFF776
:105C500073FE204670BD052E22D2DFE806F0030950
:105C60000F151B0042F22F00FFF7B9FE0446EEE7C6
:105C700042F22D10FFF7B3FE0446E8E742F22B2074
:105C8000FFF7ADFE0446E2E742F22930FFF7A7FE38
:105C90000446DCE742F22A70FFF7A1FE0446D6E78D
:105CA0008024D4E726E0052E22D2DFE806F003099F
:105CB0000F151B0042F22400FFF791FE0446C6E7D1
:105CC00042F22610FFF78BFE0446C0E742F2202086
:105CD000FFF785FE0446BAE742F22230FFF77FFE67
:105CE0000446B4E742F22170FFF779FE0446AEE7BE
:105CF0008024ACE7052E2FD2DFE806F003161C2225
:105D0000280042F23200FFF76AFE04469FE70000D7
:105D1000A00200200000C8420000204100FF7F4791
:105D200000002F430000E14342F23010FFF757FE1E
:105D300004468CE742F23620FFF751FE044686E720
:105D400042F23430FFF74BFE044680E742F23770F0
:105D5000FFF745FE04467AE7802478E77CB50546E0
:105D60000E46FFF747FE044624B94FF46040FFF7A4
:105D700036FE044614B9FFF729FE04462CB900226A
:105D8000114601A8FFF7FFFD04462CB900220121AE
:105D90006846FFF7F8FD04464CB9BDF80400FFF76C
:105DA00092FE2860BDF80000FFF77FFE3060FFF72D
:105DB000C3FD20467CBD10B5FFF71CFE044624B988
:105DC00043F26D00FFF70BFE0446FFF7B5FD2046DA
:105DD00010BD10B5FFF70EFE044624B943F266006D
:105DE000FFF7FDFD0446FFF7A7FD204610BD70B587
:105DF000FFF700FE054643F2A200FFF7F0FD40EA80
:105E00000504FFF799FD1CB94CF2503002F040FB3D
:105E1000204670BD10B5244C4FF0805020602348C0
:105E200002F036FBA0142060BDE810404CF2503068
:105E300002F02EBB38B5010A8DF800108DF8010074
:105E400002216846FFF77AFD04469DF80000FFF73F
:105E5000D9FC18B99DF80100FFF7D4FC002802D145
:105E60002046FFF7CFFC38BD10B5114919F0A8FA4C
:105E7000104919F013FB104919F0A2FC19F020FC8D
:105E800080B210BD10B50D4919F008FB0A4919F090
:105E900097FC19F015FC80B210BD03480838006863
:105EA000C0F3802070470000100C0140A086010064
:105EB0000000344200002F4300FF7F470000C8422B
:105EC000F0B503460025084600260A2A01D00670D0
:105ED000F0BD002B1DD005DA4FF02D0200F8012B8C
:105EE000C3F1000342F210724FF00A0793FBF2F481
:105EF00054EA050C06D004F1300500F8015B04FB00
:105F00001233012592FBF7F2002AEFDC06700846F7
:105F1000F0BD3022027046700846F0BD0FB430B5B7
:105F200085B005460AA800900EE05C2914D025290A
:105F30002CD0521C28460992FAF73CFF80212846B3
:105F4000FAF7A5FF0028F9D0099A11780029ECD1B9
:105F500005B030BC5DF814FB521C099210786E2815
:105F60000CD0722802D0521C0992E7E70D21284676
:105F7000FAF720FF0998401C0990DFE70A2128461C
:105F8000FAF718FF0998401C0990D7E7521C0992AC
:105F90001078642819D0732802D0521C0992CDE7DA
:105FA000009810C8009009E02846FAF703FF802106
:105FB0002846FAF76CFF0028F9D0641C21780029E4
:105FC000F2D10998401C0990B8E7009808C80090E1
:105FD0000A2201A91846FFF773FF01AC09E0284621
:105FE000FAF7E8FE80212846FAF751FF0028F9D099
:105FF000641C21780029F2D10998401C09909DE782
:1060000008B54FF4A060F2F787FB34208DF800004C
:1060100000208DF801008DF8020001208DF80300AA
:106020006846F2F77EFB08BD10B586B00121C804B2
:10603000F9F79CFE01211020F9F78DFE4FF48060E6
:10604000ADF8140018208DF8170003208DF8160005
:10605000FD4C05A92046F2F7DCFEE114ADF8141062
:1060600004218DF8171005A92046F2F7D2FE4FF44F
:10607000E13001900020ADF80800ADF80A00ADF85D
:106080000C00ADF810000C20ADF80E00EF4C01A98B
:106090002046FAF7B3FD012240F225512046FAF7D7
:1060A00034FE012240F224412046FAF72EFEFFF78B
:1060B000A7FF01212046FAF71CFE06B010BD08B567
:1060C00010208DF8030003208DF80200012120200C
:1060D000F9F741FE0420ADF800006946DC48F2F70C
:1060E00098FE08BD10B5FFF7EAFFFFF79DFF01F02E
:1060F00074FBBDE810400421D548F2F7F9BE10B595
:10610000D34C04212046F2F7F5FE4FF4FA7002F06A
:10611000DFF92046BDE810400421F2F7E9BE2DE981
:10612000F04706460D4691461F46DFF82883B8F82B
:1061300000046FF30E00A8F800040024DFF80CA39D
:106140000BE0315D5046FAF735FE80215046FAF7F4
:106150009EFE0028F9D0641CA4B2BC42F1D3B8F86A
:1061600000046FF30E00A8F8000498F8010420F072
:10617000800088F80104002404E0322002F0A8F92D
:10618000F9F7B1FC98F80104000604D42046641C19
:10619000A4B20A28F1D3B8F800140020C1F30E010C
:1061A00008F8010085B1B9F1000F0DD02946A948C2
:1061B00016F0ECFA28B94946A64816F0E7FA002886
:1061C00000D00120BDE8F0873DB12946A14816F076
:1061D000DDFA0028F6D00120F4E749469D4816F084
:1061E000D5FA0028EED00120ECE72DE9F0410D466C
:1061F00090461E46024698A19448FFF78FFE55EA46
:10620000080012D0934FB7F800046FF30E00A7F800
:10621000000497F8010420F0800087F801040024AE
:106220003220B6FBF0F086B207E00120BDE8F08135
:10623000322002F04DF9F9F756FC97F801040006F8
:1062400004D42046641CA4B2B042F1D3B7F80014C1
:106250000020C1F30E0178547DB1B8F1000F0CD0CD
:1062600029467C4816F092FA28B94146794816F03A
:106270008DFA0028DAD00120D8E73DB129467548CB
:1062800016F084FA0028D1D00120CFE741467148AA
:1062900016F07CFA0028C9D00120C7E770B50024A9
:1062A00004216B48F2F724FE4FF47A7002F010F9E3
:1062B0004FF4FA750CE02B46002269A169A0FFF7A4
:1062C00094FF08B1022070BDFFF719FF641CE4B20F
:1062D0000A2CF0D301D0012070BD002070BD40F623
:1062E000C413002805D0012807D0022809D00020B7
:1062F00070475DA25AA15FA077E75BA258A160A09A
:1063000073E759A256A161A06FE700B59FB00B4695
:10631000024661A101A8F2F75FFE41F28833002234
:106320004FA101A8FFF761FF1FB000BD00B59FB0EE
:106330000B4602465DA101A8F2F74EFE41F28833FA
:10634000002247A101A8FFF750FFEDE72DE9F0413A
:10635000CEB0642135A816F00FFB0024594D13AEC2
:10636000281906EB840190F86A000A22FFF7A8FDBD
:10637000641CE4B2042CF3D300240FAF281907EBFC
:10638000840190F86E000A22FFF79AFD641CE4B2C3
:10639000042CF3D300240DF12C08281908EB8401F8
:1063A00090F872000A22FFF78BFD641CE4B2042C03
:1063B000F3D312A811A9CDE9081010AACDE90672ED
:1063C0000EA80DA9CDE9041016A815A90CAACDE9AF
:1063D0000010CDE90282331D13AA3BA135A8F2F7C4
:1063E000FBFD35AA43A117A8F2F7F6FD4FF47A6337
:1063F00000221BA117A8FFF7F8FE4EB016E700B564
:106400009FB00B46009202463FA101A8F2F7E4FDBF
:106410004FF47A73002212A101A8FFF7E6FE83E78A
:1064200000B585B0002801D0012200E000223CA187
:106430006846F2F7D1FD4FF4FA73002208A16846CE
:10644000FFF7D3FE05B000BD00100140004C004036
:10645000001401405412002025730D0A00000000B2
:106460004F4B0000415400006E6F206368616E67FF
:106470006500000041542B43574D4F44453D3100CA
:1064800041542B43574D4F44453D320041542B431B
:10649000574D4F44453D330041542B43574A4150DB
:1064A0003D222573222C22257322000041542B43C8
:1064B000574A41505F4445463D222573222C2225F0
:1064C00073220000872200202225732E25732E259B
:1064D000732E2573222C2225732E25732E25732EC1
:1064E0002573222C2225732E25732E25732E2573BA
:1064F0002200000041542B4349505354415F44450E
:10650000463D25730000000041542B435753415032
:106510003D222573222C222573222C312C25640048
:1065200041542B4349504D55583D2564000000000F
:10653000F0B5B9B004460F4615461E46642120A8A2
:1065400016F01AFA14B1012C0FD107E03B46F6A25F
:10655000F6A120A80095F2F73FFD06E03B46F7A222
:10656000F2A120A80095F2F737FD052E06D220AB48
:106570003246F3A102A8F2F72FFD04E020AAF5A10C
:1065800002A8F2F729FD4FF47A63F6A2AFF23011B8
:1065900002A8FFF72AFE39B0F0BD2DE9F041BAB0EC
:1065A0008046409F0E4615461C46642121A816F0E1
:1065B000E3F9CDE900654346E0A2EEA121A80294EB
:1065C000F2F70AFD052F06D221AB3A46DCA103A85B
:1065D000F2F702FD04E021AADEA103A8F2F7FCFC19
:1065E0004FF47A63DFA2AFF2881103A8FFF7FDFD35
:1065F0003AB01BE610B59EB04FF4FA7400280ED0E6
:106600000B460122E0A16846F2F7E6FC2346002291
:10661000AFF2B4116846FFF7E8FD1EB010BD0B469F
:106620000022D9A16846F2F7D7FC23460022AFF238
:10663000D0116846FFF7D9FDEFE710B54FF4FA73B4
:106640000022AFF2E411D5A0FFF7CFFDD8B1D7A15A
:10665000D94816F09BF808B1022010BDD7A1D64842
:1066600016F094F808B1032010BDD7A1D24816F057
:106670008DF808B1042010BDD6A1CF4816F086F8D9
:1066800008B1052010BD062010BD10B500244FF440
:10669000FA730022AFF23821C0A0FFF7A6FD002850
:1066A0002DD0CFA1C44816F071F800B10124D0A1BB
:1066B000C14816F06BF810B144F0020401E024F078
:1066C0000204CFA1BC4816F061F810B144F00404F4
:1066D00001E024F00404CEA1B74816F057F810B139
:1066E00044F0080401E024F00804CDA1B24816F0FB
:1066F0004DF810B144F0100401E024F010042046DD
:1067000010BD2DE9FE4380460E4617464FF4FA7938
:106710004B460022AFF2B821C5A0FFF766FD002569
:106720000024C6A1A44816F031F810B1C21D002003
:106730003BE00020BDE8FE83115C2E2902D0032D32
:1067400027D028E0012C04D0022C06D0032C0ED038
:106750001BE09DF80810715517E09DF808109DF892
:10676000093001EB810103EB410171550DE09DF80A
:10677000083064214B439DF8091001EB810103EBC4
:1067800041019DF80A30194471556D1CEDB2002489
:1067900009E022290BD0303923460DF1080C641C86
:1067A000E4B20CF80310401CC0B2B842C4D3012CB0
:1067B00004D0022C06D0032C0ED01BE09DF808005C
:1067C000705517E09DF808009DF8091000EB800057
:1067D00001EB400070550DE09DF808106420414326
:1067E0009DF8090000EB800001EB40009DF80A10C5
:1067F000084470554B460022AFF29C3191A0FFF740
:10680000F4FC0025002493A16B4815F0BFFF20B1D4
:1068100000F10B0300206E462BE000208AE7195C94
:106820003A2902D0052D0ED00FE0022C07D19DF899
:1068300001109DF8002001EB021108F805106D1CF5
:10684000EDB2002413E0222915D0A1F13002092A6B
:1068500004D82146641CE4B2725408E0A1F161023C
:10686000052A04D857392246641CE4B2B154401CAE
:10687000C0B2B842D3D3022C07D19DF801009DF8D5
:10688000001000EB011008F805004B460022AFF2A3
:10689000304174A0FFF7A9FC002476A1464815F00A
:1068A00075FF18B10C300021754B0BE0002041E75B
:1068B000425C222A08D025461D44641CE4B2AA7218
:1068C000491CC9B2B942F3D3012033E72DE9FF4196
:1068D00007464FF4FA730022AFF27C4169A0FFF73C
:1068E00084FC002500246BA1334815F04FFF20B134
:1068F000431D002002AA03AE02E0002004B095E48C
:10690000195C2E2902D0032D0BD0E5E0012C04D018
:10691000022C07D0032C06D0D8E09DF80C1051555E
:10692000D4E0D7E0BAE0C3E05443500022257322FC
:106930002C222573222C25730000000055445000A2
:1069400041542B43495053544152543D25642C2506
:106950007300000041542B43495053544152543D5D
:1069600025730000414C5245415920434F4E4E453E
:1069700043540000222573222C222573222C2564E7
:106980002C25642C2564000041542B434950534569
:10699000525645523D25642C2573000041542B432B
:1069A000495053544154555300000000535441542E
:1069B00055533A320D0A00005412002053544154EA
:1069C00055533A330D0A00005354415455533A3449
:1069D0000D0A00005354415455533A350D0A000036
:1069E0002B4349505354415455533A302C00000026
:1069F0002B4349505354415455533A312C00000015
:106A00002B4349505354415455533A322C00000003
:106A10002B4349505354415455533A332C000000F2
:106A20002B4349505354415455533A342C000000E1
:106A300041542B43494653520000000053544149EE
:106A4000502C220041542B4349505354414D414353
:106A50003F0000002B4349505354414D41433A22DB
:106A60000000000041542B43574A41505F435552A8
:106A70003F0000002B43574A41505F4355523A00B4
:106A80008722002041542B4349505354415F4355C2
:106A9000523F00003A69703A220000009DF80C1045
:106AA0009DF80D4001EB810104EB410151550DE0D2
:106AB0009DF80C4064214C439DF80D1001EB8101C1
:106AC00004EB41019DF80E40214451556D1CEDB27F
:106AD000002407E022290AD03039A446641CE4B21D
:106AE00006F80C10401CC0B22828FFF405AF012C9A
:106AF00004D0022C06D0032C0ED01BE09DF80C0015
:106B0000505517E09DF80C009DF80D1000EB80002B
:106B100001EB400050550DE09DF80C1064204143FE
:106B20009DF80D0000EB800001EB40009DF80E1079
:106B300008445055DFF83484E7B19DF8080098F810
:106B40006A10884211D19DF8090098F86B108842AC
:106B50000BD19DF80A0098F86C10884205D19DF879
:106B60000B0098F86D10884207D00298C8F86A00A8
:106B70000220C3E60298C8F86A0000250024FCA1A0
:106B8000FE4815F003FE20B100F10A03002001AA1F
:106B900001E00020B2E6195C2E2902D0032D27D097
:106BA00028E0012C04D0022C06D0032C0ED01BE0D0
:106BB0009DF80C10515517E09DF80C109DF80D40F4
:106BC00001EB810104EB410151550DE09DF80C40B2
:106BD00064214C439DF80D1001EB810104EB410150
:106BE0009DF80E40214451556D1CEDB2002407E084
:106BF000222909D03039A446641CE4B206F80C10EE
:106C0000401CC0B22828C6D3012C04D0022C06D0C8
:106C1000032C0ED01BE09DF80C00505517E09DF89A
:106C20000C009DF80D1000EB800001EB400050556A
:106C30000DE09DF80C10642041439DF80D0000EB21
:106C4000800001EB40009DF80E1008445055E7B15C
:106C50009DF8040098F87210884211D19DF8050043
:106C600098F8731088420BD19DF8060098F87410BC
:106C7000884205D19DF8070098F87510884207D022
:106C80000198C8F87200022038E60198C8F872002E
:106C900000250024BAA1B94815F078FD20B100F113
:106CA0000A0300206A4601E0002027E6195C2E292D
:106CB00002D0032D27D028E0012C04D0022C06D0CE
:106CC000032C0ED01BE09DF80C10515517E09DF8D9
:106CD0000C109DF80D4001EB810104EB4101515571
:106CE0000DE09DF80C4064214C439DF80D1001EB24
:106CF000810104EB41019DF80E40214451556D1C6A
:106D0000EDB2002407E0222909D03039A446641CE2
:106D1000E4B206F80C10401CC0B22828C6D3012CDF
:106D200004D0022C06D0032C0ED01BE09DF80C00E2
:106D3000505517E09DF80C009DF80D1000EB8000F9
:106D400001EB400050550DE09DF80C1064204143CC
:106D50009DF80D0000EB800001EB40009DF80E1047
:106D600008445055E7B19DF8000098F86E1088422D
:106D700011D19DF8010098F86F1088420BD19DF851
:106D8000020098F87010884205D19DF8030098F829
:106D90007110884207D00098C8F86E000220ADE557
:106DA0000098C8F86E000120A8E510B54FF4FA74F9
:106DB00023460022AFF6581174A0FFF716FA40B12F
:106DC000234676A2AFF66811BDE8104074A0FFF725
:106DD0000CBA002010BD10B54FF47A7001F078FBAA
:106DE00072A17348FFF79AF8BDE810404FF4FA70AB
:106DF00001F06EBB70B51446ADF5167D0E461A4611
:106E0000002540F226218C4203D900200DF5167D85
:106E100070BD38B13246AFF2B8416548FFF77EF831
:106E2000012520E0052A05D2234662A16846F2F733
:106E3000D3F804E0224664A16846F2F7CDF868462C
:106E400015F0DAFC81B211B1B1F5077F01D900204C
:106E5000DCE7684600F00BFD022001F039FBA1B22F
:106E6000304600F004FD2846D0E700B59FB064210D
:106E700006A815F081FD06AA57A101A8F2F7ACF803
:106E80004FF47A630022AFF6282101A8FFF7ADF98D
:106E90001FB000BD2DE9F04781460027DFF8DC80F8
:106EA000B8F800046FF30E00A8F8000498F8010485
:106EB00020F0800088F8010440F20241404615F0BD
:106EC00039FD00240026494D3EE0022001F000FB80
:106ED0002978182904D0192914D0162919D031E09D
:106EE000FFF734FA70B3424820496A3102780A70D9
:106EF00042784A7082788A70C078C870FFF7FFF8CD
:106F00002E701FE0FFF7B1FFE0B1FFF7F8F82E7029
:106F100018E04FF4FA730022AFF6BC2135A0FFF75A
:106F200064F900B12E70114840210A3015F002FDBD
:106F30000E4820214A3015F0FDFC314901204871EE
:106F400008F062FAF8F7CFFD98F80104000604D4BF
:106F50002046641CA4B26428B7D3B8F80004C0F378
:106F60000E0008F80060B9F1000F4BE08722002006
:106F70003A676174657761793A2200005412002003
:106F80003A6E65746D61736B3A22000041542B4375
:106F900049504D4F44453D31000000003E00000087
:106FA00041542B43495053454E4400002B2B2B009A
:106FB000004C004041542B43495053454E443D251D
:106FC000642C25640D0A000041542B43495053455D
:106FD0004E443D25640D0A0041542B435744484319
:106FE000505F4445463D312C310000000F03002026
:106FF000BE84002041542B524553544F524500004B
:107000005D04002001D0624F05E062A1604815F0E8
:10701000BDFB00B15E4F3846BDE8F08770B5027A1F
:107020002C2A01D0002070BD827A3A2A10D1437AEE
:10703000303B092B0CD89BB2002205E08418E47A7F
:1070400001F8014B521C92B29A42F7D3184670BD18
:10705000C37A6FF02F053A2B03D0047B3A2C1AD059
:107060003EE0437A303B092B3AD8302A38D3392ACC
:1070700036D803EB830305EB43031A4493B2002293
:1070800005E08418247B01F8014B521C92B29A420D
:10709000F7D3184670BD447A303C092C20D8302AEA
:1070A0001ED3392A1CD8302B1AD3392B18D804EB0D
:1070B000C406303A06EB041402EB820203EB8403AD
:1070C00005EB42021A4493B2002205E08418647B67
:1070D00001F8014B521C92B29A42F7D3184670BD88
:1070E000002070BD70B5044640212C4815F022FCEC
:1070F0002A49652514B1012C02D003E00D8001E07E
:10710000672008801D204880254802788A804278C0
:10711000CA8082780A81C2784A8109228A81837969
:10712000CB81204A14780C8254784C8294788C82DB
:10713000D478CC8232F8684C0C834D83007A8883F3
:1071400019480068C0F3072444EA00244C8481F8FD
:107150002430030C1B0243EA1060A1F83900002020
:1071600081F83B0032F8662C8A8781F83E0081F86E
:107170003F000E490120087070BD0B0A037041707A
:1071800000218170C170110A0171427170470000C5
:10719000541200202B4950440000000056160020D5
:1071A000607F0020F12200200C000020A3020020BC
:1071B00070B50024F84D4FF4FA76FFF73EFAA87147
:1071C000401E032808D3304601F082F9F8F78BFC03
:1071D000641CE4B20A2CF0D3A879032807D1334603
:1071E000BDE870400022EDA1EDA0FEF7FEBF70BD2E
:1071F00070B500244FF47A7504E0F8F774FC64204D
:1072000001F066F92B460022E4A1E9A0FEF7EDFFAC
:10721000002804D12046641CE4B21428EDD370BDCC
:1072200010B5002404E0F8F75EFC642001F050F98A
:1072300064230022D9A1E1A0FEF7D7FF002804D1E2
:107240002046641CE4B21428EDD310BD10B5002410
:1072500004E0F8F748FC642001F03AF964230022C6
:10726000CEA1DAA0FEF7C1FF002804D12046641C9D
:10727000E4B21428EDD310BD2DE9F047D74E002518
:10728000B570C54FB87901284AD0387850B13570FB
:107290004FF4FA730022C1A1CCA0FEF7A6FFC820CC
:1072A00001F016F938784FF47A78012823D10020BC
:1072B000FFF715F8C82001F00BF9B7494A31A1F1E1
:1072C0004000FFF722F84FF480690FE00020FFF73D
:1072D000E1FD01464A46C24815F0ADFAAFA1C148EA
:1072E00015F054FA38B9404601F0F2F82046641C13
:1072F000E4B20528EAD3787801280ED1FFF726F802
:10730000404601F0E5F84346B7A2A4A1B8A0FEF7B5
:107310006CFFC82001F0DCF8B570BDE8F04747E726
:10732000BDE8F08710B5AD4CE078012805D1FFF736
:10733000A3FFF1F78DFE0020E07010BD8CB014208B
:107340000990A64C00262670E670934F0420F87131
:1073500078884FF6FF78002801D0404502D14FF4DD
:10736000FB7078808C48B97A0A300B90FF2906D1DF
:10737000F87AFF2803D140210B9815F0DBFA8648F4
:1073800097F84A104A300A90FF2907D197F84B0026
:10739000FF2803D120210A9815F0CCFAB88808B14B
:1073A000404502D14BF6C020B8807B480A2206A98E
:1073B0004088FEF785FDFEF795FE4FF4FA673846E4
:1073C00001F086F8FEF79BFE384601F081F8FEF7E3
:1073D00065FF089008980127022802D06E4887713F
:1073E00007E06D48052181710020FEF778FFFFF767
:1073F00043FFDFF8EC81052001F06AF8F8F773FB32
:1074000008980228F7D1DFF890A19AF80600022820
:107410004FD09AF8010038B98AF86A608AF86B6030
:107420008AF86C608AF86D60207840B94FF4FA737E
:1074300000225AA161A0FEF7D8FE00B12770207883
:1074400098B34FF00009FFF7F8F88AF806006420B7
:1074500001F03EF8F8F747FB9AF80600032806D932
:10746000484609F101091FFA89F9C828EBD3B9F197
:10747000C80F02D3FFF700FFBDE78AF80060402184
:107480000B9815F057FA20210A9815F053FA5A482C
:10749000477107F0B9FF4FF4FA7300223FA14BA0E8
:1074A000FEF7A3FE642001F013F8C82001F010F8E5
:1074B000A1E7A07830B34FF4806949464F4815F0F2
:1074C00039FA4946464815F035FA0020FFF7E2FC44
:1074D00001464A46424815F0AEF998F807003038A0
:1074E00000F0FF0945493E48FFF798FD02461000AD
:1074F0004FD0A9F1020002284CD840490878EE2864
:1075000049D0C4E0244928226A3101F10C00FFF778
:10751000F8F860B19AF86A0040B99AF86B0028B997
:107520009AF86C0010B99AF86D00C8B1A7700020E5
:10753000FFF7CCF94FF4FA794B46002217A130A09F
:10754000FEF753FE0120FEF76BFFF8F7CCFA4B462F
:10755000002212A112A0FEF748FE4FF0000903E03E
:10756000A670E4E7F8F7BFFA0096BAF80410022311
:107570000A4627A0FFF711F830B9484609F101097A
:107580001FFA89F90528EDD34FF0000940F2D24ADD
:1075900048E09FE09FE06BE0872200204F4B000017
:1075A00041542B434950434C4F53453D3500000057
:1075B00041542B524553544F5245000041542B43E4
:1075C000575354415254534D4152540041542B434C
:1075D0005753544F50534D4152540000A2020020C3
:1075E0009F1600205412002072656164790000002B
:1075F00041542B52535400005D040020871E00208C
:1076000041542B4349504D4F44453D30000000004C
:107610003235352E3235352E3235352E3235350070
:10762000F8F761FA514602230A46AFF21C000097B0
:10763000FEF7B3FF30B9484609F101091FFA89F98D
:107640000528EDD34FF0000901E0F8F74CFA09AA3C
:1076500006A90120FEF7CEFF00287FF40DAF4846B3
:1076600009F101091FFA89F90528BFF405AFECE714
:10767000487810280BD1887848B9C87838B9087983
:1076800028B9487918B9887908B9C87938B17D4AD4
:107690008879927990420CD0FF2807D08DE07F2125
:1076A0000B20FAF79DF8F1F7D3FC86E0C87919288A
:1076B00010D07549052006F04BFBE28842B198F8DE
:1076C000070072493038C3B20020FFF793FBE68011
:1076D000FFF728FE71E0B9F1000F03D0B9F1010FF7
:1076E0001CD06AE00023684901A800970BF0E3FC76
:1076F0000246501EB0F5FF7F5FD80123624901A802
:107700000DF02BFCA288EAB398F8070060493038E6
:10771000C3B20020FFF76EFBA6804EE0DFF868E101
:107720009EF80000642848D1677000219AF86A30FA
:107730009AF86BC09AF86C909AF86DA0C2F3850B1A
:1077400010E00EEB810042789A4209D182786245BE
:1077500006D1C2784A4503D10079504500D1667000
:10776000491CC9B25945ECD3607858B10020FFF7E5
:10777000B9FC48498E77CE7781F8206081F8216086
:10778000002000E019E03F4A01EB000C131893F8C9
:1077900048338CF82530401CC0B21428F4D311F8BB
:1077A0003E0F40F00200087098F807004022303881
:1077B000C3B238490020FFF71DFB28466D1CADB24F
:1077C000B0F5967F7FF658AE00250120FFF77EF8D2
:1077D00002287FF451AEA6700DE610B58CB00121E1
:1077E0000220F8F7ADFA2C4C2046F1F7B5F94FF42A
:1077F000167004901020039000210B91274A0292EA
:107800000891802206922020099025480190079136
:10781000059180140A9001A92046F1F714FA0CB0E2
:1078200010BD70B504461E4D01222D1F8021284633
:10783000F9F786FA2146184C2046F1F745FA01215E
:107840002046F1F72AFA174E3046F1F742FA00289F
:10785000FAD03046F1F74CFA00212046F1F71DFA34
:107860002846BDE8704000228021F9F769BA10B5BA
:107870000C4601462246094814F0DDFF2046FFF77A
:10788000D0FF10BD607F0020871E0020931C0020C9
:107890009F1A00205616002058040240032300209F
:1078A000044C00400000021070B50024F74D04EBBA
:1078B000840005EB800000F0F9FB641C052CF6D376
:1078C000F248643000F0F2FBF048783000F0EEFB54
:1078D000EE488C3000F0EAFBEC48A03000F0E6FB0C
:1078E000EA48B43000F0E2FBE849E948643141631A
:1078F0001431816370BD70B504461546102204F141
:10790000340015F060F8002084F84300052D00D302
:107910000425E562201D00F0D4FB04F1180000F0FE
:10792000D0FB2461C5F10500A061646270BD70B533
:1079300006460D46442000F04FFC044644B1B60014
:1079400045B12846206348B1A522314614F0EAFF2C
:10795000204670BD304600F03FFCF3E7204600F0C3
:1079600091FC0024F4E72DE9FF4F81B08246DDE968
:107970000E68109917469B463846FFF7D8FF044615
:10798000C34DECB3216B781E01EB800020F007099A
:10799000009732462046119B0299FFF7ACFF5A46EA
:1079A0005146484600F0C8FB2060B8F1000F01D0F6
:1079B000C8F8004000F0EBFBA868401CA8602868ED
:1079C00010B1A86938B10BE02C60A868012807D174
:1079D000FFF76AFF04E02868C06AB04200D82C6054
:1079E000E06A2969884200D92861E96A491CE9628C
:1079F0006969884200D9686100EB8001A34800E012
:107A000008E000EB8100211D00F05EFB012400F086
:107A1000C6FB01E04FF0FF34012C07D1A86928B163
:107A20002868C06AB04201D200F0ABFB05B0204626
:107A3000BDE8F08F70B5054600F0A9FB944E3068A4
:107A4000854200D10025FDB12C46201D00F062FBCF
:107A5000A06A18B104F1180000F05CFB8B48211DEE
:107A6000A03000F031FB7068401C7060F06A401C70
:107A7000F06200F094FBB069002807D0002D05D11A
:107A8000BDE8704000F07DBB3468DEE770BD70B5C6
:107A90007F4DE869002803D0286A401C286270BD29
:107AA000E868401CE860E8684FF0FF3670B9686B22
:107AB000A96B6963A863A86A401CA862686B006828
:107AC000A0B1686BC068C06840682863E868296B2B
:107AD0008842E4D3686B006850B1686BC068C468C2
:107AE0006068E968814205D2286370BD2E63EDE7C6
:107AF0002E6370BD201D00F00DFBA06A18B104F1CB
:107B0000180000F007FBE06A6969884200D96861E3
:107B10005E4900EB800001EB8000211D00F0D4FAEB
:107B2000D8E72DE9F041002700F031FB584EF0690D
:107B3000401EF061F069E8BBB068D8B30025DFF8FB
:107B40004C8108F18C081CE0D8F80C00C46804F1E2
:107B5000180000F0DFFA201D00F0DCFAE06A71691D
:107B6000884200D97061494900EB800001EB800038
:107B7000211D00F0A9FAE06A3168C96A884200D381
:107B80000125D8F800000028DED1306A28B908E0C5
:107B9000FFF77DFF306A401E3062306A0028F7D15F
:107BA0000125012D02D0706A012806D1012700208D
:107BB000706200E001E000F0E4FA00F0F0FA38460C
:107BC000BDE8F08170B50446314D28684460E8682E
:107BD000844206D22968A86B091DBDE8704000F0F8
:107BE00081BA2968686B091D00F07CFA286B844211
:107BF00000D22C6370BD2648C169491CC161704721
:107C000070B503460C460022FFF7F5FF18680444E0
:107C10001F49CD68A84206D9A0420AD9C868844243
:107C200007D9012205E0A04202D8C868844200D9E1
:107C300001221C6032B10868001D00F06BFA20467A
:107C4000FFF7C0FFFFF76DFF002803D1BDE87040CC
:107C500000F097BA70BD10B502460020002A0DD082
:107C6000FFF7C9FF0A48C1688C180068001D00F0C2
:107C700051FA2046FFF7A6FFFFF753FF002803D174
:107C8000BDE8104000F07DBA10BD00005C2500206A
:107C9000AC02002010B5044600F079FA0CB9F748A0
:107CA0000468E46A00F07BFA2046EDE72DE9F04134
:107CB00006460D460027052D00D3042500F067FA7F
:107CC000DFF8B883D8F80000864200D1002646B11C
:107CD0003446E06AA8422AD0854205D936B1012748
:107CE00004E0D8F80040F4E706B90127E562C5F1E1
:107CF0000501A161E24D00EB8000616905EB8000A8
:107D0000814210D1201D00F005FAE06AD8F8141065
:107D1000884201D9C8F8140000EB800005EB800010
:107D2000211D00F0D1F9012F01D100F02AFABDE8A0
:107D3000F04100F034BAD149C869002802D00120CE
:107D400048627047CE4A02E04869401E486148696F
:107D500000EB800052F820000028F5D0486900EBC5
:107D6000800002EB800042685268426000F1080324
:107D70009A4201D1526842604068C068086070470A
:107D800070B5054600F003FABC4E3068854200D15C
:107D90000025C5B12C46201D00F0BCF9A06A18B121
:107DA00004F1180000F0B6F9B548211DB43000F018
:107DB0008BF900F0F4F9002D0FD1B06928B1BDE8BE
:107DC000704000F0DEB93468E5E7AD48B4300068D3
:107DD000B168884202D10020306070BDBDE87040BB
:107DE000A9E70021A64B4269B4339A4206D1806AC2
:107DF000A3F12802904201D000B901210846704742
:107E000070B50446002C25D09C4D2868844221D0B2
:107E100000F0BDF92046FFF7E4FF012816D1201D30
:107E200000F078F9E06A6969884200D9686194498C
:107E300000EB800001EB8000211D00F045F9E06AB5
:107E40002968C96A884201D300F09BF9BDE87040F7
:107E500000F0A5B970BD70B5044600252046FFF7B7
:107E6000C0FF012808D1854EF06938B1844804F17B
:107E700018018C3000F028F9284670BDE06A31689E
:107E8000C96A884201D3012500E00025201D00F0C9
:107E900041F9E06A7169884200D97061784900EB64
:107EA000800001EB8000211D00F00EF9E4E710B521
:107EB0000446206B00F0E6F92046BDE8104000F0D3
:107EC000E1B970B56D4D686800281FD0FFF793FECB
:107ED0006B4EA0363068B8B10024FFF722FE002CAC
:107EE00014D100F054F9F068C468201D00F012F9B4
:107EF000A868401EA8606868401E686000F04FF9DE
:107F00002046BDE87040D2E70124E6E770BD5C4C36
:107F1000FFF7D7FF20680128FAD900F032F9F7E718
:107F20001FB500240094019402942346642255A1B5
:107F300056480394FFF717FD012809D1F0F7C4F95B
:107F40004E4801218161C460BDE81F4000F005B9C1
:107F50001FBD10B5F0F7B8F9484900208861BDE8A9
:107F6000104000F00DB910B500F011F94348C46895
:107F700000F015F9204687E610B5F0F7A5F93F485F
:107F8000C468F0F7A8F920467EE63C488068704750
:107F900070B50D46394C2168183100F0A3F82068FF
:107FA000001D00F0B7F8681C04D0E0682844BDE864
:107FB000704007E62168BDE870403148091DB430C3
:107FC00000F082B870B5C068C46804F118000646B5
:107FD00000F0A0F8294DEA695AB1294831468C30A1
:107FE00000F072F8E06A2968C96A884212D3012059
:107FF00070BD201D00F08EF8E06A6969884200D9E2
:1080000068611F4900EB800001EB8000211D00F03A
:108010005BF8E7E7002070BD18498A6A0260C9680A
:108020004160704770B504460D4600F0B0F828680E
:10803000411C0AD0114B21689A6A914207D06168AD
:10804000DA68914203D8012410E000240EE062684F
:10805000D968891A814208D2D968891A401A2860D9
:108060002046FFF7D9FF002400E0012400F097F834
:10807000204670BD0149012048627047AC020020D3
:108080005C25002049444C45000000000F7F01089A
:1080900005488169002903D0C06918B10220ECE7C6
:1080A0000020EAE70120E8E7AC02002000F1080127
:1080B00041604FF0FF328260C160016100210160C8
:1080C0007047002101617047426853684B60436804
:1080D0008B60536899605160416008610168491C78
:1080E0000160704710B50B685A1C02D000F10802FD
:1080F00002E0026904E05268546824689C42FAD99C
:1081000053684B6099608A60516008610168491C3E
:10811000016010BDD0E901219160D0E901125160E8
:1081200001694A68824201D182684A600022026184
:108130000868401E0860704720384FF08073C361A4
:1081400081610021416140F8202970474FF0E02013
:108150001E49416107210161704710B51C48016843
:1081600041F47F010160016841F07F410160FFF748
:10817000EDFF184900200860F0F77EF8002010BDE0
:10818000704713494FF080501C390860704710B594
:10819000F0F79AF80F480168491C016010BD0D49BD
:1081A0000868401E0860002801D1F0F794B87047B5
:1081B00010B507494FF080501C390860F0F784F87B
:1081C000FFF765FCBDE81040F0F785B83F190100E6
:1081D00020ED00E0E80200202DE9F04104460025F2
:1081E000FFF709FD384E06F10801706801F1080338
:1081F00060B936480860002048604FF4A0425A60D9
:108200001860324842600360012070603CB1103455
:10821000600704D004F00700C0F108000444601EA9
:1082200044F6FF72904228D2274A0832096801E0DA
:108230000A4601464868A04202D208680028F7D1E1
:1082400099421AD015681035086810604868001BFC
:1082500020280ED90B1958604C605C681A48083009
:1082600000E0104602685768A742FAD302681A6015
:10827000036048683168081A3060FFF752FC2846EE
:10828000BDE8F08110B5002818D010380446FFF77B
:10829000B2FC60680C49083100E011460A68536876
:1082A0008342FAD3086820600C600748616802685E
:1082B00011440160BDE81040FFF733BC10BD024817
:1082C0000068704770470000EC020020282600205C
:1082D000704770B504465F4D40212846F8F7D7FD3A
:1082E0000028F9D0A1B22846F8F764FD204670BDF9
:1082F000F0B587B00546012144F20400F7F72BFDE5
:10830000544E3046F8F732FC7015ADF818000320D3
:108310008DF81A0018208DF81B004F4F06A938461B
:10832000F0F777FD3015ADF8180048208DF81B00E8
:1083300006A93846F0F76DFDB415ADF818401020C9
:108340008DF81B0006A93846F0F763FD2146384634
:10835000F0F7CEFD25208DF8040000248DF80540AF
:108360008DF8064001208DF8070001A8F0F7D9F933
:108370000295ADF80C40ADF80E40ADF81040ADF8E8
:1083800014400C20ADF8120002A93046F8F736FC74
:10839000012240F225513046F8F7B7FC0121304662
:1083A000F8F7A7FC07B0F0BD70B586B0054601210F
:1083B0001020F7F7D0FC01212020F7F7CCFC012199
:1083C0000805F7F7D3FC254E3046F8F7CFFBB0147D
:1083D000ADF8140003208DF8160018208DF8170052
:1083E00005A91F48F0F715FD0420ADF8140048203A
:1083F0008DF8170005A91B48F0F70BFD35208DF807
:10840000000000248DF801408DF8024001208DF815
:1084100003006846F0F785F90195ADF8084070143F
:10842000ADF80A00ADF80C40ADF810400C20ADF8E6
:108430000E0001A93046F8F7E1FB012240F2255178
:108440003046F8F762FC01213046F8F752FC06B0DE
:1084500070BD00000038014000080140005000409D
:1084600000100140001401404FF0E0210A6922F0A1
:1084700004020A61224AC00810704FF47A7358430C
:10848000012353804861086940F00100086170478A
:108490002DE9F04100244FF0E0277E690546184899
:1084A00000784543FFF773FEBA69B9699142FCD081
:1084B00003D2A2EB0100044403E0A6EB0100104448
:1084C00004440A46AC42F0D3BDE8F041FFF767BE72
:1084D00070B50446FFF7DCFD60B1094D6888844241
:1084E00003D3B4FBF0F0FFF7B6FB6888B4FBF0F100
:1084F00000FB11444FF47A706043BDE87040C7E759
:1085000004030020FE49FF200870FE4908707047F0
:10851000FD4900200860FD4948734875012240F27A
:108520002551FB48F8F7F1BB10B5F84CA07B801E35
:10853000C1B2F84805F054FCF649A27BA37B0A447B
:1085400012F8012C194411F8021C02EB012181429E
:1085500001D1012010BD002010BD2DE9F05FDFF832
:10856000B08340F225514046F8F79CFCDFF8A8A301
:1085700001270026DFF8A493E44C012829D040F21B
:10858000277529464046F8F78DFC012855D18AF811
:10859000077099F80610032901D000294DD1A28B4C
:1085A000608B824273D340214046F8F770FC00286C
:1085B000F9D040214046F8F771FC00222946404698
:1085C000F8F7A3FBA683FFF7A3FFBDE8F05F0CF06D
:1085D00061BD8AF8087099F8061003290AD00029AD
:1085E0002BD14046F8F7EAFBC1B2BDE8F05FCC48BA
:1085F0000CF06CBC607BC74DDC2807D24046F8F716
:10860000DDFB617B4A1C6273685401E0FFF780FF69
:10861000607B01280DD0607B042810D0607B072888
:108620001CD0607BDFF8FC824FF00309062841D0A4
:1086300043E05020A073207DE074BDE8F09FE8780F
:10864000A97800EB01200A28F7D168780628F4D130
:108650000C20A073207D0830E074EEE768780328D2
:1086600016D0062814D010281DD029785529E4D119
:10867000FF28E2D1A8780128DFD168790028DCD171
:10868000A8790028D9D1277005206070D5E769E066
:10869000E878A97800EB01200A28CED00820A07342
:1086A000207DE074C9E7A87900F10901A1730830C1
:1086B000E074C2E76878192828D0607BA17B8842E3
:1086C000BBD16878032803D0062801D01028B4D184
:1086D0002878DFF854B2FF2803D09BF806108842B0
:1086E0003DD1FFF721FFB0B3A078012824D08AF84C
:1086F00008709BF8D80030B18C49C0EB00108000A6
:1087000008808B480670E67400201DE0208B00284E
:1087100093D1607A002890D0607BA073E67484F8CF
:108720001590002004E0295C08F80010401CC0B23D
:10873000A17B8842F7D380E7BDE8F05FE8E6295CDB
:1087400008F80010401CC0B2A17B8842F7D384F81F
:108750001590277271E7FFE7BDE8F05FD8E6BDE846
:10876000F05FD5E6501CA0837248815C4046F8F764
:1087700021FBBDE8F05F0CF08DBC70B56E4D40F292
:1087800025512846F8F78EFB6C4CB8B12846F8F70F
:1087900015FBC2B2B4F8000440F2FF31C0F30E0082
:1087A00088420BD2B4F80004B4F80034C0F30E01D0
:1087B000481C60F30E03A4F80034625440F22441D4
:1087C0002846F8F76FFB01280AD194F8010440F01D
:1087D000800084F801042846BDE87040F8F7EEBA3E
:1087E00070BD49490120086070474849488301220B
:1087F00040F227714648F8F788BA10B5FFF788FEAF
:1088000042480A210175C17410BD70B54C4B012559
:108810004C4E5418B0F5FA6F2DD0A0F5E061D33965
:1088200019D0891C32D0091F33D0491C37D0C91E3A
:108830003BD0C91E1F2943D8C80629D103F10A001D
:108840004021054614F076F8E11D2846BDE8704049
:10885000402213F0F0BF6079012819D1FEF7C8FC5F
:108860007C21374814F066F8757106F0CDFDBDE83F
:108870007040F0F7EDBB60791870757106F0C4FDBB
:10888000FEF7B6FCBDE87040F0F7E2BB60795870C7
:1088900070BD6079217900EB0120988070BD60790E
:1088A000217900EB0120588070BD6079012803D048
:1088B000BDE87040FEF7CABCBDE87040FEF7B0BC32
:1088C000A0F2FA710F290ED80807EDD11C4820211B
:1088D0004A30054614F02EF8E11D2846BDE87040E8
:1088E000202213F0A8BFA0F500610A39DCD1A0F660
:1088F0000A000C2190FBF1F201FB1200002823E09A
:10890000C0030020C1030020A00121420803002071
:108910000038014054770020961100209616002060
:10892000CCA5002054790020607F00205C0000204E
:108930005A000020547B0020004C004054120020BC
:10894000872200205D040020AED1207A03F86A0F50
:10895000A07A5870207B9870A07BD870207C18710A
:10896000A07C5871207D9871A07DD871207E1872EE
:10897000A07E5872207F9872A07FD87270BD2DE9BA
:10898000FF5F0446DFF814A44FF001088AF8028064
:10899000002902D0042900D0A41DE078A17800EBC2
:1089A000012085B26178FE4F10291ED11FFA80F98F
:1089B000A079182801D91820A071A9F2B3100728AE
:1089C00014D800260EE004EB060906F2911099F87F
:1089D0000710F8F705FFB91999F8070081F8910118
:1089E000761CF6B2A079B042EDD8CFE1A9F2BB1067
:1089F00003903F2870D8002688E0039804EB060B0C
:108A000006EB400000F2A1109BF8071080B2F8F7C7
:108A1000E7FEA9F58070BF381CD0001F20D0001FD2
:108A200024D0001F28D0001F2CD0001F30D0001FE2
:108A300034D0001F38D0001F3CD0001F40D0001F92
:108A400044D0001F49D0001F4DD0001F51D0001F3F
:108A500055D059E0B9199BF8070081F8A90153E0F6
:108A6000B9199BF8070081F8B1014DE0B9199BF8DD
:108A7000070081F8B90147E0B9199BF8070081F8B0
:108A8000C10141E0B9199BF8070081F8C9013BE039
:108A9000B9199BF8070081F8D10135E0B9199BF8A5
:108AA000070081F8D9012FE0B9199BF8070081F878
:108AB000E10129E0B9199BF8070081F8E90123E0F9
:108AC000B9199BF8070081F8F1011DE0B9199BF86D
:108AD000070081F8F90117E01DE0B9199BF80700BC
:108AE00081F8010210E0B9199BF8070081F809022A
:108AF0000AE0B9199BF8070081F8110204E0B919DE
:108B00009BF8070081F81902761CF6B2A079B042F2
:108B10003FF673AF3AE1A9F2E120029013281CD886
:108B2000002613E0029804EB060B06EB400909F25D
:108B300081309BF8071080B2F8F752FE09EB07016D
:108B40009BF8070081F88103761CF6B2A079B04249
:108B5000E8D8944880F8028018E1A9F2CB200928CF
:108B600014D800260EE004EB060906F5527099F8B9
:108B70000710F8F735FEB91999F8070081F848038E
:108B8000761CF6B2A079B042EDD8FFE0A9F5CD7021
:108B900006280FD80A208AF80700207DA17CCDE99D
:108BA0000010207A237CA27BA17A00F5FA60F8F706
:108BB00022FFEBE0A9F22D30DFF8ECB10B2817D83B
:108BC00000260EE004EB460906F2B53099F80810CD
:108BD000F8F706FEB91999F8080081F8B503761C74
:108BE000F6B2A079B6EB500FECD38BF80080CDE055
:108BF000A9F239300B2817D800260EE004EB4609FD
:108C000006F2C13099F80810F8F7EAFDB91999F899
:108C1000080081F8C103761CF6B2A079B6EB500FBC
:108C2000ECD38BF80080B1E0A9F245300B2817D8BF
:108C300000260EE004EB460906F2CD3099F8081044
:108C4000F8F7CEFDB91999F8080081F8CD03761C24
:108C5000F6B2A079B6EB500FECD38BF8008095E01C
:108C6000A9F251300B2817D800260EE004EB460974
:108C700006F2D93099F80810F8F7B2FDB91999F849
:108C8000080081F8D903761CF6B2A079B6EB500F34
:108C9000ECD38BF8008079E0A9F25D300B2817D86F
:108CA00000260EE004EB460906F2E53099F80810BC
:108CB000F8F796FDB91999F8080081F8E503761CD4
:108CC000F6B2A079B6EB500FECD38BF800805DE0E4
:108CD000A9F269300B2817D800260EE004EB4609EC
:108CE00006F2F13099F80810F8F77AFDB91999F8F9
:108CF000080081F8F103761CF6B2A079B6EB500FAC
:108D0000ECD38BF8008041E0A9F275300B2817D81E
:108D100000260EE004EB460906F2FD3099F8081033
:108D2000F8F75EFDB91999F8080081F8FD03761C83
:108D3000F6B2A079B6EB500FECD38BF8008025E0AB
:108D4000A9F281300B2817D800260EE004EB460963
:108D500006F2094099F80810F8F742FDB91999F898
:108D6000080081F80904761CF6B2A079B6EB500F22
:108D7000ECD38BF8008009E0A9F5FA60642805D8E7
:108D80000023224619464846FFF73FFD60784FF022
:108D90000009062842F05B87F5B307E008030020CE
:108DA000607F00209611002028000020022D7CD03A
:108DB000DFF840B4062D79D0102D78D0082D77D06B
:108DC0000E2D76D0142D75D00A2D74D0162D73D09B
:108DD000172D72D0A5F5407022386FD0401E6ED08E
:108DE000652D6DD0672D6CD0682D6BD0692D6AD044
:108DF0006A2D69D06B2D68D06C2D67D0DFF8F8B381
:108E0000FE486D2D72D00F2D71D06F2D70D0712D49
:108E10006FD0DFF8ECB300E078E0722D6AD0732DEC
:108E200069D0742D68D0752D67D0782D7DD0152D23
:108E30007CD0792D7BD0822DFCD04FF0080B7A2D81
:108E400076D07B2D75D07C2D74D07D2D73D07E2D6A
:108E500072D07F2D71D0802D70D0812D6FD0A5F173
:108E6000830BBBF1070F6BD86079217900EB0120F0
:108E700086B20BF0FF01E348F1F732FE002870D014
:108E800007EB4B0595F86B0395F86A1300EB01208F
:108E9000B04202F0D08640F26A3000EB4B002179FC
:108EA00080B2F8F79DFC617911E05BE078E0AFE01B
:108EB000CDE0E0E0E6E0F6E026E12CE11EE034E182
:108EC0003BE14DE157E166E16CE172E178E140F2AE
:108ED0006B3000EB4B0080B2F8F782FC207985F80C
:108EE0006A03607985F86B0302F0A5BE6FE100E2CA
:108EF00009E215E21CE26AE2BCE2EFE2617987F87E
:108F0000271340F22730F8F76BFCEDE79AF80A00D8
:108F1000C107E9D1617939702179797040F0010098
:108F20008AF80A00617900200BE0E8E205E332E309
:108F30008AE397E3A4E3B1E3BEE3CBE3D8E3E5E35D
:108F4000F2E3F8F74DFC21790120F8F749FC9AF893
:108F50000A104FF45A70F8F743FC0D208AF8070006
:108F6000C2E7E2E39AF80A008107BDD46179B970DB
:108F70002179F97040F002008AF80A006179022034
:108F8000F8F72EFC21790320F8F72AFC9AF80A104A
:108F90004FF45A70F8F724FC0E208AF80700A3E774
:108FA000607997F8CF1088429ED397F8D110884205
:108FB0009AD89AF80B00012807D097F8F30220B14D
:108FC0008AF80B808AF80C908EE787F8F39240F2CB
:108FD000F32500212846F8F703FC61790620F8F70D
:108FE000FFFB6079ABF80000012282498648EFF769
:108FF000E6FA6079B87160798AF80F0087F8F38231
:1090000001212846F8F7ECFB0C208AF80700D9E785
:109010006179F9728E2904D09F290DD07F2910D053
:1090200062E710208AF8070000214FF45A70F8F721
:10903000D7FB8AF80A9057E7F4F778FBF3F7D0FBF1
:1090400052E70B20F8F7CCFB8AF807804CE79AF838
:109050000A00000784D4617939720820F8F7C0FB50
:109060009AF80A0040F008018AF80A104FF45A7082
:10907000F8F7B6FB38E7617987F8D710D720F8F70B
:10908000AFFB31E7207987F89702617987F896126C
:1090900040F29620F8F7A4FB97F8971240F2972039
:1090A000F8F79EFB20E7207955280CD0662819D0C8
:1090B000772824D0607987F87701617940F27710BA
:1090C000F8F78EFB10E76079B87161790620F8F740
:1090D00087FBB879ABF80000012246494A48EFF710
:1090E0006EFA01E7607938B1C0EB00108000AAF891
:1090F00018008AF80980F7E68AF80990F4E6AAF8D9
:1091000018908AF80980EFE66079012888D1162046
:109110008AF80700E8E6617901298CD93B4801709B
:1091200040F29C40F8F75CFBDEE6617987F8281393
:109130004FF44A70F8F754FBD6E6617987F8A91323
:1091400040F2A930F8F74CFB87F86B9000216B20B8
:10915000F8F746FB2E4880F8058080F80380C3E6C8
:10916000617987F86A106A20F8F73AFB294997F87D
:109170006A000870B8E697F86E006179884291D06D
:1091800087F86E106E20F8F72BFB214880F80080DE
:10919000F2F7E3FCA8E6617987F86F106F20F8F723
:1091A0001FFBA1E6617987F878107820F8F718FBA3
:1091B0009AE6617987F87A107A20F8F711FB93E63E
:1091C000607901288DD102208AF807008CE697F893
:1091D0009E1204295DD097F89F12042959D0617915
:1091E0000E4ACB070C492ED081F80080797A41F0E5
:1091F000010115E0500000204C0000202C00002050
:109200009600002034800020007700085C040020D5
:1092100096110020770000203A0000206E00002008
:109220007972FA4B197839B997F8631021B1C1EB0B
:1092300001118900CBF800100421197087F89B10E8
:109240000170117013E081F80090797A01F0FE014D
:109250007972EE4981F8009087F89B9080F8009031
:10926000EB4880F80090CBF8009082F80090E94835
:1092700080F8028080F8048080F80180797A0920E3
:10928000F8F7AEFAE148017887F89B109B20F8F7D1
:10929000A7FA60798AF81200797A00F0040201F0E6
:1092A00004039A420CD0400706D541F004017972BC
:1092B0000920F8F795FA03E0F2F7CAF9F3F790FA04
:1092C0006079800607D5787A40F020007872042013
:1092D0008AF8160006E0787A00F0DF007872022043
:1092E0008AF81600797A0920F8F77AFAF0F752FA34
:1092F000FAE5617987F865106520F8F771FA0420BE
:109300008AF80700F0E5617987F863106320F8F7C1
:1093100067FA6079C0EB00108000CBF80000E3E54D
:1093200061796B20F8F75CFA607987F86B00DBE510
:10933000207987F8CC00607987F8CB002179CC20A0
:10934000F8F74EFA6179CB20F8F74AFA217909B992
:109350006079B8B397F8DB00012801D002280CD15E
:10936000CE20F8F73DFA207987F8CE006179CD203C
:10937000F8F736FA607987F8CD0097F8CD0097F8BE
:10938000CE1000EB012080B2ABF80000A24981F8BA
:109390000090A24981F8008010B1A14981F80080B5
:1093A00097F8DB10032907D19D4981F800909D496A
:1093B00081F8008081F8018097F8D3100122F4F73A
:1093C0008DFD91E5FFE7964880F800908CE52079C7
:1093D00087F8CE00607987F8CD002179CE20F8F7A4
:1093E000FFF96179CD20F8F7FBF9217909B96079A6
:1093F000D8B397F8DB00012801D002280CD1CC208B
:10940000F8F7EEF9207987F8CC006179CB20F8F7EE
:10941000E7F9607987F8CB00CC377878B97800EB3A
:10942000012080B2ABF800007B4981F800907B49B5
:1094300081F8008017F8CC1911B997F8CB1011B149
:10944000774981F8008097F8DB10032907D1744928
:1094500081F80090734981F8008081F8018097F8C5
:10946000D3100122F4F73AFD3EE5FFE76C4880F89F
:10947000009039E5607987F8DB0097F8CC1011B9D6
:1094800097F8CB1059B197F8CE1011B997F8CD20B5
:109490002AB1032807D0624880F800800BE06048BA
:1094A00080F8009020E55E4880F800905D4880F8E4
:1094B000008080F80180594880F80080564880F884
:1094C000009097F8CD0000EB012080B2ABF80000CF
:1094D00097F8D3100122F4F701FD05E5617987F8CB
:1094E000D810D820F8F77CF997F8D800C0EB001016
:1094F00081004D4801804D4880F80090F4E4607987
:1095000001280BD0022810D000218220F8F768F93A
:1095100087F8829009208AF80700E5E4012182207B
:10952000F8F75EF987F88280F4E702218220F8F7E5
:1095300057F9022087F88200ECE760793C4D01285A
:1095400018D10B208AF807009AF8030090B985F823
:10955000069087F8928001219220F8F741F90021C6
:10956000D620F8F73DF987F8D69005F066FE002082
:109570000BF062FD6079002894D10320A87187F870
:10958000929004208AF8070000219220F8F728F929
:10959000EFF75EFDA8E400212648F1F7A1FA30B10B
:1095A000207987F87A03607987F87B039CE4207937
:1095B000617901EB002081B297F85F00022804D0A6
:1095C000132802D0042816D08EE41B481B4C0088B8
:1095D000081A2080C1B25B20F8F702F92088C0F396
:1095E00007215C20F8F7FCF8208887F85B00000A68
:1095F00087F85C0078E412480078081A114908706E
:10960000C1B25D20F8F7ECF86EE400003B000020EA
:10961000D8000020961100208C000020D9000020E6
:109620007E000020AD0000205C0000205A000020D9
:1096300096160020358000207A0200206402002067
:10964000720200203C0200206179E520F8F7C8F89A
:10965000607987F8E500FE4880F800B0FD4880F8A2
:1096600000B041E46179E620F8F7BAF8607987F84C
:10967000E600F74880F800B0F64880F800B033E420
:109680006179E720F8F7ACF8607987F8E700F048EF
:1096900080F800B0EF4880F800B025E46179E82058
:1096A000F8F79EF8607987F8E800E94880F800B09C
:1096B000E84880F800B017E46179E920F8F790F8FD
:1096C000607987F8E900E24880F800B0E14880F866
:1096D00000B009E46179EA20F8F782F8607987F848
:1096E000EA00DB4880F800B0DA4880F800B00CE40B
:1096F0006179EB20F8F774F8607987F8EB00D448CB
:1097000080F800B0D34880F800B029E46179EC20FB
:10971000F8F766F8607987F8EC00CD4880F800B07B
:10972000CC4880F800B01BE418E0CB48CB4C30F8B4
:109730001B00301A24F81B00C1B2472000EB4B007D
:1097400080B2F8F74DF834F81B00C0F30721482029
:1097500000EB4B0080B2F8F743F820E44FF481723D
:109760008B2D14D08C2D26D08D2D3AD08E2D3FD020
:10977000A5F18F01092943D805F16800617980B20C
:10978000F8F72EF87919607981F8680007E46079B4
:10979000217900EB0120B249B24C0988401A20809F
:1097A000C0F307211046F8F71BF8217840F20110AA
:1097B000F8F716F808E46079217900EB0120AA494E
:1097C000AA4C0988401A2080C1B240F27D30F8F7D7
:1097D00007F82088C0F3072140F27E30F8F700F840
:1097E0001EE4617987F8D410D420F7F7F9FF17E465
:1097F000607987F8600061796020F7F7F1FF0FE486
:10980000992D22D09A2D28D09B2D3AD09C2D4CD02A
:109810009D2D5ED09E2D76D09F2D6FD0A02D6ED029
:10982000A12D6DD0A22D6CD06CD1207987F8560077
:10983000607987F8550061794FF05100F7F7D0FF54
:1098400021795220F7F7CCFF14E489496079087038
:10985000C1B25D20F7F7C4FF0CE4257961795B376D
:109860007D7039705B20F7F7BBFF29465C20F7F766
:10987000B7FF397878785B3FF1F7A4F97D49088024
:1098800010E42579617947377D7039704720F7F703
:10989000A7FF29464820F7F7A3FF38787978473F94
:1098A00000EB01216D4801800CE42579617949378D
:1098B0007D7039704920F7F793FF29464A20F7F762
:1098C0008FFF38787978493F40EA01206349488022
:1098D00007E4257961794B377D7039704B20F7F7B4
:1098E0007FFF29464C20F7F77BFF387879784B3F8C
:1098F00040EA01205949888005E404E017E02BE0A4
:109900003FE053E067E0257961794D377D7039702C
:109910004D20F7F765FF29464E20F7F761FF3878AD
:1099200079784D3F40EA01204C49C88004E44F3724
:10993000207978706079387061794F20F7F750FF9F
:1099400021795020F7F74CFF387879784F3F40EA7B
:109950000120424908810DE45137207978706079FF
:10996000387061795120F7F73BFF21795220F7F7E2
:1099700037FF38787978513F40EA012137484181F3
:1099800008E4533720797870607938706179532012
:10999000F7F726FF21795420F7F722FF38787978F6
:1099A000533F40EA01202D49888108E4553720794A
:1099B00078706079387061795520F7F711FF217957
:1099C0005620F7F70DFF38787978553F40EA0120A7
:1099D0002249C8818CE4A72D68D0A82D76D0A92D66
:1099E0006ED0AA2D6DD0AB2D6CD0AC2D6BD0AD2D23
:1099F0006AD0AE2D69D0DFF880B0AF2D6FD0B02D1A
:109A00006ED0B12D6DD0B22D6CD0B32D6BD0B42DE6
:109A10006AD0B52D69D0B62D68D0B72D67D0B82DD6
:109A20006FD0B92D6ED0BA2D6DD0BB2D6CD0BC2DA2
:109A30006BD0BD2D6AD0BE2D69D0BF2D68D0C02D92
:109A400067D0C12D6FD0C22D6ED0C32D6DD015E063
:109A5000450200204602002004120020E0110020F0
:109A60005A020020700200206C00002040000020FC
:109A70003C0200206402002074020020C42D70D03B
:109A8000A5F1CA0104296DD8A5F11100617980B250
:109A9000F7F7A6FE7919607901F8110C6179F84899
:109AA000491E02297ED280F8008021E4607987F87F
:109AB0009E02617940F29E20F7F792FE18E405E0DD
:109AC00016E027E032E03AE042E04CE0607987F8C7
:109AD0009F02617940F29F20F7F782FE08E44BE095
:109AE00068E074E081E08FE09DE0ABE0B9E0C7E0C2
:109AF000607987F8A00261794FF42870F7F770FE5B
:109B00000DE4CCE0DAE0F6E012E120E12EE13CE108
:109B10004AE158E1607987F8A102617940F2A12019
:109B2000F7F75EFE4DE45DE16BE179E1607987F87E
:109B3000A202617940F2A220F7F752FE41E4607977
:109B400087F8A302617940F2A320F7F749FE38E4D1
:109B5000607987F8A40261794FF42970F7F740FE25
:109B60002FE46CE18EE1607987F8A502617940F21B
:109B7000A520F7F735FE24E46079F8762079387768
:109B800061791B20F7F72CFE21791C20F7F728FEBE
:109B9000F87E397F00EB012197F82F0000EB0020C1
:109BA000814200E068E102D28BF8008009E48BF882
:109BB000009006E4607978772079B87761791D2084
:109BC000F7F70EFE21791E20F7F70AFE4CE46079C4
:109BD000F877207987F8200061791F20F7F700FED9
:109BE00021792020F7F7FCFD3EE4607987F8210019
:109BF000207987F8220061792120F7F7F1FD21799A
